S01500006376615F6173775F6D303134362E7372656394
S214010000F0EF0020F17B0200E3690100076A0100BE
S2140100107B8E01006B9A01009BBD010015820200D8
S21401002015820200158202001582020053C00100EB
S21401003073C70100158202006FD80100F96B020038
S2140100401582020015820200158202001582020046
S2140100501582020015820200158202001582020036
S2140100601582020015820200158202001582020026
S2140100701582020015820200158202001582020016
S2140100801582020015820200158202001582020006
S21401009015820200158202001582020015820200F6
S2140100A015820200158202001582020015820200E6
S2140100B0C5C00100158202001582020001D00100B0
S2140100C015820200158202001582020015820200C6
S2140100D015820200158202001582020015820200B6
S2140100E015820200158202001582020015820200A6
S2140100F01582020015820200158202001582020096
S2140101001582020015820200158202001582020085
S2140101101582020015820200158202001582020075
S2140101201582020015820200158202001582020065
S2140101301582020015820200158202001582020055
S2140101401582020015820200158202001582020045
S2140101501582020015820200158202001582020035
S2140101601582020015820200158202001582020025
S2140101701582020015820200158202001582020015
S2140101801582020015820200158202001582020005
S21401019015820200158202001582020015820200F5
S2140101A015820200158202001582020015820200E5
S2140101B015820200158202001582020015820200D5
S2140101C015820200158202001582020015820200C5
S2140101D015820200158202001582020015820200B5
S2140101E015820200158202001582020015820200A5
S2140101F0158202001582020015820200E5C5010083
S2140102001582020015820200158202001582020084
S2140102101582020015820200158202001582020074
S2140102201582020015820200158202001582020064
S2140102301582020015820200158202001582020054
S2140102401582020015820200158202001582020044
S2140102501582020015820200158202001582020034
S2140102601582020015820200158202001582020024
S2140102701582020015820200158202001582020014
S2140102801582020015820200158202001582020004
S21401029015820200158202001582020015820200F4
S2140102A015820200158202001582020015820200E4
S2140102B015820200158202001582020015820200D4
S2140102C015820200158202001582020015820200C4
S2140102D015820200158202001582020015820200B4
S2140102E015820200158202001582020015820200A4
S2140102F01582020015820200158202001582020094
S2140103001582020015820200158202001582020083
S2140103101582020015820200158202001582020073
S2140103201582020015820200158202001582020063
S2140103301582020015820200158202001582020053
S2140103401582020015820200158202001582020043
S2140103501582020015820200158202001582020033
S2140103601582020015820200158202001582020023
S2140103701582020015820200158202001582020013
S2140103801582020015820200158202001582020003
S21401039015820200158202001582020015820200F3
S2140103A015820200158202001582020015820200E3
S2140103B015820200158202001582020015820200D3
S2140103C015820200158202001582020015820200C3
S2140103D015820200158202001582020015820200B3
S2140103E015820200158202001582020015820200A3
S2140103F01582020015820200158202001582020093
S214010400DDCCBBAA31303A34373A31360000000031
S2140104104170722031312032303235000000000048
S2140104205357303130315F3230323530343031006D
S214010430FF000000000000000000000000000000B7
S214010440020010688068C0F34000C0B200280AD0DD
S2140104501068C068C0F34000C0B2002803D010691D
S2140104600860012000E00020704730B4020000233D
S2140104701468A56835F002051800C0B2400010F0F7
S21401048002000543A5600878002812D001201368F1
S2140104909C6834F002040500EDB26D0015F002050B
S2140104A02C439C601068C068C0F34000C0B20028AE
S2140104B0F8D0012030BC7047020010688068C0F395
S2140104C08000C0B200280AD01068C068C0F380005F
S2140104D0C0B2002803D090690860012000E0002027
S2140104E07047F0B5020000231468A56835F00405CE
S2140104F01800C0B2800010F004000543A56008781B
S214010500002842D09069224B984201D2002312E083
S2140105109069204B984201D201230CE090691E4B52
S214010520984201D2022306E090691C4B984201D200
S214010530032300E004231800C0B2042801D10020E0
S21401054024E018001468256835F00C050600F6B29C
S214010550B60016F00C063543256001261768D7F855
S21401056008C03CF0040CB6465FFA8EFE5FEA8E0EBB
S2140105701EF0040E5EEA0C0CC7F808C01068C068CE
S214010580C0F38000C0B20028F8D00120F0BD000002
S21401059000093D0000127A0000366E01015A62021F
S2140105A002001068806810F00100C0B200280AD06E
S2140105B01068C06810F00100C0B2002803D050696E
S2140105C00860012000E00020704730B402000023DC
S2140105D01468A5686D086D001800C0B210F001001F
S2140105E00543A5600878002811D0012013689C688F
S2140105F0640864000500EDB215F001052C439C600B
S2140106001068C06810F00100C0B20028F8D00120C0
S21401061030BC7047F8B504000D00002620688068DD
S214010620C0F3C000C0B2002869D02068C068C0F31B
S214010630C000C0B2002862D02068406810F00300F5
S214010640C0B2002803D002280DD006D311E06946B7
S2140106502000FFF7F5FE06000BE069462000FFF7D5
S2140106609FFF060005E069462000FFF725FF06000C
S214010670FFE73000C0B2002801D1002041E001228E
S21401068020684068C0F38100C0B2002805D0022867
S21401069009D005D3032809D00BE00120020008E0A9
S2140106A00220020005E00420020002E00820020009
S2140106B0FFE720684168090A11F07F01C9B20029E5
S2140106C001D18021FFE720684068C0F30210C0B264
S2140106D0002801D10820FFE723685B681B0C13F094
S2140106E00103DBB25B1C009F4F435F4300FB02FC30
S2140106F05FEA4C0CB7FBFCF72F6001273E00300089
S214010700C0B2F2BDF0B4020000201468A56835F04E
S21401071008050300DBB2DB0013F008031D43A560E8
S21401072001234E78002E03D0022E19D00CD323E0DD
S214010730022014686568AD08AD000600F6B216F032
S21401074003063543656019E0012014686568AD0845
S214010750AD000600F6B216F00306354365600DE0FF
S214010760002014686568AD08AD000600F6B216F004
S21401077003063543656001E0002003001800C0B29F
S214010780002801D1002088E0C868012801D1002492
S2140107900FE0C868022801D101240AE0C8680428CD
S2140107A001D1022405E0C868082801D1032400E02D
S2140107B0FF242000C0B2FF2801D100206DE02500F3
S2140107C01668776837F00C072800C0B2800010F072
S2140107D00C00074377604888002817D0488881288E
S2140107E014DA4888802801D1002500E04D88166873
S2140107F0776837F4FE472800C0B2000210F4FE40C6
S214010800074377600869002802D119E0002044E018
S2140108100869092814D20869082801D1002000E0D7
S214010820086915686E6836F070060700FFB23F016A
S21401083017F070073E436E608F68012F02D104E007
S21401084000202AE08868022810D18868451E1668AC
S214010850776837F480372800C0B2000410F480307F
S214010860074377600878002802D114E0002014E0DE
S21401087001201568AE6836F008060700FFB2FF00D3
S21401088017F008073E43AE601068C068C0F3C000AA
S214010890C0B20028F8D01800C0B2F0BC70477CB5D2
S2140108A004000D00002600200090A0684068C0F3F8
S2140108B08000C0B2002817D069462000FFF7FCFD73
S2140108C006003000C0B200280ED0A068016911F001
S2140108D0070101208840412804D20099B1FBF0F0BD
S2140108E0286001E000210E003000C0B276BDF0B4F1
S2140108F00300002000229C68656835F00405160098
S214010900F6B2B60016F00406354365608E88012EF1
S21401091001D100241EE08A88022A01D1012419E0AF
S2140109208A88042A01D1022414E08A88082A01D17F
S21401093003240FE08A88102A01D104240AE08A8859
S214010940202A01D1052405E08A88402A01D10624FF
S21401095000E007242200D2B2072A0CD022009D68AC
S2140109602E69F608F6001700FFB217F007073E4398
S2140109702E61012738000A78002A01D0012200E002
S21401098000229D686E6836F004061700FFB2BF00AD
S21401099017F004073E436E60C0B2F0BC70477CB5EA
S2140109A004000D00002600200090A0684068C0F3F7
S2140109B0C000C0B2002817D069462000FFF77CFDB2
S2140109C006003000C0B200280ED0A0680069C0F34F
S2140109D0021101208840412804D20099B1FBF0F0B1
S2140109E0286001E000210E003000C0B276BDF0B4F0
S2140109F00300002000229C68656835F00805160093
S214010A00F6B2F60016F00806354365608E88012EAC
S214010A1001D100241EE08A88022A01D1012419E0AE
S214010A208A88042A01D1022414E08A88082A01D17E
S214010A3003240FE08A88102A01D104240AE08A8858
S214010A40202A01D1052405E08A88402A01D10624FE
S214010A5000E007242200D2B2072A0DD022009D68AA
S214010A602E6936F070061700FFB23F0117F07007C7
S214010A703E432E61012738000A78002A01D0012260
S214010A8000E000229D686E6836F008061700FFB287
S214010A90FF0017F008073E436E60C0B2F0BC704717
S214010AA07CB504000D00002600200090A068406878
S214010AB0C0F30010C0B2002817D069462000FFF727
S214010AC06FFD06003000C0B200280ED0A068016A93
S214010AD011F0070101208840412804D20099B1FB9A
S214010AE0F0F0286001E000210E003000C0B276BDB3
S214010AF0F0B40300002000229C68656835F01005FC
S214010B001600F6B2360116F01006354365608E887B
S214010B10012E01D100241EE08A88022A01D1012477
S214010B2019E08A88042A01D1022414E08A88082A56
S214010B3001D103240FE08A88102A01D104240AE097
S214010B408A88202A01D1052405E08A88402A01D115
S214010B50062400E007242200D2B2072A0CD0220085
S214010B609D682E6AF608F6001700FFB217F0070711
S214010B703E432E62012738000A78002A01D001225E
S214010B8000E000229D686E6836F010061700FFB27E
S214010B903F0117F010073E436E60C0B2F0BC7047CD
S214010BA07CB504000D00002600200090A068406877
S214010BB0C0F34010C0B2002817D069462000FFF7E6
S214010BC0EFFC06003000C0B200280ED0A068006A14
S214010BD0C0F3021101208840412804D20099B1FBDC
S214010BE0F0F0286001E000210E003000C0B276BDB2
S214010BF0F0B40300002000229C68656835F02005EB
S214010C001600F6B2760116F02006354365608E882A
S214010C10012E01D100241EE08A88022A01D1012476
S214010C2019E08A88042A01D1022414E08A88082A55
S214010C3001D103240FE08A88102A01D104240AE096
S214010C408A88202A01D1052405E08A88402A01D114
S214010C50062400E007242200D2B2072A0DD0220083
S214010C609D682E6A36F070061700FFB23F0117F036
S214010C7070073E432E62012738000A78002A01D009
S214010C80012200E000229D686E6836F020061700FB
S214010C90FFB27F0117F020073E436E60C0B2F0BC82
S214010CA070477CB504000D00002600200090A06867
S214010CB04068C0F38010C0B2002817D069462000F3
S214010CC0FFF7BEFB06003000C0B200280ED0A068B9
S214010CD0016B11F0070101208840412804D20099D8
S214010CE0B1FBF0F0286001E000210E003000C0B238
S214010CF076BDF0B40300002000229C68656835F0DC
S214010D0040051600F6B2B60116F04006354365609A
S214010D108E88012E01D100241EE08A88022A01D184
S214010D20012419E08A88042A01D1022414E08A8861
S214010D30082A01D103240FE08A88102A01D104244D
S214010D400AE08A88202A01D1052405E08A88402AFB
S214010D5001D1062400E007242200D2B2072A0CD0D3
S214010D6022009D682E6BF608F6001700FFB217F0FA
S214010D7007073E432E63012738000A78002A01D070
S214010D80012200E000229D686E6836F040061700DA
S214010D90FFB2BF0117F040073E436E60C0B2F0BC21
S214010DA070477CB504000D00002600200090A06866
S214010DB04068C0F3C010C0B2002817D069462000B2
S214010DC0FFF73EFB06003000C0B200280ED0A06838
S214010DD0006BC0F3021101208840412804D200991B
S214010DE0B1FBF0F0286001E000210E003000C0B237
S214010DF076BDF0B40300002000229C68656835F0DB
S214010E0080051600F6B2F60116F0800635436560D9
S214010E108E88012E01D100241EE08A88022A01D183
S214010E20012419E08A88042A01D1022414E08A8860
S214010E30082A01D103240FE08A88102A01D104244C
S214010E400AE08A88202A01D1052405E08A88402AFA
S214010E5001D1062400E007242200D2B2072A0DD0D1
S214010E6022009D682E6B36F070061700FFB23F0118
S214010E7017F070073E432E63012738000A78002AD0
S214010E8001D0012200E000229D686E6836F08006DF
S214010E901700FFB2FF0117F080073E436E60C0B235
S214010EA0F0BC70477CB504000D00002600200090C1
S214010EB0A0684068000A10F00100C0B2002817D0F0
S214010EC069462000FFF7A6FB06003000C0B20028E6
S214010ED00ED0A068016C11F007010120884041285E
S214010EE004D20099B1FBF0F0286001E000210E0069
S214010EF03000C0B276BDF0B40300002000229C682A
S214010F00656835F480751600F6B2360216F48076FA
S214010F10354365608E88012E01D100241EE08A8843
S214010F20022A01D1012419E08A88042A01D1022467
S214010F3014E08A88082A01D103240FE08A88102A3F
S214010F4001D104240AE08A88202A01D1052405E07B
S214010F508A88402A01D1062400E007242200D2B262
S214010F60072A0CD022009D682E6CF608F6001700A2
S214010F70FFB217F007073E432E64012738000A78B0
S214010F80002A01D0012200E000229D686E6836F436
S214010F9080761700FFB23F0217F480773E436E60FB
S214010FA0C0B2F0BC70477CB504000D0000260020DE
S214010FB00090A0684068400A10F00100C0B2002806
S214010FC017D069462000FFF725FB06003000C0B2A7
S214010FD000280ED0A068006CC0F3021101208840E2
S214010FE0412804D20099B1FBF0F0286001E000210D
S214010FF00E003000C0B276BDF0B40300002000221F
S2140110009C68656835F400751600F6B2760216F42B
S2140110100076354365608E88012E01D100241EE0DE
S2140110208A88022A01D1012419E08A88042A01D17A
S214011030022414E08A88082A01D103240FE08A8852
S214011040102A01D104240AE08A88202A01D1052425
S21401105005E08A88402A01D1062400E00724220000
S214011060D2B2072A0DD022009D682E6C36F070068B
S2140110701700FFB23F0117F070073E432E640127A9
S21401108038000A78002A01D0012200E000229D687B
S2140110906E6836F400761700FFB27F0217F4007709
S2140110A03E436E60C0B2F0BC704770B504000D00E0
S2140110B000262068C068C0F30110C0B2002805D021
S2140110C002280FD008D3032812D017E029002000E9
S2140110D0FFF7B6F9060011E029002000FFF7ECF94A
S2140110E006000BE029002000FFF794FA060005E051
S2140110F029002000FFF754FA0600FFE73000C0B2CF
S21401110070BD70B402004878022801D100230FE0B8
S2140111104878002801D101230AE04878032801D144
S214011120022305E04878012801D1032300E0FF23CC
S2140111301800C0B2FF2801D1002014E0180014687E
S2140111402569AD08AD000600F6B216F00306354374
S21401115025611068C068C0F301101C00C0B2E4B27B
S214011160A042F6D1012070BC70477CB504000D008A
S214011170002669462000FFF798FF01000800C0B26C
S214011180002801D100200BE020680069C0F303109D
S214011190009AC0B2401CB2FBF0F028600800C0B252
S2140111A076BD30B402008888002811D088881128BE
S2140111B00EDA8888431E1468256935F0F005180094
S2140111C0C0B2000110F0F00005432561012000E0E7
S2140111D0002030BC70477CB504000D00002669462F
S2140111E02000FFF7C2FF01000800C0B2002801D1AD
S2140111F000200CE0A0680068000A10F00F00009ABA
S214011200C0B2401CB2FBF0F028600800C0B276BD48
S21401121030B402008888002811D0888811280EDA98
S2140112208888431E9468256835F470651800C0B236
S214011230000210F4706005432560012000E00020E4
S21401124030BC70477CB504000D00002669462000BE
S214011250FFF78BFF01000800C0B2002801D1002073
S21401126015E0E068006910F00100C0B200280AD05D
S214011270A068006810F01F00009AC0B2401CB2FBC4
S214011280F0F0286001E0002001000800C0B276BD41
S21401129030B402008888002820D0888809281DDA02
S2140112A08888431E946825686D096D011800C0B2D0
S2140112B010F01F00054325600878002801D001239F
S2140112C000E00023D46825696D086D001800C0B2DF
S2140112D010F0010005432561012000E0002030BC2C
S2140112E070477CB504000D00002669462000FFF714
S2140112F03CFF01000800C0B2002801D1002016E022
S214011300A068406810F00100C0B200280BD0A068A9
S2140113100068000F10F00700009AC0B2401CB2FB34
S214011320F0F0286001E0002001000800C0B276BDA0
S21401133070B40300002000249D686E68760876006D
S2140113402200D2B212F0010216436E608A88002A89
S21401135011D08A88092A0EDA8A88521E9C68256866
S21401136035F0E0451600F6B2360716F0E04635438E
S2140113702560012630000A78002A01D0012200E00B
S21401138000229C6865686D086D001600F6B216F0BE
S214011390010635436560C0B270BC70477CB5040079
S2140113A00D00A0684068C0F34000C0B2002801D11B
S2140113B000209AE0002600200090A0688068C0F314
S2140113C00210C0B2002843D1A068806810F0070060
S2140113D0C0B200280BD0022815D00ED304281ED088
S2140113E017D3062827D020D307282AD02FE069460E
S2140113F02000FFF727FF060066E069462000FFF79A
S2140114005BF8060060E069462000FFF7C9F80600B1
S2140114105AE069462000FFF713F8060054E06946D3
S2140114202000FFF7F7F806004EE069462000FFF7B8
S2140114309CFE060048E069462000FFF7CCFE060049
S21401144042E069462000FFF7ACFC06003CE03BE0CA
S214011450A0688068C0F30210C0B201280AD033D356
S214011460032813D00CD305281CD015D3072825D064
S2140114701ED329E069462000FFF791FA060023E013
S21401148069462000FFF78FFD06001DE06946200033
S214011490FFF786FB060017E06946200000F02AFAEF
S2140114A0060011E06946200000F0FFF906000BE097
S2140114B06946200000F0D4F9060005E069462000E0
S2140114C000F01EFA0600FFE73000C0B201280AD17C
S2140114D0A0688068000A10F007000099C0B2401C9E
S2140114E0B1FBF0F028603000C0B276BDF0B5030065
S2140114F00A00012000219C68656835F002050E008F
S214011500F6B2760016F00206354365605678002E70
S21401151045D0012E61D0022E7DD0032E00F0998099
S214011520052E00F00E81072E00F02581092E00F011
S214011530EA800B2E00F012810D2E00F0A8800E2EF0
S21401154000F0C3800F2E0CD0132E00F03B81142E1A
S21401155000F02B81152E00F01B81162E00F03F8126
S2140115604AE100219C68A56835F070050E00F6B2C8
S214011570360116F070063543A56000269F68D7F839
S21401158008C05FEADC0C5FEACC0CB6465FFA8EFE5A
S2140115901EF0070E5EEA0C0CC7F808C02EE100210B
S2140115A09C68A56835F070050E00F6B2360116F097
S2140115B070063543A56001269F68D7F808C05FEA24
S2140115C0DC0C5FEACC0CB6465FFA8EFE1EF0070E08
S2140115D05EEA0C0CC7F808C010E100219C68A568FB
S2140115E035F070050E00F6B2360116F0700635437A
S2140115F0A56002269F68D7F808C05FEADC0C5FEAA0
S214011600CC0CB6465FFA8EFE1EF0070E5EEA0C0C98
S214011610C7F808C0F2E000219C68A56835F070059F
S2140116200E00F6B2360116F070063543A5600326A5
S2140116309F68D7F808C05FEADC0C5FEACC0CB646B8
S2140116405FFA8EFE1EF0070E5EEA0C0CC7F808C0A5
S214011650D4E000219C68A56835F070050E00F6B24E
S214011660360116F070063543A56004269F68D7F844
S21401167008C05FEADC0C5FEACC0CB6465FFA8EFE69
S2140116801EF0070E5EEA0C0CC7F808C0B6E0002193
S2140116909C68A56835F070050E00F6B2360116F0A6
S2140116A070063543A56005269F68D7F808C05FEA2F
S2140116B0DC0C5FEACC0CB6465FFA8EFE1EF0070E17
S2140116C05EEA0C0CC7F808C098E000219C68A56883
S2140116D035F070050E00F6B2360116F07006354389
S2140116E0A56006269F68D7F808C05FEADC0C5FEAAB
S2140116F0CC0CB6465FFA8EFE1EF0070E5EEA0C0CA8
S214011700C7F808C07AE000219C68A56835F0700526
S2140117100E00F6B2360116F070063543A5600726B0
S2140117209F68D7F808C05FEADC0C5FEACC0CB646C7
S2140117305FFA8EFE1EF0070E5EEA0C0CC7F808C0B4
S2140117405CE001219C68A56835F070050E00F6B2D4
S214011750360116F070063543A5604FE002219C68FD
S214011760A56835F070050E00F6B2360116F0700663
S2140117703543A56042E003219C68A56835F07005F5
S2140117800E00F6B2360116F070063543A56035E058
S21401179004219C68A56835F070050E00F6B2360186
S2140117A016F070063543A56028E005219C68A568FB
S2140117B035F070050E00F6B2360116F070063543A8
S2140117C0A5601BE006219C68A56835F070050E0033
S2140117D0F6B2360116F070063543A5600EE0072115
S2140117E09C68A56835F070050E00F6B2360116F055
S2140117F070063543A56001E0002108000100C9B26A
S214011800002915D09188002910D0918809290DDA70
S2140118109188491E9C68A56835F4E0650E00F6B20D
S214011820360216F4E0663543A56001E000210800A3
S2140118301178002901D0012100E000219C6865682B
S21401184035F002050E00F6B2760016F002063543B4
S2140118506560C0B2F0BD0200D06908600120704723
S214011860020050684068C0F3C000C0B2002804D02F
S2140118704FF47A700860012000E00020704730B411
S21401188002000878002801D0012300E000235468F4
S214011890656835F008051800C0B2C00010F00800F1
S2140118A005436560012030BC7047020050684068FF
S2140118B0C0F30010C0B2002804D04FF4FA4008600C
S2140118C0012000E00020704730B4020008780028AC
S2140118D001D0012300E000235468656835F0100547
S2140118E01800C0B2000110F0100005436560012029
S2140118F030BC704702005FF4FA3008600120704780
S21401190070B504000D00002660684068C0F3400012
S214011910C0B2002801D100201AE060680068C0F358
S2140119200010C0B2002805D129002000FFF7BDFF36
S21401193006000BE060680068C0F30010C0B2012822
S21401194004D129002000FFF786FF06003000C0B250
S21401195070BD70B40300002000225C68656835F035
S21401196002051600F6B2760016F0020635436560EB
S2140119704E78142E0ED100225C68256835F01005CD
S2140119801600F6B2360116F010063543256001261C
S214011990300010E04A78122A0DD101225C682568D1
S2140119A035F010051600F6B2360116F0100635436E
S2140119B02560012630000A78002A01D0012200E0C5
S2140119C000225C68656835F002051600F6B27600FE
S2140119D016F0020635436560C0B270BC704770B53C
S2140119E004000D00002660680068000B10F001007E
S2140119F0C0B2002805D129002000FFF7ECFB060045
S214011A000CE060680068000B10F00100C0B201280D
S214011A1004D15FF4FA302860012006003000C0B21D
S214011A2070BD70B4020000204B780E2B0ED100233F
S214011A305468256835F480551E00F6B2360316F450
S214011A408056354325600126300010E04B78152B73
S214011A500DD101235468256835F480551E00F6B271
S214011A60360316F480563543256001263000C0B291
S214011A7070BC704770B504000D00002660684068B1
S214011A80C0F38010C0B2002801D100202EE06068AB
S214011A900068400B10F00700C0B2002806D00228EC
S214011AA010D009D3042819D012D31DE02900200034
S214011AB0FFF777F9060017E029002000FEF76FFF11
S214011AC0060011E029002000FFF76DFA06000BE082
S214011AD029002000FFF764F8060005E05FF4FA30FD
S214011AE0286001200600FFE73000C0B270BD70B468
S214011AF00300012000225C68656835F04005160089
S214011B00F6B2B60116F04006354365604E78052EEE
S214011B1015D0072E2DD0092E04D00B2E1CD0152E35
S214011B2034D040E000225C68256835F46045160034
S214011B30F6B2760316F460463543256035E0012299
S214011B405C68256835F460451600F6B2760316F42F
S214011B5060463543256028E002225C68256835F436
S214011B6060451600F6B2760316F4604635432560E6
S214011B701BE003225C68256835F460451600F6B262
S214011B80760316F46046354325600EE004225C6851
S214011B90256835F460451600F6B2760316F46046FD
S214011BA03543256001E0002210000A78002A01D0A2
S214011BB0012200E000225C68656835F040051600E9
S214011BC0F6B2B60116F0400635436560C0B270BC89
S214011BD070477CB504000D00002600200090606868
S214011BE04068C0F38000C0B2002801D1002054E054
S214011BF060680068000C10F00700C0B200280BD027
S214011C00022815D00ED304281ED017D3062827D0B5
S214011C1020D307282AD02FE069462000FFF7C1F815
S214011C20060029E069462000FEF7B9FE060023E01B
S214011C3069462000FFF7B7F906001DE06946200057
S214011C40FEF7AEFF060017E069462000FFF752FEDA
S214011C50060011E069462000FFF702FE06000BE0D1
S214011C6069462000FFF721FE060005E069462000D0
S214011C70FFF7F1FD0600FFE73000C0B200280AD0EA
S214011C8060680068000D10F00700C0B2401C0099A3
S214011C90B1FBF0F028603000C0B276BD70B403002E
S214011CA0012000225C68656835F004051600F6B26E
S214011CB0B60016F00406354365604E78052E1BD037
S214011CC0072E33D0092E0AD00B2E22D0122E61D029
S214011CD0132E45D0142E50D0152E34D067E0002296
S214011CE05C68256835F4E0251600F6B2360416F46D
S214011CF0E026354325605CE001225C68256835F402
S214011D00E0251600F6B2360416F4E02635432560C3
S214011D104FE002225C68256835F4E0251600F6B22D
S214011D20360416F4E0263543256042E003225C685B
S214011D30256835F4E0251600F6B2360416F4E026DA
S214011D403543256035E004225C68256835F4E025D6
S214011D501600F6B2360416F4E0263543256028E070
S214011D6005225C68256835F4E0251600F6B23604CF
S214011D7016F4E026354325601BE006225C682568DC
S214011D8035F4E0251600F6B2360416F4E02635439F
S214011D9025600EE007225C68256835F4E02516000C
S214011DA0F6B2360416F4E0263543256001E000223B
S214011DB010008A88002A10D08A88092A0DDA8A88B3
S214011DC0521E5C68256835F4E0051600F6B2360545
S214011DD016F4E0063543256001E0002210000A787B
S214011DE0002A01D0012200E000225C68656835F017
S214011DF004051600F6B2B60016F004063543656013
S214011E00C0B270BC704770B504000D000026606853
S214011E10406810F00100C0B2002801D100201AE08D
S214011E2060680068C0F34010C0B2002805D12900E0
S214011E302000FFF765FD06000BE060680068C0F350
S214011E404010C0B2012804D129002000FFF708FD88
S214011E5006003000C0B270BD70B40300002000223E
S214011E605C6865686D086D001600F6B216F001062E
S214011E70354365604E78162E0ED100225C682568C3
S214011E8035F020051600F6B2760116F02006354329
S214011E9025600126300010E04A78132A0DD1012270
S214011EA05C68256835F020051600F6B2760116F056
S214011EB0200635432560012630000A78002A01D025
S214011EC0012200E000225C6865686D086D0016005E
S214011ED0F6B216F0010635436560C0B270BC7047B5
S214011EE070B504000D00002660680068000E10F052
S214011EF00100C0B2002805D129002000FFF76BF9C8
S214011F0006000CE060680068000E10F00100C0B228
S214011F10012804D129002000FFF7ECFC0600300060
S214011F20C0B270BD70B4020000204B780E2B0CD1ED
S214011F3000235468256835F080751E00F6B2360613
S214011F4016F08076354325600EE04B78152B0BD1C5
S214011F5001235468256835F080751E00F6B23606F2
S214011F6016F0807635432560C0B270BC704770B5F8
S214011F7004000D00002660680068400E10F00100A5
S214011F80C0B2002805D129002000FFF724F9060079
S214011F900CE060680068400E10F00100C0B2012835
S214011FA004D129002000FFF7A5FC06003000C0B2CE
S214011FB070BD70B4020000204B780E2B0CD10023AC
S214011FC05468256835F000751E00F6B2760616F0E0
S214011FD00076354325600EE04B78152B0BD1012397
S214011FE05468256835F000751E00F6B2760616F0C0
S214011FF0007635432560C0B270BC704770B50400EA
S2140120000D00002660680068800E10F00100C0B266
S214012010002805D129002000FFF7DDF806000CE0B6
S21401202060680068800E10F00100C0B2012804D17B
S21401203029002000FFF75EFC06003000C0B270BD2C
S21401204070B4020000204B780E2B0CD1002354688C
S214012050256835F080651E00F6B2B60616F0806675
S214012060354325600EE04B78152B0BD101235468C0
S214012070256835F080651E00F6B2B60616F0806655
S21401208035432560C0B270BC704770B504000D00C2
S214012090002660680068C00E10F00100C0B200287B
S2140120A005D129002000FFF796F806000CE06068CD
S2140120B00068C00E10F00100C0B2012804D129004A
S2140120C02000FFF717FC06003000C0B270BD70B4E8
S2140120D0020000204B780E2B0CD100235468256893
S2140120E035F000651E00F6B2F60616F000663543BA
S2140120F025600EE04B78152B0BD10123546825681B
S21401210035F000651E00F6B2F60616F00066354399
S2140121102560C0B270BC704770B504000D00002683
S21401212060680068000F10F00100C0B2002805D1F9
S21401213029002000FFF74FF806000CE060680068F1
S214012140000F10F00100C0B2012804D129002000C0
S214012150FFF7D0FB06003000C0B270BD70B40200BD
S21401216000204B780E2B0CD100235468256835F0DF
S21401217080551E00F6B2360716F0805635432560A8
S2140121800EE04B78152B0BD101235468256835F0EA
S21401219080551E00F6B2360716F080563543256088
S2140121A0C0B270BC704770B504000D0000266068B0
S2140121B04068000A10F00100C0B2002804D02900CF
S2140121C02000FFF708F806003000C0B270BD30B43A
S2140121D002000878002801D0012300E0002354689B
S2140121E0656835F480751800C0B2000210F480707E
S2140121F005436560012030BC704770B504000D00D2
S214012200002660684068400A10F00100C0B200284D
S21401221004D029002000FEF7DEFF06003000C0B221
S21401222070BD30B402000878002801D0012300E018
S21401223000235468656835F400751800C0B2400282
S21401224010F4007005436560012030BC704770B51E
S21401225004000D00002660684068800A10F0010046
S214012260C0B2002804D029002000FEF7B4FF060003
S2140122703000C0B270BD30B402000878002801D02A
S214012280012300E000235468656835F48065180072
S214012290C0B2800210F4806005436560012030BC46
S2140122A0704770B504000D00002660684068C00ADB
S2140122B010F00100C0B2002804D029002000FEF76B
S2140122C08AFF06003000C0B270BD30B40200087844
S2140122D0002801D0012300E000235468656835F426
S2140122E000651800C0B2C00210F4006005436560C6
S2140122F0012030BC704770B504000D0000266068F0
S2140123004068000B10F00100C0B2002804D029007C
S2140123102000FEF760FF06003000C0B270BD30B48A
S21401232002000878002801D0012300E00023546849
S214012330656835F480551800C0B2000310F480506B
S21401234005436560012030BC704770B504000D0080
S214012350002660684068C0F34010C0B2002801D172
S21401236000201CE060680068C00D10F00100C0B2DB
S214012370002805D129002000FEF72DFF06000CE0FD
S21401238060680068C00D10F00100C0B2012804D1D9
S21401239029002000FFF71DFC06003000C0B270BD0A
S2140123A070B40300002000225C68656835F02005E3
S2140123B01600F6B2760116F02006354365604E78B3
S2140123C00E2E0ED100225C68256835F40005160035
S2140123D0F6B2F60516F400063543256001263000F0
S2140123E010E04A78192A0DD101225C68256835F477
S2140123F000051600F6B2F60516F40006354325600C
S214012400012630000A78002A01D0012200E00022CD
S2140124105C68656835F020051600F6B2760116F0A0
S214012420200635436560C0B270BC704738B50400FD
S2140124300D00E0680069C0F34000C0B2002801D179
S214012440002003E029002000FEF78FFE32BD30B4E5
S21401245002000878002801D0012300E00023D46898
S214012460256935F002051800C0B2400010F00200E0
S21401247005432561012030BC704738B504000D00C6
S214012480E0680069C0F38000C0B2002801D10020D6
S21401249003E029002000FEF768FE32BD30B40200DA
S2140124A00878002801D0012300E00023D4682569BC
S2140124B035F004051800C0B2800010F00400054392
S2140124C02561012030BC704738B504000D00E06876
S2140124D00069C0F3C000C0B2002801D1002003E0AB
S2140124E029002000FEF741FE32BD30B40200087814
S2140124F0002801D0012300E00023D468256935F0C7
S21401250008051800C0B2C00010F008000543256198
S214012510012030BC704738B504000D00E068006942
S214012520C0F34010C0B2002801D1002003E029000A
S2140125302000FEF71AFE32BD30B4020008780028EB
S21401254001D0012300E00023D468256935F0200579
S2140125501800C0B2400110F020000543256101209B
S21401256030BC704738B504000D00E0680069000F04
S21401257010F00100C0B2002801D1002003E02900BC
S2140125802000FEF7F2FD32BD30B4020008780028C4
S21401259001D0012300E00023D468256935F0805579
S2140125A01800C0B2000710F08050054325610120D5
S2140125B030BC704738B504000D00E0680069400F74
S2140125C010F00100C0B2002801D1002003E029006C
S2140125D02000FEF7CAFD32BD30B40200087800289C
S2140125E001D0012300E00023D468256935F00055A9
S2140125F01800C0B2400710F00050054325610120C5
S21401260030BC704738B504000D00E0684069C0F37F
S2140126108000C0B2002801D1002003E0290020007C
S214012620FEF7A3FD32BD30B402000878002801D0C1
S214012630012300E00023D468656935F0040518001D
S214012640C0B2800010F0040005436561012030BC73
S214012650704738B504000D00E0684069C0F3C0005B
S214012660C0B2002801D1002003E029002000FEF7B7
S2140126707CFD32BD30B402000878002801D0012369
S21401268000E00023D468656935F008051800C0B27B
S214012690C00010F0080005436561012030BC70479A
S2140126A038B504000D00E0684069C0F30010C0B200
S2140126B0002801D1002003E029002000FEF755FD87
S2140126C032BD30B402000878002801D0012300E0B2
S2140126D00023D468656935F010051800C0B2000102
S2140126E010F0100005436561012030BC704738B515
S2140126F004000D00E0684069C0F34010C0B2002835
S21401270001D1002003E029002000FEF72EFD32BD96
S21401271030B402000878002801D0012300E000232D
S214012720D468656935F020051800C0B2400110F084
S214012730200005436561012030BC7047020000207F
S2140127407047020000207047020000207047020018
S2140127500020704738B504000D00E0680069C0F33A
S2140127600010C0B2002801D1002003E0290020009B
S214012770FEF731FD32BD30B402000878002801D0E2
S214012780012300E00023D468256935F01005180000
S214012790C0B2000110F0100005432561012030BCD5
S2140127A0704738B504000D00E0680069000A10F0B3
S2140127B00100C0B2002801D1002003E0290020005A
S2140127C0FEF709FD32BD30B402000878002801D0BA
S2140127D0012300E00023D468256935F480751800CC
S2140127E0C0B2000210F4807005432561012030BCA0
S2140127F0704738B504000D00E0680069C00B10F0A2
S2140128000100C0B2002801D1002003E02900200009
S214012810FEF7E1FC32BD30B402000878002801D092
S214012820012300E00023D468256935F4004518002B
S214012830C0B2C00310F4004005432561012030BC3E
S214012840704738B504000D00E0680069000C10F010
S2140128500100C0B2002801D1002003E029002000B9
S214012860FEF7B9FC32BD30B402000878002801D06A
S214012870012300E00023D468256935F4803518006B
S214012880C0B2000410F4803005432561012030BC3D
S214012890704738B504000D00E0684069800A10F002
S2140128A00100C0B2002801D1002003E02900200069
S2140128B0FEF791FC32BD30B402000878002801D042
S2140128C0012300E00023D468656935F480651800AB
S2140128D0C0B2800210F4806005436561012030BCFF
S2140128E0704738B504000D00E0684069C00A10F072
S2140128F00100C0B2002801D1002003E02900200019
S214012900FEF769FC32BD30B402000878002801D019
S214012910012300E00023D468656935F400651800DA
S214012920C0B2C00210F4006005436561012030BCEE
S214012930704738B504000D00E0684069000B10F0E0
S2140129400100C0B2002801D1002003E029002000C8
S214012950FEF741FC32BD30B402000878002801D0F1
S214012960012300E00023D468656935F4805518001A
S214012970C0B2000310F4805005436561012030BCED
S214012980704738B504000D00E0684069400B10F050
S2140129900100C0B2002801D1002003E02900200078
S2140129A0FEF719FC32BD30B402000878002801D0C9
S2140129B0012300E00023D468656935F4005518004A
S2140129C0C0B2400310F4005005436561012030BCDD
S2140129D0704738B504000D00E0684069800B10F0C0
S2140129E00100C0B2002801D1002003E02900200028
S2140129F0FEF7F1FB32BD30B402000878002801D0A2
S214012A00012300E00023D468656935F48045180089
S214012A10C0B2800310F4804005436561012030BCDC
S214012A20704738B504000D00E0680069800F10F0AB
S214012A300100C0B2002801D1002003E029002000D7
S214012A40FEF7C9FB32BD30B402000878002801D079
S214012A50012300E00023D468256935F0804518007D
S214012A60C0B2800710F0804005432561012030BCCC
S214012A70704738B504000D00E0684069800E10F01C
S214012A800100C0B2002801D1002003E02900200087
S214012A90FDF712FD32BD30B402000878002801D0DF
S214012AA0012300E00023D468656935F080651800CD
S214012AB0C0B2800610F0806005436561012030BC1D
S214012AC0704738B504000D00E0684069000E10F04C
S214012AD00100C0B2002801D1002003E02900200037
S214012AE0FDF7AEFC32BD30B402000878002801D0F4
S214012AF0012300E00023D468656935F0807518006D
S214012B00C0B2000610F0807005436561012030BC3C
S214012B10704738B504000D00E0684069C00E10F03B
S214012B200100C0B2002801D1002003E029002000E6
S214012B30FDF786FC32BD30B402000878002801D0CB
S214012B40012300E00023D468656935F000651800AC
S214012B50C0B2C00610F0006005436561012030BCBC
S214012B60704738B504000D00E0684069400E10F06B
S214012B700100C0B2002801D1002003E02900200096
S214012B80FDF748FD32BD30B402000878002801D0B8
S214012B90012300E00023D468656935F0007518004C
S214012BA0C0B2400610F0007005436561012030BCDC
S214012BB0704770B504000D00E0680069400E10F023
S214012BC00100C0B2002801D1002023E00126E06800
S214012BD0006810F00300C0B2002805D002280DD00E
S214012BE007D303280FD013E029002000FEF7D9F8F9
S214012BF00FE029002000FDF7D2FE0AE029002000A0
S214012C00FEF7D1F905E029002000FDF7C9FF00E035
S214012C100020C0B270BDF0B4030000200022DC68C2
S214012C20256935F000751600F6B2760616F00076C0
S214012C30354325614E78092E01D100240FE04A78EC
S214012C40052A01D101240AE04A780B2A01D102247F
S214012C5005E04A78072A01D1032400E0FF24220078
S214012C60D2B2FF2A0CD02200DD682E68B608B60064
S214012C701700FFB217F003073E432E600127380006
S214012C800A78002A01D0012200E00022DD682E69C0
S214012C9036F000761700FFB27F0617F000773E4346
S214012CA02E61C0B2F0BC704770B504000D00E0683C
S214012CB00069400C10F00100C0B2002801D10020CC
S214012CC024E00126E0680068000D10F00300C0B2A1
S214012CD0002805D002280DD007D303280FD013E013
S214012CE029002000FEF75DF80FE029002000FDF71F
S214012CF056FE0AE029002000FEF755F905E02900F6
S214012D002000FDF74DFF00E00020C0B270BDF0B41A
S214012D10030000200022DC68256935F40035160022
S214012D20F6B2760416F40036354325614E78092E40
S214012D3001D100240FE04A78052A01D101240AE0D6
S214012D404A780B2A01D1022405E04A78072A01D1E4
S214012D50032400E0FF242200D2B2FF2A0DD0220075
S214012D60DD682E6836F440161700FFB23F0517F4EB
S214012D7040173E432E60012738000A78002A01D00A
S214012D80012200E00022DD682E6936F400361700C5
S214012D90FFB27F0417F400373E432E61C0B2F0BC89
S214012DA0704770B504000D00E0680069800C10F0F3
S214012DB00100C0B2002801D1002024E00126E0680D
S214012DC00068800D10F00300C0B2002805D002286C
S214012DD00DD007D303280FD013E029002000FDF7FC
S214012DE0E0FF0FE029002000FDF7D9FD0AE02900E9
S214012DF02000FEF7D8F805E029002000FDF7D0FEF8
S214012E0000E00020C0B270BDF0B403000020002234
S214012E10DC68256935F480251600F6B2B60416F48A
S214012E208026354325614E78092E01D100240FE016
S214012E304A78052A01D101240AE04A780B2A01D1F1
S214012E40022405E04A78072A01D1032400E0FF2482
S214012E502200D2B2FF2A0DD02200DD682E6836F499
S214012E6040061700FFB2BF0517F440073E432E6029
S214012E70012738000A78002A01D0012200E000224A
S214012E80DD682E6936F480261700FFB2BF0417F4FA
S214012E9080273E432E61C0B2F0BC704770B5040077
S214012EA00D00E0680069C00C10F00100C0B20028F7
S214012EB001D1002024E00126E0680068000E10F031
S214012EC00300C0B2002805D002280DD007D303287E
S214012ED00FD013E029002000FDF763FF0FE0290063
S214012EE02000FDF75CFD0AE029002000FEF75BF8F4
S214012EF005E029002000FDF753FE00E00020C0B2E7
S214012F0070BDF0B4030000200022DC68256935F4AA
S214012F1000251600F6B2F60416F4002635432561A0
S214012F204E78092E01D100240FE04A78052A01D1F6
S214012F3001240AE04A780B2A01D1022405E04A78E6
S214012F40072A01D1032400E0FF242200D2B2FF2A7F
S214012F500DD02200DD682E6836F040761700FFB2ED
S214012F603F0617F040773E432E60012738000A7867
S214012F70002A01D0012200E00022DD682E6936F425
S214012F8000261700FFB2FF0417F400273E432E6108
S214012F90C0B2F0BC7047020000207047020000205B
S214012FA0704770B504000D00E0680069400D10F030
S214012FB00100C0B2002801D1002024E00126E0680B
S214012FC00068000A10F00300C0B2002805D00228ED
S214012FD00DD007D303280FD013E029002000FDF7FA
S214012FE0E0FE0FE029002000FDF7D9FC0AE02900E9
S214012FF02000FDF7D8FF05E029002000FDF7D0FDF1
S21401300000E00020C0B270BDF0B403000020002232
S214013010DC68256935F400151600F6B2760516F457
S2140130200016354325614E78092E01D100240FE0A4
S2140130304A78052A01D101240AE04A780B2A01D1EF
S214013040022405E04A78072A01D1032400E0FF2480
S2140130502200D2B2FF2A0DD02200DD682E6836F497
S21401306040761700FFB23F0217F440773E432E60CA
S214013070012738000A78002A01D0012200E0002248
S214013080DD682E6936F400161700FFB27F0517F4C7
S21401309000173E432E61C0B2F0BC704770B5040005
S2140130A00D00E0680069800D10F00100C0B2002834
S2140130B001D1002024E00126E0680068800A10F0B3
S2140130C00300C0B2002805D002280DD007D303287C
S2140130D00FD013E029002000FDF763FE0FE0290062
S2140130E02000FDF75CFC0AE029002000FDF75BFFED
S2140130F005E029002000FDF753FD00E00020C0B2E6
S21401310070BDF0B4030000200022DC68256935F4A8
S21401311080051600F6B2B60516F48006354325611D
S2140131204E78092E01D100240FE04A78052A01D1F4
S21401313001240AE04A780B2A01D1022405E04A78E4
S214013140072A01D1032400E0FF242200D2B2FF2A7D
S2140131500DD02200DD682E6836F440661700FFB2F7
S214013160BF0217F440673E432E60012738000A78F5
S214013170002A01D0012200E00022DD682E6936F423
S21401318080061700FFB2BF0517F480073E432E6185
S214013190C0B2F0BC704770B504000D00E06800696D
S2140131A0C00D10F00100C0B2002801D1002024E0BB
S2140131B00126E0680068000B10F00300C0B200288A
S2140131C005D002280DD007D303280FD013E029001D
S2140131D02000FDF7E6FD0FE029002000FDF7DFFBEC
S2140131E00AE029002000FDF7DEFE05E029002000A8
S2140131F0FDF7D6FC00E00020C0B270BDF0B40300BD
S21401320000200022DC68256935F400051600F6B2B8
S214013210F60516F40006354325614E78092E01D1D0
S21401322000240FE04A78052A01D101240AE04A78F1
S2140132300B2A01D1022405E04A78072A01D103248A
S21401324000E0FF242200D2B2FF2A0DD02200DD6862
S2140132502E6836F440561700FFB23F0317F4405766
S2140132603E432E60012738000A78002A01D0012249
S21401327000E00022DD682E6936F400061700FFB272
S214013280FF0517F400073E432E61C0B2F0BC70473D
S2140132900200002070470200002070477CB5040041
S2140132A00D00E0680069800E10F00100C0B2002831
S2140132B001D1002033E0012600200090E06800687C
S2140132C0C0F30110C0B2002805D002280DD007D3E4
S2140132D003280FD013E069462000FDF7B1F80FE090
S2140132E069462000FDF7E8F80AE069462000FDF788
S2140132F091F905E069462000FDF752F900E000204B
S214013300E168496811F03F01C9B2491C022901D29E
S21401331002221100009AB2FBF1F22A60C0B276BD19
S214013320F0B4030000200022DC68256935F08065D2
S2140133301600F6B2B60616F08066354325614E785D
S214013340022E01D100240FE04A78002A01D101247F
S2140133500AE04A78032A01D1022405E04A78012AC4
S21401336001D1032400E0FF242200D2B2FF2A0DD0AF
S2140133702200DD682E6836F030061700FFB23F01E6
S21401338017F030073E432E60012738000200D2B204
S214013390002A14D08A88022A0FDB8A88412A0CDA8E
S2140133A08A88521EDD686E68B609B6011700FFB23C
S2140133B017F03F073E436E6001E0002210000A78D6
S2140133C0002A01D0012200E00022DD682E6936F0D5
S2140133D080661700FFB2BF0617F080673E432E6176
S2140133E0C0B2F0BC704702000020704730B4020043
S2140133F00878002801D0012300E00023D46825695D
S21401340035F000651800C0B2C00610F00060054334
S2140134102561012030BC70477CB504000D00E068D2
S2140134200069400B10F00100C0B2002801D1002055
S21401343034E0012600200090E068806810F0030068
S214013440C0B2002805D002280DD007D303280FD01C
S21401345013E069462000FCF7F3FF0FE06946200001
S214013460FDF72AF80AE069462000FDF7D3F805E0E3
S21401347069462000FDF794F800E00020E1688968BD
S214013480090A11F00701C9B2002901D1012100E0A2
S2140134904900009AB2FBF1F22A60C0B276BDF0B4E0
S2140134A003000A0000200021DC68256935F4005578
S2140134B00E00F6B2760316F40056354325615678AB
S2140134C0022E01D100240FE05178002901D10124F8
S2140134D00AE05178032901D1022405E05178012937
S2140134E001D1032400E0FF242100C9B2FF290CD03A
S2140134F02100DD68AE68B608B6000F00FFB217F00F
S21401350003073E43AE60012738000100C9B2002917
S21401351017D0918849080D00EDB2082D0FDA0D007D
S214013520DE68B76837F4E067AC465FFA8CFC5FEAA2
S2140135300C2C1CF4E06C5CEA0707B76001E0002580
S21401354028001178002901D0012100E00021DD6862
S2140135502E6936F400560F00FFB27F0317F40057AA
S2140135603E432E61C0B2F0BC70477CB504000D002E
S214013570E0680069800B10F00100C0B2002801D19C
S214013580002034E0012600200090E0688068C0F347
S214013590C100C0B2002805D002280DD007D30328E9
S2140135A00FD013E069462000FCF74AFF0FE069469A
S2140135B02000FCF781FF0AE069462000FDF72AF8A3
S2140135C005E069462000FCF7EBFF00E00020E1681B
S2140135D08968090B11F00701C9B2002901D101213F
S2140135E000E04900009AB2FBF1F22A60C0B276BD53
S2140135F0F0B403000A0000200021DC68256935F4D8
S21401360080450E00F6B2B60316F4804635432561B2
S2140136105678022E01D100240FE05178002901D1FD
S21401362001240AE05178032901D1022405E05178EA
S214013630012901D1032400E0FF242100C9B2FF299A
S2140136400DD02100DD68AE6836F018060F00FFB217
S214013650FF0017F018073E43AE600127380001004F
S214013660C9B2002917D0918849080D00EDB2082D7E
S2140136700FDA0D00DE68B76837F4E047AC465FFA4C
S2140136808CFC5FEA0C3C1CF4E04C5CEA0707B76074
S21401369001E0002528001178002901D0012100E071
S2140136A00021DD682E6936F480460F00FFB2BF03A5
S2140136B017F480473E432E61C0B2F0BC704702004B
S2140136C0106A0860012070470200506A08600120F5
S2140136D070470200906A08600120704770B50400C8
S2140136E00D00E0684069C0F38000C0B2002801D137
S2140136F0002038E00126E068C06810F00700C0B27C
S21401370000280BD0022813D00DD304281AD014D3C6
S214013710062821D01BD307281ED022E0290020002E
S214013720FFF7CDFF1EE029002000FFF7CDFF19E0CF
S21401373029002000FFF7CDFF14E029002000FDF747
S214013740B0FA0FE029002000FDF7A9F80AE02900E9
S2140137502000FDF7A7FB05E029002000FDF7A0F9F2
S21401376000E00020C0B270BD70B40300012000224A
S214013770DC68656935F004051600F6B2B60016F089
S2140137800406354365614E78042E3CD0062E52D091
S214013790082E2CD00A2E42D04D2E04D04E2E0ED0FE
S2140137A04F2E18D053E00022DC68E568ED08ED00E6
S2140137B01600F6B216F007063543E56049E0012229
S2140137C0DC68E568ED08ED001600F6B216F00706AF
S2140137D03543E5603DE00222DC68E568ED08ED0072
S2140137E01600F6B216F007063543E56031E003220F
S2140137F0DC68E568ED08ED001600F6B216F007067F
S2140138003543E56025E00422DC68E568ED08ED0057
S2140138101600F6B216F007063543E56019E00522F4
S214013820DC68E568ED08ED001600F6B216F007064E
S2140138303543E5600DE00622DC68E568ED08ED003D
S2140138401600F6B216F007063543E56001E00022E1
S21401385010000A78002A01D0012200E00022DC686C
S214013860656935F004051600F6B2B60016F00406D2
S21401387035436561C0B270BC704770B504000D0079
S214013880E0684069C0F3C000C0B2002801D1002042
S21401389038E00126E068C068C0F30210C0B2002814
S2140138A00BD0022813D00DD304281AD014D306281F
S2140138B021D01BD307281ED022E029002000FFF7C5
S2140138C0FEFE1EE029002000FFF7FEFE19E029009B
S2140138D02000FFF7FEFE14E029002000FDF7E1F9C5
S2140138E00FE029002000FCF7DAFF0AE0290020009B
S2140138F0FDF7D8FA05E029002000FDF7D1F800E031
S2140139000020C0B270BD70B4030001200022DC6844
S214013910656935F008051600F6B2F60016F00806D9
S214013920354365614E78042E40D0062E58D0082EB9
S2140139302FD00A2E47D04D2E04D04E2E0FD04F2E0C
S2140139401AD05AE00022DC68E56835F070051600EA
S214013950F6B2360116F070063543E5604FE00122F7
S214013960DC68E56835F070051600F6B2360116F02B
S21401397070063543E56042E00222DC68E56835F012
S21401398070051600F6B2360116F070063543E5608E
S21401399035E00322DC68E56835F070051600F6B2FE
S2140139A0360116F070063543E56028E00422DC682F
S2140139B0E56835F070051600F6B2360116F07006A9
S2140139C03543E5601BE00522DC68E56835F07005E7
S2140139D01600F6B2360116F070063543E5600EE0C5
S2140139E00622DC68E56835F070051600F6B2360189
S2140139F016F070063543E56001E0002210000A78F3
S214013A00002A01D0012200E00022DC68656935F059
S214013A1008051600F6B2F60016F00806354365618D
S214013A20C0B270BC704770B504000D00E068406914
S214013A30C0F30010C0B2002801D1002039E00126F1
S214013A40E068C068000A10F00700C0B200280BD07A
S214013A50022813D00DD304281AD014D3062821D057
S214013A601BD307281ED022E029002000FFF727FEDF
S214013A701EE029002000FFF727FE19E0290020009C
S214013A80FFF727FE14E029002000FDF70AF90FE0F2
S214013A9029002000FCF703FF0AE029002000FDF7BB
S214013AA001FA05E029002000FCF7FAFF00E00020FB
S214013AB0C0B270BD70B4030001200022DC686569E5
S214013AC035F010051600F6B2360116F0100635432D
S214013AD065614E78042E40D0062E58D0082E2FD081
S214013AE00A2E47D04D2E04D04E2E0FD04F2E1AD070
S214013AF05AE00022DC68E56835F4E0651600F6B2A7
S214013B00360216F4E0663543E5604FE00122DC68D4
S214013B10E56835F4E0651600F6B2360216F4E0669E
S214013B203543E56042E00222DC68E56835F4E0658D
S214013B301600F6B2360216F4E0663543E56035E067
S214013B400322DC68E56835F4E0651600F6B2360255
S214013B5016F4E0663543E56028E00422DC68E56893
S214013B6035F4E0651600F6B2360216F4E066354323
S214013B70E5601BE00522DC68E56835F4E0651600C3
S214013B80F6B2360216F4E0663543E5600EE006222C
S214013B90DC68E56835F4E0651600F6B2360216F420
S214013BA0E0663543E56001E0002210000A78002A4D
S214013BB001D0012200E00022DC68656935F01005BD
S214013BC01600F6B2360116F0100635436561C0B22E
S214013BD070BC704770B504000D00E0684069C0F322
S214013BE04010C0B2002801D1002039E00126E0686B
S214013BF0C068000B10F00700C0B200280BD00228E6
S214013C0013D00DD304281AD014D3062821D01BD3E1
S214013C1007281ED022E029002000FFF750FD1EE0F5
S214013C2029002000FFF750FD19E029002000FFF7CA
S214013C3050FD14E029002000FDF733F80FE02900BD
S214013C402000FCF72CFE0AE029002000FDF72AF9E7
S214013C5005E029002000FCF723FF00E00020C0B2A9
S214013C6070BD70B4030001200022DC68656935F080
S214013C7020051600F6B2760116F02006354365617A
S214013C804E78042E40D0062E58D0082E2FD00A2E5D
S214013C9047D04D2E04D04E2E0FD04F2E1AD05AE0BC
S214013CA00022DC68E56835F4E0451600F6B2360316
S214013CB016F4E0463543E5604FE00122DC68E5682E
S214013CC035F4E0451600F6B2360316F4E046354301
S214013CD0E56042E00222DC68E56835F4E04516005E
S214013CE0F6B2360316F4E0463543E56035E00322C6
S214013CF0DC68E56835F4E0451600F6B2360316F4DE
S214013D00E0463543E56028E00422DC68E56835F4E2
S214013D10E0451600F6B2360316F4E0463543E56094
S214013D201BE00522DC68E56835F4E0451600F6B2CE
S214013D30360316F4E0463543E5600EE00622DC68FD
S214013D40E56835F4E0451600F6B2360316F4E046AB
S214013D503543E56001E0002210000A78002A01D010
S214013D60012200E00022DC68656935F020051600B6
S214013D70F6B2760116F0200635436561C0B270BC16
S214013D8070470200002070470200002070470200C2
S214013D900020704702000020704770B504000D0037
S214013DA0E0680069C0F38010C0B2002801D100208D
S214013DB01CE00126E0680068C0F38110C0B200284C
S214013DC003D002280BD005D30EE029002000FDF712
S214013DD091FD0AE029002000FDF767FD05E02900B6
S214013DE02000FDF73DFD00E00020C0B270BD70B4BC
S214013DF0030001200022DC68256935F04005160025
S214013E00F6B2B60116F04006354325614E78132EFC
S214013E101ED02AD3152E01D00DD326E00022DC6851
S214013E20256835F0C0051600F6B2B60116F0C006D4
S214013E30354325601BE00122DC68256835F0C005A6
S214013E401600F6B2B60116F0C006354325600EE040
S214013E500222DC68256835F0C0051600F6B2B60108
S214013E6016F0C0063543256001E0002210000A78EE
S214013E70002A01D0012200E00022DC68256935F025
S214013E8040051600F6B2B60116F040063543256128
S214013E90C0B270BC7047F0B4049C059D01604260DE
S214013EA08360C4602E6806616E684661AE6886618E
S214013EB0EE68C661002600273E00F6B2032E0DD23C
S214013EC03E00F6B205EB86063669BC465FFA8CFC08
S214013ED000EB8C0CCCF820607F1CEDE7F0BC704743
S214013EE0F8B504000E0015003000C0B2572801DBFB
S214013EF0002011E00027354A3000C0B252F83000E9
S214013F00002807D0290020003300DBB252F8332006
S214013F10904707003800C0B2F2BD2DE9F64F85B0D4
S214013F2083460C002000C0B2572801DB00204AE07F
S214013F300025264A2000C0B202EBC00040680028D7
S214013F403FD0234EDBF80070C7F88060DFF884802E
S214013F50DBF8040004900498C0F84080DFF87890FD
S214013F60DBF80C0003900398C0F84090DFF86CA0D3
S214013F70DBF8080002900298C0F880A0069958461F
S214013F802300DBB202EBC302526890470500002013
S214013F90DBF80010C1F880000022DBF80430019342
S214013FA0019B1A640023DBF80CE0CDF800E0DDF895
S214013FB000C0CCF840305FF0000CDBF808E0CEF82B
S214013FC080C02800C0B207B0BDE8F08F2C570200B1
S214013FD0E42386FA9C1FC5C177756370656D4353EC
S214013FE0010000200A00D2B2002A05D0022A09D018
S214013FF005D3032A09D00AE01022100007E0182290
S214014000100004E02822100001E048221000C0B28F
S21401401070472DE9F04704000D00206810F1800676
S2140140205FF000085FF0000AD4F8009000275046C1
S214014030C0B2002819D0022809D00FD303281BD1FB
S214014040D9F8000C400E10F00300070014E0D9F870
S214014050000C800D10F0030007000DE0D9F8000CED
S214014060C00C10F00300070006E0D9F8000C000CA5
S21401407010F003000700FFE73800C0B2FFF7B0FFFB
S2140140800100C9B289083800C0B2002807D10A0069
S214014090D2B2280080B2424316EB820636E03800E0
S2140140A0C0B201280FD10800C0B22A0092B22B007C
S2140140B09BB25FF0150C93FBFCF35B0002FB003038
S2140140C016EB800622E03800C0B202280FD10800A5
S2140140D0C0B22A0092B22B009BB25FF00C0C93FB8D
S2140140E0FCF39B0002FB003016EB80060EE0080096
S2140140F0C0B22A0092B22B009BB25FF0070C93FB72
S214014100FCF35B0002FB003016EB80063000BDE8D6
S214014110F087010000200A00D2B2002A082A0ED930
S214014120093A0ED0521E0FD0521E10D0521E11D078
S214014130521E12D0521E13D0521E14D016E0080082
S21401414014E00C22100011E0102210000EE01422E0
S21401415010000BE01822100008E02022100005E0F5
S2140141603022100002E040221000FFE7C0B2704784
S2140141702DE9F84304000D0000275FF0000929002F
S21401418089B22000FFF745FF0600D6F800805FEAF7
S214014190184818F00F084046C0B2FFF7BAFFC0B281
S2140141A0BDE8F28330B400241300DBB2002B0BD041
S2140141B0036853F4C0030360456815F0604521F0B9
S2140141C060431D4345600BE0036833F4C00303609E
S2140141D043686FF39C437F4D15EA81451D43456057
S2140141E030BC7047026832F47022026002680B002D
S2140141F0DBB21B0413F470231A4302607047026893
S21401420022F000420260026832F0804202600A0038
S214014210D2B2002A07D0026852F000420260026859
S21401422052F08042026070470A00D2B2002A06D1DC
S214014230026832F070620260026802600BE00A00F7
S214014240D2B2012A07D1026832F0706202600268B7
S21401425052F080620260704710B44168496C11F0F8
S2140142600101C9B2002909D05B494268116441685D
S214014270496C11F00101C9B20029F8D1017C00296D
S21401428020D101214268536933F080530C00E4B217
S214014290240714F080542343536144686469240F4F
S2140142A014F00104E4B2002C39D1012142685369AB
S2140142B033F080530C00E4B2240714F080542343F7
S2140142C053612CE0017C01290CD10121426853691C
S2140142D033F000530C00E4B2640714F00054234397
S2140142E053611CE0017C02290CD10121426853690B
S2140142F033F080430C00E4B2A40714F08044234357
S21401430053610CE0017C032909D1012142685369FC
S21401431023F000430C00E4B253EAC473536110BCAB
S214014320704710B42C4A43681A64017C002920D1D6
S21401433001214268136933F400730C00E4B264028D
S21401434014F400742343136144682469640A14F066
S2140143500104E4B2002C3BD101214268136933F415
S21401436000730C00E4B2640214F400742343136176
S2140143702EE0017C01290CD101214268136933F436
S21401438080630C00E4B2A40214F480642343136136
S2140143901EE0017C02290CD101214268136933F425
S2140143A000630C00E4B2E40214F4006423431361D6
S2140143B00EE0017C03290BD101214268136933F415
S2140143C080530C00E4B2240314F480542343136195
S2140143D010BC70470000FC1F7775637030B402682C
S2140143E0803200230024B4F5007F06D202EB84035A
S2140143F0190000230B60641CF5E70023802B08D20C
S21401440002EB830414F50064210000240C605B1C9D
S214014410F4E700240B2C08D202EB840313F5206387
S214014420190000230B60641CF4E700230B2B08D251
S21401443002EB830414F52364210000240C605B1C4A
S214014440F4E70024352C08D202EB840303F6A863B4
S214014450190000230B60641CF4E7036813F500538E
S2140144600025B5F5207F06D203EB85021100002258
S2140144700A606D1CF5E700220468D2B204EB8202E2
S21401448012F540520024802C06D202EB8403190058
S21401449000230B60641CF6E730BC704770B4039CC5
S2140144A0049D6E7846742E780674016042608360BF
S2140144B0C46070BC70470021816000210161002149
S2140144C04161002181610021C1600021C16100219B
S2140144D04162002181620021C16200210162012145
S2140144E001700021C170002141715FF0FF3141630D
S2140144F08163C163002180F84410002141700021CE
S2140145008170002180F83010002180F845100021CC
S21401451080F84710002180F84810002180F85110DB
S214014520002180F85010002180F85210002180F8F8
S2140145305310002180F849100021C1647047F0B47F
S21401454000210268136833F080430C00E4B2A4072C
S21401455014F0804423431360002405682E6836F067
S21401456080562700FFB23F0717F080573E432E6064
S21401457001680968090E11F00101C9B20029F7D1D5
S214014580F0BC7047F8B5040020680068000D10F014
S2140145900100C0B2002815D0002021680A6822F068
S2140145A000420300DBB252EAC3720A602068006868
S2140145B0000D10F00100C0B2002803D02000FFF764
S2140145C0B0FEF3E7012021680A6832F000720300AA
S2140145D0DBB25B0613F000731A430A6020680068BA
S2140145E0400E10F00100C0B20028F7D1012021686A
S2140145F00A6832F080420300DBB29B0713F0804367
S2140146001A430A60012325682E6836F080561F007B
S214014610FFB23F0717F080573E432E6020680068C0
S214014620000E10F00100C0B20028F7D02068006824
S214014630C00E10F00100C0B20028EFD0F1BDF8B5F1
S21401464004000D0016003100C9B289B22000FFF740
S214014650E0FC07002A7A69683800FFF7A3FDA97A0B
S2140146603800FFF7BFFDE97A3800FFF7C8FD697A21
S2140146703800FFF7D9FD287B002804D03100C9B2E5
S214014680200001F0CAFD687A012808D128693100A6
S21401469022680B00DBB202EB8303C3F88008F1BD8E
S2140146A02DE9F04F86B0040000208DF807000020A9
S2140146B08DF8060000208DF8050000208DF8040016
S2140146C0002500260020039000275FF0000E5FF013
S2140146D0000C5FF000081000C0B299465FFA89F935
S2140146E019F101095FEA59095FEA490919EB40091D
S2140146F0B9F1810F80F07C811800C0B250FA82F0C7
S2140147000128C0F275811000C0B200280CD0D00775
S21401471002D5501C050000E01500D00706D55FF055
S21401472001098DF8069001E0002005001800C0B2CE
S214014730002817D01800C0B2401C40084019B0F13C
S21401474001098DF804909DF80400402803D35FF01A
S2140147503F098DF80490D80708D55FF001098DF858
S214014760059003E0B5F101098DF804909DF80490D9
S2140147708DF80190D4F80090D9F80CAC3AF47C5A34
S2140147809DF80100000210F47C5050EA0A0ACDF8A8
S21401479008A00298C9F80C0C8DF80050D4F800A0B7
S2140147A0DAF80CBC3BF4FE0B9DF80000000410F494
S2140147B0FE0050EA0B0BCAF80CBC0020804691F8AC
S2140147C049901FFA88F81FFA89F9C84580F0A28037
S2140147D05FF01408D1F84C9082461FFA8AFA08FB5B
S2140147E00AFAD14499F80990B9F1010F40F0908086
S2140147F0D1F84C9082461FFA8AFA08FB0AFAD1448D
S21401480099F80890B9F1010F40F082801EF1010E6F
S2140148105FF0000A5FF00009CDF800A0D1F84CB0B7
S21401482082461FFA8AFA08FB0AFADA44DAF804A082
S214014830DDF800B05AEA0B0A5646D1F84CA083467A
S2140148401FFA8BFB08FB0BF8D044D8F8108028F031
S214014850604858EA0909CDF80C900596ADF808C0ED
S214014860D4F800A04FF44059BDF808800AEB880838
S214014870DDF814B048F809B01CF1010CADF800C021
S214014880DDF80C80CDF81080BDF80080ADF8028010
S214014890D4F80080BDF802C008EB8C0CDDF810B02F
S2140148A04CF809B0BDF800C01CF1010C93465FFA44
S2140148B08BFBDE452CD19DF80680B8F1000F26D083
S2140148C00596ADF808C0D4F800A0BDF808800AEB3C
S2140148D08808DDF814B048F809B01CF1010CADF8F1
S2140148E000C0DDF80C80CDF81080BDF80080ADF872
S2140148F00280D4F80080BDF802C008EB8C0CDDF80D
S21401490010B04CF809B0BDF800C01CF1010C01E074
S214014910401C53E75FF00008404691F8499080B28A
S2140149201FFA89F948455FD25FF01409C86CC24680
S2140149301FFA8AFA09FB0AFA5044407A012850D134
S214014940C86CC2461FFA8AFA09FB0AFA5044007A72
S214014950002846D17F1C0020D1F84CA0C3461FFA80
S2140149608BFB09FB0BFBDA44DAF804A050EA0A4099
S214014970D1F84CA0C3461FFA8BFB09FB0BF9D144B7
S214014980D9F810905FEA49595FEA595959EA000087
S21401499006000296ADF800C020684FF44059BDF8F5
S2140149A000A000EB8A0ADDF808B04AF809B01CF14D
S2140149B0010C9A465FFA8AFA574512D19DF805000E
S2140149C000280DD00296ADF800C02068BDF800A002
S2140149D000EB8A0ADDF808B04AF809B01CF1010CB0
S2140149E002E018F1010897E75FF001098DF80790DA
S2140149F09DF8070006B0BDE8F08F2DE9F44F85B0AD
S214014A0005000C0000208DF80600002600208DF819
S214014A10050000208DF8040000208DF8010000201C
S214014A208DF80000002100225FF0000C00275FF0E7
S214014A30000E5FF000089DF81400401C400840007E
S214014A4099465FFA89F919F1010910EB5900812895
S214014A5080F039829DF8140050FA83F00128C0F2E4
S214014A6032829DF81400002815D09DF81400C00766
S214014A7008D59DF8149019F101095FEA59098DF8D6
S214014A8000900CE09DF814905FFA89F95FEA5909E5
S214014A908DF8009003E05FF000098DF80090180093
S214014AA0C0B2002824D09DF8000099465FFA89F923
S214014AB019F101095FEA590919F101095FEA590972
S214014AC019EB0000B0F101098DF801909DF8010085
S214014AD0402803D35FF03F098DF8019013F0030FD0
S214014AE00CD013F00309D9F104098DF8059005E0FF
S214014AF09DF80000B0F101098DF801909DF8019034
S214014B008DF80390D5F80090CDF808900298D0F86B
S214014B100C9C39F47C599DF80300000210F47C507B
S214014B2050EA0909CDF80C900398DDF80890C9F809
S214014B300C0C9DF800908DF802902868D0F80CAC0B
S214014B403AF4FE0A9DF802905FEA094919F4FE0953
S214014B5059EA0A0AC0F80CAC5FF00009484694F816
S214014B60498080B21FFA88F8404580F0BD805FF02A
S214014B701408E06CCA461FFA8AFA08FB0AFA50447F
S214014B80407A012840F0AD80E06CCA461FFA8AFAE6
S214014B9008FB0AFA5044007A012840F0A2807F1CE4
S214014BA03000C0B2002849D1012006005FF0000A9B
S214014BB000200200E06CCB461FFA8BFB08FB0BFBC8
S214014BC05844406850EA0A0A51469DF81400874244
S214014BD040F0878052F08042E06CCA461FFA8AFA9B
S214014BE008FB0AF84044406802430492ADF80AE024
S214014BF0D5F800804FF4405ABDF80A0008EB800053
S214014C00DDF810B040F80AB01EF1010EADF802E072
S214014C100391BDF802E0ADF808E02868BDF808E0A9
S214014C2000EB8E0EDDF80CB04EF80AB0BDF802E0CF
S214014C301EF1010E5FF0000A564655E0E06CCA46CA
S214014C401FFA8AFA08FB0AFA5044406881420FD2DA
S214014C5052F080421000E26CCA461FFA8AFA08FB3C
S214014C600AF84244D2F80480020058EA02020CE034
S214014C70080050F080400200E06CCA461FFA8AFA2B
S214014C8008FB0AF84044406801000492ADF80AE0C7
S214014C90D5F800804FF4405ABDF80A0008EB8000B2
S214014CA0DDF810B040F80AB01EF1010EADF802E0D2
S214014CB00391BDF802E0ADF808E02868BDF808E009
S214014CC000EB8E0EDDF80CB04EF80AB0BDF802E02F
S214014CD01EF1010E5FF0000A56469DF814A05745D6
S214014CE002D019F1010939E75FF00008404694F84F
S214014CF0499080B21FFA89F9484580F07F805FF0BD
S214014D001409E06CC2461FFA8AFA09FB0AFA5044F3
S214014D10407A01286FD1E06CC2461FFA8AFA09FB75
S214014D200AFA5044007A002865D11CF1010C3000C3
S214014D30C0B2002819D101200600002050F08040A2
S214014D40D4F84CA0C3461FFA8BFB09FB0BF9D144E0
S214014D50D9F8049059EA000949461800C0B28445BA
S214014D6049D1C1468DF8049048E04805400DD4F875
S214014D704CA0C3461FFA8BFB09FB0BFBDA44DAF89F
S214014D8004A050450AD2E06CC2461FFA8AFA09FB13
S214014D900AF94844406851EA004113E04805400DCD
S214014DA002005FF08040D4F84CA0C3461FFA8BFB8C
S214014DB009FB0BF9D144D9F8049059EA000959EADC
S214014DC00249494602917046D5F80090DDF808A0E0
S214014DD083461FFA8BFB09EB8B0B1BF5405BCBF86D
S214014DE000A01EF1010E5FF0000A56469A465FFAD1
S214014DF08AFAD44502D018F1010877E79DF8050034
S214014E00002805D0022822D003D3032831D056E04B
S214014E1055E0D4F84C909DF804A0142000FB0AFA43
S214014E2009EB0A00406851EA004102917046D5F844
S214014E300090DDF808A083461FFA8BFB09EB8B0B6D
S214014E401BF5405BCBF800A01EF1010E37E0029186
S214014E507046D5F80090DDF808A083461FFA8BFB54
S214014E6009EB8B0B1BF5405BCBF800A01EF1010E86
S214014E7025E00491ADF80AE0D5F800904FF4405AC9
S214014E80BDF80A0009EB8000DDF810B040F80AB062
S214014E901EF1010EADF802E00391BDF802E0ADF897
S214014EA008E02868BDF808E000EB8E0EDDF80CB0CF
S214014EB04EF80AB0BDF802E01EF1010EFFE75FF002
S214014EC001098DF806909DF8060006B0BDE8F08F42
S214014ED02DE9F84F85B005000B00140000208DF871
S214014EE00600002600208DF8050000208DF804003D
S214014EF000208DF8010000208DF80000002100221E
S214014F0000275FF0000C5FF0000E5FF00008200045
S214014F10C0B2401C400840009DF8149019F10109E8
S214014F2010EB5900812880F001829DF8140050FA98
S214014F3084F00128C0F2FA812000C0B2002813D004
S214014F40E00709D5A1465FFA89F919F101095FEA77
S214014F5059098DF800900BE0A1465FFA89F95FEADE
S214014F6059098DF8009003E05FF000098DF8009074
S214014F709DF81400002827D09DF800009DF8149095
S214014F8019F101095FEA590919F101095FEA59099D
S214014F9019EB0000B0F101098DF801909DF80100B0
S214014FA0402803D35FF03F098DF801909DF8140067
S214014FB010F0030F0ED09DF8149019F00309D9F1E3
S214014FC004098DF8059005E09DF80000B0F101098F
S214014FD08DF801909DF801908DF80390D5F800901A
S214014FE0CDF808900298D0F80C9C39F47C599DF8BD
S214014FF00300000210F47C5050EA0909CDF80C9029
S2140150000398DDF80890C9F80C0C9DF800908DF80F
S21401501002902868D0F80CAC3AF4FE0A9DF802908B
S2140150205FEA094919F4FE0959EA0A0AC0F80CAC04
S2140150305FF00009484693F8498080B21FFA88F865
S214015040404580F0A4805FF01408D86CCA461FFA69
S2140150508AFA08FB0AFA5044407A012840F0948004
S214015060D86CCA461FFA8AFA08FB0AFA5044007A34
S214015070012840F089801CF1010C3000C0B20028E4
S21401508048D1012006005FF0000A002002005AF015
S214015090004AD86CCB461FFA8BFB08FB0BFB584427
S2140150A0406850EA0A0A51462000C0B284456BD1D6
S2140150B0D86CCA461FFA8AFA08FB0AF840444068C8
S2140150C002430491ADF80AE0D5F800804FF4405A47
S2140150D0BDF80A0008EB8000DDF810B040F80AB011
S2140150E01EF1010EADF802E00392BDF802E0ADF844
S2140150F008E02868BDF808E000EB8E0EDDF80CB07D
S2140151004EF80AB0BDF802E01EF1010E5FF0000A8B
S21401511056463CE01000DA6CCA461FFA8AFA08FBCB
S2140151200AF84244D2F80480020058EA02020491C6
S214015130ADF80AE0D5F800804FF4405ABDF80A00F1
S21401514008EB8000DDF810B040F80AB01EF1010E41
S214015150ADF802E00392BDF802E0ADF808E0286879
S214015160BDF808E000EB8E0EDDF80CB04EF80AB084
S214015170BDF802E01EF1010E5FF0000A5646A24697
S2140151805FFA8AFAD44502D019F1010952E75FF0B5
S2140151900008404693F8499080B21FFA89F94845BD
S2140151A055D25FF01409D86CC2461FFA8AFA09FB79
S2140151B00AFA5044407A012846D1D86CC2461FFAF2
S2140151C08AFA09FB0AFA5044007A00283CD17F1C6F
S2140151D03000C0B2002819D101200600002050F08E
S2140151E00040D3F84CA0C3461FFA8BFB09FB0BF912
S2140151F0D144D9F8049059EA000949469DF81400AB
S214015200874221D1C1468DF8049020E0D86CC24671
S2140152101FFA8AFA09FB0AF94844406851EA004134
S21401522002917046D5F80090DDF808A083461FFA73
S2140152308BFB09EB8B0B1BF5405BCBF800A01EF13B
S214015240010E5FF0000A564618F10108A1E79DF825
S2140152500500012804D065D3032831D01ED361E0B0
S214015260D3F84C909DF804A0142000FB0AFA09EB31
S2140152700A00406851EA004102917046D5F8009054
S214015280DDF808A083461FFA8BFB09EB8B0B1BF599
S214015290405BCBF800A01EF1010E43E00291704680
S2140152A0D5F80090DDF808A083461FFA8BFB09EBC2
S2140152B08B0B1BF5405BCBF800A01EF1010E31E015
S2140152C0D3F84C909DF804A0142000FB0AFA09EBD1
S2140152D00A00406851EA00410491ADF80AE0D5F8A9
S2140152E000904FF4405ABDF80A0009EB8000DDF843
S2140152F010B040F80AB01EF1010EADF802E00391BD
S214015300BDF802E0ADF808E02868BDF808E000EB5B
S2140153108E0EDDF80CB04EF80AB0BDF802E01EF1B4
S214015320010EFFE75FF001098DF806909DF8060073
S21401533006B0BDE8F08F2DE9F04704000D00002609
S214015340002700205FF000085FF000095FF0000A08
S214015350504695F84910C0B2884227D21421E86C0D
S2140153605246D2B24A431044407A01281BD1E86C17
S2140153705246D2B24A431044007A002801D17F1C1B
S21401538000E0761CE86C5246D2B201FB02F10844FA
S214015390807AFEF7BEFE814640464946C0B2C9B293
S2140153A0884200D2C8461AF1010AD1E76879012875
S2140153B018D100204146C9B21031042291FBF2F106
S2140153C0491E0A002368D3F80CCC3CF0F84C9646EC
S2140153D05FFA8EFE5FEA8E6E1EF0F84E5EEA0C0CE9
S2140153E0C3F80CCC95F85500002803D0022813D03A
S2140153F009D31AE03B00DBB23200D2B2290020000A
S214015400FFF74EF911E03B00DBB23200D2B22900C1
S2140154102000FFF7F2FA08E03B00DBB23200D2B21E
S21401542029002000FFF754FDFFE7BDE8F0872DE9CE
S214015430F24F88B0040000208DF805002568286822
S21401544030F000509DF80510490711F0005108434F
S21401545007900798286001208DF804002668D6F882
S2140154600C0C20F000409DF8041050EAC170069024
S2140154700698C6F80C0C2768D7F8140C50F0006094
S214015480C7F8140C00208DF80300D4F80080D8F873
S214015490100C20F000409DF8031050EAC1700590F2
S2140154A00598C8F8100C00208DF80200D4F800907A
S2140154B0D9F8100C30F080409DF80210890711F0E1
S2140154C08041084304900498C9F8100C00208DF818
S2140154D00100D4F800A0DAF8100C30F000509DF866
S2140154E00110490711F00051084303900398CAF8C8
S2140154F0100C00208DF80000D4F800B0DBF8100C7A
S21401550030F080509DF80010090711F080510843D3
S21401551002900298CBF8100C08992000FFF70BFFB9
S21401552000202168D1F80C2C520952010300DBB28D
S21401553013F01F031A43C1F80C2C09B0BDE8F08F15
S2140155402DE9F04F8BB004000D0000208DF801000E
S2140155502000FEF781FE01208DF8030026683068E2
S21401556020F000409DF8031050EAC17004900498A2
S214015570306028788DF800002768786830F400508D
S2140155809DF80010490311F4005108430390039855
S21401559078602000FEF7F6FF5FF00108D4F800906F
S2140155A0D9F8000030F400004146C9B2C90511F42B
S2140155B00001084302900298C9F800005FF0010A52
S2140155C0D4F800B0DBF8340030F080505146C9B250
S2140155D0090711F08051084301900198CBF8340077
S2140155E02000FEF7FBFE95F83000FEF7F9FC8DF87B
S2140155F002009DF80200002809D04FF400709DF8C3
S2140156000210B0FBF1F1607C41438DF801109DF86A
S21401561001008DF8030021680868C009C0019DF8E3
S214015620032012F07F02104309900998086095F84C
S21401563059008DF800002268506830F080009DF80F
S2140156400030DB0113F0800318430890089850607F
S21401565001232668306D20F000401F00FFB250EA9B
S214015660C770079007983065A868401EADF80A0015
S2140156702768386D6FF35E50BDF80AC0DFF8C8E9D9
S2140156801EEA4C5E5EEA0000069006983865E868F9
S214015690401EADF80800D4F800E0DEF8500030F403
S2140156A0F810BDF808C05FEA0C4C1CF4F81C5CEA64
S2140156B0000005900598CEF850002869401EADF808
S2140156C00600D4F80080D8F8500030F47C40BDF8CD
S2140156D006C05FEA8C2C1CF47C4C5CEA000004904B
S2140156E00498C8F850006869401EADF80400D4F864
S2140156F00090D9F8500030F47870BDF804C05FEA25
S2140157004C1C1CF4787C5CEA000003900398C9F8F2
S2140157105000A869B0F1010AD4F800C0DCF850B016
S2140157205FEA5B1B5FEA4B1B504680B210F01F001E
S21401573050EA0B0BCCF850B06878002800F0B9811D
S21401574068788DF803002168086830F400609DF8D9
S2140157500320D20212F4006210430A900A980860ED
S21401576001222368D3F8000C20F000401600F6B2A0
S21401577050EAC67009900998C3F8000CE869401E03
S214015780ADF80C002668D6F8040C6FF31D50BDF872
S2140157900C70DFF8B8C81CEA075C5CEA00000890E9
S2140157A00898C6F8040C286A401EADF80A00276857
S2140157B0D7F8040C30F4E020BDF80AC05FEA0C4CC0
S2140157C01CF4E02C5CEA000007900798C7F8040C6C
S2140157D0686AADF80800D4F800E0DEF8040C30F48E
S2140157E0F840BDF808C05FEA8C2C1CF4F84C5CEA63
S2140157F0000006900698CEF8040CA86A401EADF884
S2140158000600D4F80080D8F8040C30F0E000BDF8AB
S21401581006C05FEA4C1C1CF0E00C5CEA0000059038
S2140158200598C8F8040CE86A401EADF80400D4F8E0
S2140158300090D9F8040CC008C000BDF804C01CF0E4
S214015840070C5CEA000004900498C9F8040C95F86B
S21401585030008DF800005FF0000CD4F800A0DAF8F4
S214015860000CE3465FFA8BFBBBF1000F24D0BBF1C3
S214015870020F0DD016D3BBF1030F27D130F0C06055
S21401588001009DF80000400610F0C06008431DE0CE
S21401589030F4400001009DF80000800510F440003F
S2140158A0084313E030F4C01001009DF80000C00466
S2140158B010F4C010084309E030F4403001009DF8B0
S2140158C00000000410F440300843FFE7CAF8000C5B
S2140158D095F8301001222368D3F8006C1700FFB248
S2140158E0002F22D0022F0CD015D3032F27D136F04C
S2140158F0C06630000E00F6B2760616F0C0660643A5
S2140159001DE036F4400630000E00F6B2B60516F479
S2140159104006064313E036F4C01630000E00F6B219
S214015920F60416F4C016064309E036F44036300095
S2140159300E00F6B2360416F440360643FFE7C3F807
S214015940006C95F830005FF0020E2768D7F800CC9F
S214015950F0465FFA88F8B8F1000F2DD0B8F1020FC3
S21401596010D01CD3B8F1030F33D13CF0C06C6146A4
S21401597084465FFA8CFC5FEA4C6C1CF0C06C5CEAF7
S214015980010C26E03CF4400C614684465FFA8CFC30
S2140159905FEA8C5C1CF4400C5CEA010C19E03CF4F8
S2140159A0C01C614684465FFA8CFC5FEACC4C1CF452
S2140159B0C01C5CEA010C0CE03CF4403C61468446A9
S2140159C05FFA8CFC5FEA0C4C1CF4403C5CEA010C70
S2140159D0FFE7C7F800CC95F8301003222368D3F808
S2140159E0006C90465FFA88F8B8F1000F24D0B8F141
S2140159F0020F0DD016D3B8F1030F27D136F0C066CB
S214015A0030000E00F6B2760616F0C06606431DE0BC
S214015A1036F4400630000E00F6B2B60516F440061F
S214015A20064313E036F4C01630000E00F6B2F60454
S214015A3016F4C016064309E036F4403630000E0070
S214015A40F6B2360416F440360643FFE7C3F8006C98
S214015A5095F84500002820D195F847002168D1F82F
S214015A60002C32F400420300DBB2DB0313F40043E4
S214015A701A43C1F8002C95F848302668D6F8007C01
S214015A8037F4F8579C465FFA8CFC5FEA0C2C1CF442
S214015A90F85C5CEA0707C6F8007CA87821684A6BC0
S214015AA032F480520300DBB21B0313F480531A4313
S214015AB04A63E878002843D0207C00280BD10020D8
S214015AC02168D1F80C2C22F000420300DBB252EA26
S214015AD0C372C1F80C2C012021680A6832F000520A
S214015AE00300DBB25B0713F000531A430392039AD9
S214015AF00A602A6C02922268029B93646B6B019384
S214015B002368019E1E61AE6B27687E61D5F83CC096
S214015B10D4F800E0CEF818C095F84480D4F8009088
S214015B20D9F800A03AF4803AC3465FFA8BFB5FEAE5
S214015B300B4B1BF4803B5BEA0A0AC9F800A09AE00B
S214015B402879002808D0207C002840F0948029007D
S214015B502000FFF76CFC8EE000212268136833F00A
S214015B6000530800C0B2400710F000500343136012
S214015B70207C002863D100208DF800002068D0F832
S214015B800C1C21F000419DF8002051EAC2710491DD
S214015B900499C0F80C1C2168D1F8142C52F000624C
S214015BA0C1F8142C00222368D3F8106C26F00046A6
S214015BB01700FFB256EAC7760396039EC3F8106C29
S214015BC000262768D7F810EC3EF0804EB4465FFA00
S214015BD08CFC5FEA8C7C1CF0804C5CEA0E0ECDF8E7
S214015BE008E0DDF808C0C7F810CC5FF0000ED4F866
S214015BF00080D8F8109C39F00059F4465FFA8CFC06
S214015C005FEA4C7C1CF0005C5CEA0909CDF8049064
S214015C10DDF804C0C8F810CC5FF0000CD4F8009092
S214015C20D9F810AC3AF0805AE3465FFA8BFB5FEA8C
S214015C300B7B1BF0805B5BEA0A0AC9F810AC686B49
S214015C4021680861AA6B23685A61EE6B2768BE61FA
S214015C5095F844C0D4F800E0DEF8008038F48038C7
S214015C60E1465FFA89F95FEA094919F4803959EA88
S214015C700808CEF8008069792268136833F4004377
S214015C800800C0B2C00310F400400343136095F847
S214015C90450000281BD0002021680A6832F4003233
S214015CA00300DBB25B0413F400331A430A600123DA
S214015CB02668776837F480579C465FFA8CFC5FEA63
S214015CC00C3C1CF4805C5CEA070777601AE0012054
S214015CD021680A6832F400320300DBB25B0413F475
S214015CE000331A430A6000232668776837F4805722
S214015CF09C465FFA8CFC5FEA0C3C1CF4805C5CEA18
S214015D000707776095F846102268536833F0080352
S214015D100800C0B2C00010F008000343536095F8B5
S214015D20500000282ED0012021680A6832F4800233
S214015D300300DBB29B0513F480031A430A600123B8
S214015D402668376837F080679C465FFA8CFC5FEA06
S214015D508C6C1CF0806C5CEA070737605FF0010C06
S214015D60D4F800E0DEF8008038F48028E1465FFAD7
S214015D7089F95FEA894919F4802959EA0808CEF8B1
S214015D8000802DE0002021680A6832F480020300BA
S214015D90DBB29B0513F480031A430A6000232668CE
S214015DA0376837F080679C465FFA8CFC5FEA8C6C3C
S214015DB01CF0806C5CEA070737605FF0000CD4F8D3
S214015DC000E0DEF8008038F48028E1465FFA89F9C1
S214015DD05FEA894919F4802959EA0808CEF8008053
S214015DE001212268506830F0400006900698506005
S214015DF095F851008DF806002368186830F4805035
S214015E009DF80660360316F48056304305900598D3
S214015E10186095F852008DF805002668706830F411
S214015E2000409DF80570FF0317F4004738430490BF
S214015E300498706095F853008DF804002768786818
S214015E4030F480409DF804C05FEA8C3C1CF4804C22
S214015E505CEA000003900398786095F854008DF88A
S214015E600300D4F800E0DEF8000030F400109DF8DE
S214015E7003C05FEA4C5C1CF4001C5CEA0000029064
S214015E800298CEF8000095F854008DF80000D4F87A
S214015E9000C0DCF8048038F400689DF80000C002F9
S214015EA010F4006050EA0808CCF8048095F854A075
S214015EB0D4F80090D9F804B03BF4806B5046C0B2D9
S214015EC0800210F4806050EA0B0BC9F804B0287900
S214015ED000282ED100200026300095F84910C0B2C7
S214015EE088425DD200201427E96C3200D2B27A4390
S214015EF031F80280404680B2E96C3200D2B27A4371
S214015F00895AEA6C3300DBB27B431A445288511833
S214015F1088420CDA4246D2B2E86C3100C9B2794303
S214015F2001442000FEF78BFB18F10108E2E7761C1E
S214015F30D2E700200026300095F84910C0B288420A
S214015F402ED200201427E96C3200D2B27A4331F8FF
S214015F500280404680B2E96C3200D2B27A43895A56
S214015F60EA6C3300DBB27B431A44528851188842EC
S214015F7014DAE86C3100C9B279430844407A002843
S214015F8009D14246D2B2E86C3100C9B27943014424
S214015F902000FEF754FB18F10108DAE7761CCAE781
S214015FA095F856008DF800002668706B30F40040B6
S214015FB09DF80010C90311F40041084302900298AD
S214015FC0706395F85870D4F80080D8F8340030F42F
S214015FD040703900C9B2090211F4407108430190BA
S214015FE00198C8F8340095F85790D4F800A0DAF86C
S214015FF034B03BF0C00B4846C0B2800110F0C00080
S21401600050EA0B0BCAF834B0200000F089F8207C67
S214016010002807D12879012804D15FF070412000BB
S21401602000F000FB2000FEF78AFA002021680A68CB
S21401603032F400020300DBB2DB0513F400031A435B
S2140160400A600BB0BDE8F08F0000E07F0000F03F73
S21401605038B504000D00297889B22000FDF7D9FF74
S214016060016851F04061016031BDF8B504000D00D2
S214016070297889B22000FDF7CCFF10F108062978AF
S21401608089B22000FEF774F8002100221100C9B27F
S214016090814244D212F0030F0AD1002131603168E7
S2140160A01300DBB22B441B7A51EA0361316034E002
S2140160B01100C9B2042391FBF3F703FB1711012961
S2140160C008D131681300DBB22B441B7A51EA034135
S2140160D0316022E01100C9B2042391FBF3F703FB00
S2140160E01711022908D131681300DBB22B441B7A41
S2140160F051EA0321316010E01100C9B2042391FB7B
S214016100F3F703FB1711032907D133681100C9B24E
S2140161102944097A0B433360361D521CB6E7F1BD9C
S214016120F0B4417C032937D15FF0FF310A00022623
S2140161300368002E0AD0022E04D005D3032E07D101
S2140161401A6705E05A6703E0DA6201E01A63FFE7BF
S2140161500C0001270568002F0AD0022F04D005D3B2
S214016160032F07D12C6705E06C6703E0EC6201E0C2
S2140161702C63FFE700230268002B0AD0022B04D011
S21401618005D3032B07D1116705E0516703E0D16200
S21401619001E01163FFE73EE0417C022925D15FF073
S2140161A0FF310A0001250368002D0AD0022D04D014
S2140161B005D3032D07D11A6705E05A6703E0DA62B3
S2140161C001E01A63FFE700260468002E0AD0022EBB
S2140161D004D005D3032E07D1216705E0616703E0EC
S2140161E0E16201E02163FFE715E0417C012912D15C
S2140161F05FF0FF3100230268002B0AD0022B04D087
S21401620005D3032B07D1116705E0516703E0D1627F
S21401621001E01163FFE7F0BC7047F0B400240A0008
S214016220D2B2202392FBF3F503FB15220123934000
S2140162300D00EDB2402D1ADB1C0002260568002E6B
S21401624010D0022E06D009D3032E0FD1AF6E2743EE
S214016250AF660BE0EF6E2743EF6607E06F6A2743F2
S2140162606F6203E0AF6A2743AF62FFE738E00C00D6
S214016270E4B2202C1ADB1C0001260568002E10D083
S214016280022E06D009D3032E0FD1AF6E2743AF6679
S2140162900BE0EF6E2743EF6607E06F6A27436F62F6
S2140162A003E0AF6A2743AF62FFE719E01C00002650
S2140162B00568002E10D0022E06D009D3032E0FD16A
S2140162C0AF6E2743AF660BE0EF6E2743EF6607E03E
S2140162D06F6A27436F6203E0AF6A2743AF62FFE747
S2140162E0F0BC70472DE9F14F2DED068B8AB008EE14
S2140162F0101A08EE902A9A469FED840A012005900E
S214016300012004905FF00809032001900221142067
S21401631008909FED7F9AF5EE009A9DF86C00002894
S21401632010D040F2FF3007905E24032006901F2015
S2140163300290DDF8088018EB040818F101085FF0F8
S214016340080B0FE040F2FF3007902624032006904A
S21401635007200290DDF8088018EB040818F1010800
S2140163605FF0080BF8EE680A01250798A84246DB9D
S214016370B8EE480A01EE105AB8EEC11A80EE010ACC
S214016380B8EE681A80EE011ABDEEC11A8DED001A3C
S2140163900098002802D00098584500DA2FE09DEDBD
S2140163A0001AB8EEC11A80EE011AF8EE681A71EEFC
S2140163B0611AF5EE401AF1EE10FA04DDF8EE681AED
S2140163C071EE611A03E0F8EE681A71EEC11A0098D0
S2140163D0804512DBF4EE610AF1EE10FA0DDB05954D
S2140163E000988146F0EE610A0898009A904204DB14
S2140163F0F4EE491AF1EE10FA01D46D1CB5E75046D9
S21401640080B200EE100AB8EE400A20EE290AA14535
S21401641000DA4C4626000698864227DB721C42F2BA
S2140164201070424392FBF9F0524692B2821A012A48
S21401643005DB524692B2821A00EE902A04E05246DA
S21401644092B2121A00EE902A524692B290420DDB98
S214016450B8EEE01AB4EE401AF1EE10FA04D5019641
S214016460F8EEE00AB0EE600A761ED4E70198B9EBC2
S2140164700000401E03909FED27AA01270398B8420B
S21401648023DB42F2107000FB07F090FBF9F0BDF839
S2140164906810411A012905DBBDF86810411A00EEA3
S2140164A0101A04E0BDF86810091A00EE101AF8EE8A
S2140164B0C00AF4EE4A0AF1EE10FA04D50497B8EED3
S2140164C0C00AB0EE40AA7F1CD8E70598109908606C
S2140164D0019800F09FF95FF033320F4B00F0ACF9F2
S2140164E000F080FA10998860019910988068091A5E
S2140164F01098C16003981099086104981099486033
S2140165000AB0BDEC068BBDE8F18F0000000000006C
S214016510CDCCCC3D00401C463333E33F70B4130072
S214016520DBB2012B3ED1CB000DD501230468D4F894
S214016530105C35F080551E00F6B2360716F0805610
S2140165403543C4F8105C8B000DD501230468D4F8DC
S214016550105C35F000551E00F6B2760716F00056B0
S2140165603543C4F8105C4B000DD501230468D4F8FC
S214016570105C35F080451E00F6B2B60716F0804670
S2140165803543C4F8105C00294AD501230468D4F8C1
S214016590105C25F000451E00F6B255EAC675C4F833
S2140165A0105C3DE0CB000DD500230468D4F8105CE8
S2140165B035F080551E00F6B2360716F08056354384
S2140165C0C4F8105C8B000DD500230468D4F8105C69
S2140165D035F000551E00F6B2760716F00056354324
S2140165E0C4F8105C4B000DD500230468D4F8105C89
S2140165F035F080451E00F6B2B60716F080463543E4
S214016600C4F8105C00290BD500230468D4F8105C8C
S21401661025F000451E00F6B255EAC675C4F8105CB2
S21401662070BC7047CA0004D502685FF08053C2F898
S214016630143C8A0004D502685FF00053C2F8143C8B
S2140166404A0004D502685FF08043C2F8143C002972
S21401665004D502685FF00043C2F8143C704702009C
S21401666000200B00B3F1805F09D0B3F1005F12D0B8
S214016670B3F1804F1BD0B3F1004F24D02DE0136847
S214016680D3F8143C1B0F13F00103DBB2002B01D02F
S2140166900123180021E01368D3F8143C5B0F13F0B4
S2140166A00103DBB2002B01D00123180015E01368AB
S2140166B0D3F8143C9B0F13F00103DBB2002B01D07F
S2140166C00123180009E01368D3F8143CDB0FDBB292
S2140166D0002B01D001231800FFE7C0B2704701006C
S2140166E000200A68D2F8142C520C12F00102D2B221
S2140166F0002A01D001221000C0B27047010000201C
S2140167000A68D2F8142C120C12F00102D2B2002A36
S21401671001D001221000C0B27047010000220868B3
S214016720D0F8140C10F03F00C0B270472DE9F047C6
S21401673004000D00206810F5005A5FF000090026DD
S214016740DAF800703F0C17F00F07DAF80000A5F82A
S2140167504A003800C0B2FDF7DCFC85F84800DAF8DC
S2140167600000C0F3405818F001081AF10400414631
S214016770C9B2002904D0016821F06041696003E0D4
S2140167800168C1F38A416960001D5FF0000949464E
S21401679095F84820C9B2914232D219F0030F06D1BA
S2140167A00168090E4A46D2B22A44117225E04946CA
S2140167B0C9B2042291FBF2F302FB1311012906D19F
S2140167C00168090C4A46D2B22A44117215E04946BC
S2140167D0C9B2042291FBF2F302FB1311022906D17E
S2140167E00168090A4A46D2B22A44117205E00168D4
S2140167F04A46D2B22A441172001D19F10109C6E7B0
S214016800061D3068E8645FF080512000FFF70AFF3C
S214016810BDE8F08710F0004160B148BF4042B0FAD1
S21401682080F29040D21CC2F5846241EA025202EB29
S214016830D02140057047020030B540F2FF7C1CEACB
S21401684011541DBF1CEA1355644565453FE06419A4
S21401685081EA030C6FF35F530CF0004C43F4801392
S214016860C90241F0004141EA505EC5021100A5FB94
S214016870020200284FF00000EEFB01204FF000015D
S214016880E3FB052118BF42F00102401800214941EF
S214016890E3FB0E01A4F580640D0302D29218404179
S2140168A0494154F1010470DD450872F1004250F18E
S2140168B0000051EB0451A1F5801102D441EA0C010C
S2140168C030BD40F2FF7E4CEA0E51002030BD0CEA8E
S2140168D01355644518BF654581EA030C0CF0004C5E
S2140168E041D050EA410E1CBF52EA430E02E0614617
S2140168F0002030BD24422C441BD15FEA050EF6D0A1
S214016900090302BF01460020AEF1140EB1FA81F56B
S214016910AEEB050401FA05FE0C35C5F1200100FABF
S21401692005F5C8404EEA000E6FF35F5343F480133B
S2140169309CE733F00043B3FA83F504BFB2FA82FE54
S21401694075440B3D641BB5F1200E2FBF02FA0EF302
S214016950AB40C5F1200E22FA0EFE38BF43EA0E0305
S214016960AA40641C7CE750EA410E14BF52EA430E6B
S2140169706FF000014FF4001515EB430F8EBF19465B
S21401698015EB410F9DE7B4D830BDD4F10104B4F145
S21401699020050FDAC4F12005520828BF42F0010293
S2140169A010FA05FE01FA05F57244E2BFE0402843FD
S2140169B0E1400FE0352C9ADCC5F1200452EA400292
S2140169C020FA05F218BF42F0010231FA05F0A140A3
S2140169D00A43002172F1004250F1000051EB0C0114
S2140169E030BDFEE7400D40F21E4C40EAC120BCEB34
S2140169F0115C40F0004003D48CF30701C840704797
S214016A006FEAE1707047FEE710B4020012B2002A86
S214016A1006D40A01DFF82435040024B21A5509E029
S214016A200A01DFF81C35040024B214F00F042344D5
S214016A3003F8042C10BC704710B50400601EB0F1BA
S214016A40807F01D3012011E0601EDFF8F814086092
S214016A500F215FF0FF30FFF7D7FF0020DFF8E814C3
S214016A6008600720DFF8E4140860002010BD38B580
S214016A7086B000200590DFF81C4514F5FC7001F087
S214016A8085FFDFF8CC14002002F0E9F901208DF82B
S214016A90000014F118056A4620212800FDF73DFA8A
S214016AA06A4621212800FDF738FA6A462221280085
S214016AB0FDF733FA6A4623212800FDF72EFA6A46C7
S214016AC024212800FDF729FA01208DF80000032073
S214016AD08DF801000120ADF804006A460B2128005C
S214016AE0FDF71BFA01208DF8000000208DF801004B
S214016AF00120ADF804006A4605212800FDF70DFACD
S214016B0001208DF800000B208DF801006A46432114
S214016B102800FDF702FA14F5F070006E05900321C7
S214016B2005A802F02DFF01208DF800006A463421E9
S214016B302800FDF7F2F96A4635212800FDF7EDF940
S214016B4001208DF8000003208DF801000420ADF827
S214016B5004006A464B212800FDF7DFF96A464C21FE
S214016B602800FDF7DAF901208DF800006A46332186
S214016B702800FDF7D2F901208DF800006A4626218B
S214016B802800FDF7CAF96A4636212800FDF7C5F93F
S214016B9001208DF8000005208DF801006A46452188
S214016BA02800FDF7BAF907B030BDF0B5C5B0002032
S214016BB00100C9B20A2907DA0021E64A0300DBB25E
S214016BC042F82310401CF3E7E3480088ADF82400A0
S214016BD0E2480A90EF4C14F5F27509A9280003F073
S214016BE044FADF4FDF4838601030786040A803F081
S214016BF080FB14F15C0640AADB49300003F0ABFBD6
S214016C0005A803F09BFB00208DF8140046208DF8A4
S214016C10160000208DF8150005AA3900300003F093
S214016C2000FC01208DF8140047208DF81600002086
S214016C308DF8150005AA3900300003F0F2FB052097
S214016C40019001208DF8080001208DF80900002030
S214016C50039000208DF8100000208DF81100002010
S214016C608DF8120000208DF81300206810F5C07012
S214016C700B90B84F0C9702208DF834000420ADF825
S214016C8036000420ADF838007FF013000F90109006
S214016C9000208DF8440000208DF845000420129055
S214016CA000208DF84C000020149000208DF8540030
S214016CB001208DF8550001A816900BAA002130007E
S214016CC003F086FCE06810F5C0700B9017F1140015
S214016CD00C900BAA0121300003F07AFC0021300051
S214016CE003F094FC0121300003F090FC17A804F097
S214016CF06FFD01208DF85C0001208DF86A000320ED
S214016D008DF8690000208DF8680003208DF86B006F
S214016D1000208DF86D0001208DF86F000F208DF892
S214016D20710007208DF8730001208DF89F00012067
S214016D308DF8610017A9200004F0BCFB200004F0C8
S214016D408CFD05208DF86B0002208DF86D00072064
S214016D508DF86F001A208DF8710019208DF87300D8
S214016D6014F10C0617A9300004F0A4FB300004F05F
S214016D7074FD6A46342114F11800FDF7B1F829A80C
S214016D8004F042FE00208DF8A40000208DF8A80033
S214016D9001208DF8AB0007208DF8A70003208DF8A1
S214016DA0AA0002208DF8E00003208DF8E100032000
S214016DB08DF8E20003208DF8E30003208DF8E4004F
S214016DC00098C0092821B0FBF1F04FF47A71B0FBAE
S214016DD0F1F0ADF8AC000020ADF8B00000208DF861
S214016DE0FE0014F58C7629A9300004F069FE14F52E
S214016DF0907429A9200004F063FE300004F03FFDE2
S214016E00200004F03CFD0A21280003F0D9F945B022
S214016E10F0BD30B585B0002000905E4C6A460E216C
S214016E2014F11800FDF75CF8504D280005F03EF807
S214016E3000986421B0FBF1F028600120287114F558
S214016E40AE742900200005F013F801A805F099F8A2
S214016E5000208DF8040004208DF8050001208DF82F
S214016E60100002208DF811000020029000200390EF
S214016E7001AA0021200005F01EF8200005F08AF87E
S214016E8005B030BD10B586B0394C200001F0A4FD28
S214016E90684601F05DFD01208DF8000000208DF8A8
S214016EA0010000208DF8030001208DF80400002069
S214016EB08DF8050001208DF8060000208DF80800E9
S214016EC04FF4485004904FF47A70039069462000BE
S214016ED001F00AFC06B010BD80B500200090FFF757
S214016EE0D1FFFFF7C4FD2349002001F0B8FF05F0EC
S214016EF0B1F805F0D0FA00F045F86A460D211E48B3
S214016F00FCF7EEFF00984FF47A71B0FBF1F0FFF753
S214016F1093FD4FF6FF7005F025FC05F091FC17492F
S214016F20002001F09CFFFFF740FEFFF772FF05F01F
S214016F30ACFF1349002001F092FF01BD00E400E020
S214016F4018ED00E014E000E018E000E010E000E0DA
S214016F5018810200402F002036680100F8810200E7
S214016F60A82F0020E82F0020682F0020E8300020FE
S214016F70B833002074810200D831002088810200D5
S214016F80308102002DE9F04FADF5806D83B0014CE4
S214016F9002E000BFC031002014F5A07601220121D5
S214016FA0300006F036F801208DF850000120B09030
S214016FB0D4F84001AF90AF98B09950F8210030F066
S214016FC040009DF85010890111F040010843CDF8AA
S214016FD00804DDF80804AF99B09A41F822000120B0
S214016FE08DF84F000120AE90D4F84001AD90AD98D9
S214016FF0AE9950F8210030F020009DF84F1049015D
S21401700011F020010843CDF80404DDF80404AD991D
S214017010AE9A41F8220001220121300006F02EF836
S21401702001220021300005F0F4FF01208DF84E000A
S2140170300020AC90D4F84001AB90AB98AC9950F8D6
S214017040210030F040009DF84E10890111F04001FA
S2140170500843CDF80004DDF80004AB99AC9A41F87A
S214017060220001208DF84D000020AA90D4F840019E
S214017070A990A998AA9950F8210030F020009DF80F
S2140170804D10490111F020010843FF90FF98A9997E
S214017090AA9A41F8220001220021300005F0EEFFF5
S2140170A014F5A47501220B21280005F0B2FF01207A
S2140170B08DF84C000B20A890D4F84801A790A7980B
S2140170C0A89950F8210030F040009DF84C10890135
S2140170D011F040010843FE90FE98A799A89A41F83E
S2140170E0220001208DF84B000B20A690D4F8480111
S2140170F0A590A598A69950F8210030F020009DF89B
S2140171004B10490111F020010843FD90FD98A59907
S214017110A69A41F8220001220B21280005F0AEFFB5
S21401712001220A21280005F074FF01208DF84A008B
S2140171300A20A490D4F84801A390A398A49950F8E3
S214017140210030F040009DF84A10890111F04001FD
S2140171500843FC90FC98A399A49A41F822000120C8
S2140171608DF849000A20A290D4F84801A190A19870
S214017170A29950F8210030F020009DF849104901ED
S21401718011F020010843FB90FB98A199A29A41F8BF
S214017190220001220A21280005F070FF01220521A4
S2140171A0280005F036FF01208DF848000520A09044
S2140171B0D4F848019F909F98A09950F8210030F08C
S2140171C040009DF84810890111F040010843FA90EB
S2140171D0FA989F99A09A41F8220001208DF847005D
S2140171E005209E90D4F848019D909D989E9950F850
S2140171F0210030F020009DF84710490111F02001D0
S2140172000843F990F9989D999E9A41F82200012227
S2140172100521280005F032FF01220421280005F08F
S214017220F8FE01208DF8460004209C90D4F8480111
S2140172309B909B989C9950F8210030F040009DF857
S2140172404610890111F040010843F890F8989B997F
S2140172509C9A41F8220001208DF8450004209A905E
S214017260D4F84801999099989A9950F8210030F0ED
S21401727020009DF84510490111F020010843F790C0
S214017280F79899999A9A41F8220001220421280038
S21401729005F0F4FE01220321280005F0BAFE0120C4
S2140172A08DF8440003209890D4F848019790979859
S2140172B0989950F8210030F040009DF8441089015B
S2140172C011F040010843F690F6989799989A41F87C
S2140172D0220001208DF8430003209690D4F848013F
S2140172E095909598969950F8210030F020009DF8D9
S2140172F04310490111F020010843F590F59895993E
S214017300969A41F8220001220321280005F0B6FED4
S21401731001221021300005F07CFE01208DF842008C
S21401732010209490D4F8400193909398949950F833
S214017330210030F040009DF84210890111F0400113
S2140173400843F490F4989399949A41F82200012006
S2140173508DF8410010209290D4F8400191909198B8
S214017360929950F8210030F020009DF84110490113
S21401737011F020010843F390F3989199929A41F8FD
S214017380220001221021300005F078FE01220F2193
S214017390300005F03EFE01208DF840000F20909051
S2140173A0D4F840018F908F98909950F8210030F0D2
S2140173B040009DF84010890111F040010843F29009
S2140173C0F2988F99909A41F8220001208DF83F009B
S2140173D00F208E90D4F840018D908D988E9950F89C
S2140173E0210030F020009DF83F10490111F02001E6
S2140173F00843F190F1988D998E9A41F82200012266
S2140174000F21300005F03AFE01220921280005F07F
S21401741000FE01208DF83E0009208C90D4F848012A
S2140174208B908B988C9950F8210030F040009DF895
S2140174303E10890111F040010843F090F0988B99B5
S2140174408C9A41F8220001208DF83D0009208A908F
S214017450D4F84801899089988A9950F8210030F02B
S21401746020009DF83D10490111F020010843EF90DE
S214017470EF9889998A9A41F8220001220921280069
S21401748005F0FCFD01220821280005F0C2FD0120BF
S2140174908DF83C0008208890D4F84801879087989A
S2140174A0889950F8210030F040009DF83C10890181
S2140174B011F040010843EE90EE988799889A41F8BA
S2140174C0220001208DF83B0008208690D4F8480160
S2140174D085908598869950F8210030F020009DF817
S2140174E03B10490111F020010843ED90ED98859974
S2140174F0869A41F8220001220821280005F0BEFDE7
S21401750014F5987701220521380005F082FD012047
S2140175108DF83A0005208490D4F830018390839842
S214017520849950F8210030F040009DF83A10890106
S21401753011F040010843EC90EC988399849A41F845
S214017540220001208DF8390005208290D4F8300100
S21401755081908198829950F8210030F020009DF8A2
S2140175603910490111F020010843EB90EB988199FD
S214017570829A41F8220001220521380005F07EFD9D
S21401758001220421380005F044FD01208DF8380061
S21401759004208090D4F830017F907F98809950F82D
S2140175A0210030F040009DF83810890111F04001AB
S2140175B00843EA90EA987F99809A41F822000120D0
S2140175C08DF8370004207E90D4F830017D907D98A8
S2140175D07E9950F8210030F020009DF837104901BF
S2140175E011F020010843E990E9987D997E9A41F8C7
S2140175F0220001220421380005F040FD0122062167
S214017600300005F006FD01208DF8360006207C903E
S214017610D4F840017B907B987C9950F8210030F09B
S21401762040009DF83610890111F040010843E890AA
S214017630E8987B997C9A41F8220001208DF8350064
S21401764006207A90D4F84001799079987A9950F882
S214017650210030F020009DF83510490111F020017D
S2140176600843E790E79879997A9A41F8220001222F
S2140176700621300005F002FD01220521300005F04B
S214017680C8FC01208DF8340005207890D4F840011C
S21401769077907798789950F8210030F040009DF85F
S2140176A03410890111F040010843E690E698779975
S2140176B0789A41F8220001208DF833000520769053
S2140176C0D4F8400175907598769950F8210030F0FD
S2140176D020009DF83310490111F020010843E59080
S2140176E0E5987599769A41F8220001220521300025
S2140176F005F0C4FC14F59C7900221121484605F0DA
S21401770088FC01208DF8320001207490D4F83801ED
S21401771073907398749950F8210030F004009DF826
S2140177203210890011F004010843E490E49873993B
S214017730749A41F8220001208DF8310001207290E0
S214017740D4F8380171907198729950F8210030F090
S21401775020009DF83110490111F020010843E39003
S214017760E3987199729A41F8220000220121484655
S21401777005F084FC0021484605F08FFC012210210B
S214017780484605F046FC01208DF830001020709028
S214017790D4F838016F906F98709950F8210030F046
S2140177A040009DF83010890111F040010843E29035
S2140177B0E2986F99709A41F8220001208DF82F0007
S2140177C010206E90D4F838016D906D986E9950F82F
S2140177D0210030F020009DF82F10490111F0200102
S2140177E00843E190E1986D996E9A41F822000122D2
S2140177F01021484605F042FC00220321380005F01E
S21401780008FC01208DF82E0003206C90D4F830017E
S2140178106B906B986C9950F8210030F004009DF83D
S2140178202E10890011F004010843E090E0986B994E
S2140178306C9A41F8220001208DF82D0003206A90F1
S214017840D4F83001699069986A9950F8210030F0AF
S21401785020009DF82D10490111F020010843DF900A
S214017860DF9869996A9A41F82200002203213800BC
S21401787005F004FC0021380005F00FFC012202216E
S214017880380005F0C6FB01208DF82C000220689018
S214017890D4F8300167906798689950F8210030F065
S2140178A040009DF82C10890111F040010843DE903C
S2140178B0DE986799689A41F8220001208DF82B001E
S2140178C002206690D4F8300165906598669950F864
S2140178D0210030F020009DF82B10490111F0200105
S2140178E00843DD90DD986599669A41F822000122E9
S2140178F00921484605F08DFB01208DF82A00092054
S2140179006490D4F8380163906398649950F8210024
S21401791030F040009DF82A10890111F0400108431B
S214017920DC90DC986399649A41F8220001208DF876
S214017930290009206290D4F8380161906198629913
S21401794050F8210030F020009DF82910490111F06F
S21401795020010843DB90DB986199629A41F8220086
S21401796001220921484605F089FB012208214846E3
S21401797005F04FFB01208DF8280008206090D4F810
S21401798038015F905F98609950F8210030F0400010
S2140179909DF82810890111F040010843DA90DA9821
S2140179A05F99609A41F8220001208DF8270008208F
S2140179B05E90D4F838015D905D985E9950F821008C
S2140179C030F020009DF82710490111F020010843EE
S2140179D0D990D9985D995E9A41F8220014F5947869
S2140179E000220721404605F014FB01208DF82600F1
S2140179F007205C90D4F828015B905B985C9950F85E
S214017A00210030F004009DF82610890011F00401D1
S214017A100843D890D8985B995C9A41F822000120D7
S214017A208DF8250007205A90D4F8280159905998C6
S214017A305A9950F8210030F020009DF82510490190
S214017A4011F020010843D790D79859995A9A41F8CE
S214017A50220000220721404605F010FB0021404687
S214017A6005F01BFB01220621404605F0D2FA012053
S214017A708DF8240006205890D4F82801579057987E
S214017A80589950F8210030F040009DF824108901E3
S214017A9011F040010843D690D6985799589A41F864
S214017AA0220001208DF8230006205690D4F82801E4
S214017AB055905598569950F8210030F020009DF8C1
S214017AC02310490111F020010843D590D598559906
S214017AD0569A41F8220001220721280005F099FA5A
S214017AE000220721280005F0C9FA01208DF822009E
S214017AF007205490D4F8480153905398549950F85D
S214017B00210030F020009DF82210490111F02001DB
S214017B100843D490D4985399549A41F822000022ED
S214017B200C21380005F075FA01208DF821000C2093
S214017B305290D4F8300151905198529950F8210042
S214017B4030F004009DF82110890011F0040108436B
S214017B50D390D3985199529A41F8220001208DF87A
S214017B6020000C205090D4F830014F904F98509937
S214017B7050F8210030F020009DF82010490111F046
S214017B8020010843D290D2984F99509A41F822008A
S214017B9000220C21380005F071FA0021380005F0AA
S214017BA07CFA01220421300005F033FA01208DF819
S214017BB01F0004204E90D4F840014D904D984E99E8
S214017BC050F8210030F040009DF81F10890111F097
S214017BD040010843D190D1984D994E9A41F8220020
S214017BE001208DF81E0004204C90D4F840014B90E3
S214017BF04B984C9950F8210030F020009DF81E104B
S214017C00490111F020010843D090D0984B994C9A25
S214017C1041F8220001220321300005F0FAF9012083
S214017C208DF81D0003204A90D4F8400149904998E8
S214017C304A9950F8210030F040009DF81D10890146
S214017C4011F040010843CF90CF9849994A9A41F8DC
S214017C50220001208DF81C0003204890D4F8400132
S214017C6047904798489950F8210030F020009DF839
S214017C701C10490111F020010843CE90CE98479977
S214017C80489A41F8220000220221300005F0C1F98D
S214017C9001208DF81B0002204690D4F84001459043
S214017CA04598469950F8210030F004009DF81B10C5
S214017CB0890011F004010843CD90CD984599469A64
S214017CC041F8220001208DF81A0002204490D4F8D1
S214017CD0400143904398449950F8210030F0200029
S214017CE09DF81A10490111F020010843CC90CC9858
S214017CF04399449A41F8220000220221300005F0FF
S214017D00BDF90021300005F0C8F9012203214046E3
S214017D1005F07FF901208DF8190003204290D4F870
S214017D20280141904198429950F8210030F04000D6
S214017D309DF81910890111F040010843CB90CB98AA
S214017D404199429A41F8220001208DF8180003203B
S214017D504090D4F828013F903F98409950F8210070
S214017D6030F020009DF81810490111F02001084359
S214017D70CA90CA983F99409A41F8220001220321ED
S214017D80404605F07BF905220221404605F041F9FF
S214017D9000220121404605F03CF901208DF817002C
S214017DA001203E90D4F828013D903D983E9950F828
S214017DB0210030F004009DF81710890011F004012D
S214017DC00843C990C9983D993E9A41F8220001207E
S214017DD08DF8160001203C90D4F828013B903B9882
S214017DE03C9950F8210030F020009DF8161049010A
S214017DF011F020010843C890C8983B993C9A41F875
S214017E00220000220121404605F038F900214046B3
S214017E1005F043F900220021404605F0FAF801205A
S214017E208DF8150000203A90D4F828013990399839
S214017E303A9950F8210030F004009DF81510890099
S214017E4011F004010843C790C79839993A9A41F846
S214017E50220001208DF8140000203890D4F8280163
S214017E6037903798389950F8210030F020009DF867
S214017E701410490111F020010843C690C69837999D
S214017E80389A41F8220000220021404605F0F6F813
S214017E900021404605F001F900220721484605F079
S214017EA0B8F801208DF8130007203690D4F8380171
S214017EB035903598369950F8210030F004009DF839
S214017EC01310890011F004010843C590C59835992F
S214017ED0369A41F8220001208DF8120007203490CE
S214017EE0D4F8380133903398349950F8210030F0A3
S214017EF020009DF81210490111F020010843C4909A
S214017F00C4983399349A41F8220000220721484642
S214017F1005F0B4F80021484605F0BFF80122062115
S214017F20484605F076F801208DF8110006203290BB
S214017F30D4F8380131903198329950F8210030F058
S214017F4040009DF81110890111F040010843C390CB
S214017F50C3983199329A41F8220001208DF8100019
S214017F6006203090D4F838012F902F98309950F889
S214017F70210030F020009DF81010490111F0200179
S214017F800843C290C2982F99309A41F822000122E4
S214017F900621484605F072F801220621280005F060
S214017FA038F801208DF80F0006202E90D4F84801ED
S214017FB02D902D982E9950F8210030F040009DF814
S214017FC00F10890111F040010843C190C1982D9905
S214017FD02E9A41F8220001208DF80E0006202C90E2
S214017FE0D4F848012B902B982C9950F8210030F0AA
S214017FF020009DF80E10490111F020010843C090A1
S214018000C0982B992C9A41F82200012206212800BB
S21401801005F034F801220221280004F0FAFF0120BD
S2140180208DF80D0002202A90D4F84801299029984D
S2140180302A9950F8210030F040009DF80D10890172
S21401804011F040010843BF90BF9829992A9A41F838
S214018050220001208DF80C0002202890D4F8480157
S21401806027902798289950F8210030F020009DF895
S2140180700C10490111F020010843BE90BE982799C3
S214018080289A41F8220001220221280004F0F6FF76
S21401809001220D21404604F0BCFF01208DF80B00A3
S2140180A00D202690D4F8280125902598269950F879
S2140180B0210030F040009DF80B10890111F04001BD
S2140180C00843BD90BD982599269A41F822000120C3
S2140180D08DF80A000D202490D4F8280123902398C7
S2140180E0249950F8210030F020009DF80A1049012B
S2140180F011F020010843BC90BC982399249A41F8BA
S214018100220001220C21404604F0B8FF01220C2176
S214018110404604F07EFF01208DF809000C202290D5
S214018120D4F8280121902198229950F8210030F0A6
S21401813040009DF80910890111F040010843BB90E9
S214018140BB982199229A41F8220001208DF8080057
S2140181500C202090D4F828011F901F98209950F8E1
S214018160210030F020009DF80810490111F020018F
S2140181700843BA90BA981F99209A41F82200012222
S2140181800C21404604F07AFF01220B21404604F000
S21401819040FF01208DF807000B201E90D4F828011F
S2140181A01D901D981E9950F8210030F040009DF852
S2140181B00710890111F040010843B990B9981D993B
S2140181C01E9A41F8220001208DF806000B201C9013
S2140181D0D4F828011B901B981C9950F8210030F008
S2140181E020009DF80610490111F020010843B890BF
S2140181F0B8981B991C9A41F8220001220A21404690
S21401820004F007FF01208DF805000A26D4F828019E
S2140182101A901A9850F8260030F040009DF8051084
S214018220890111F040010843B790B7981A9941F8AF
S214018230260001208DF804000A27D4F82801199099
S214018240199850F8270030F020009DF804104901D5
S21401825011F020010843B690B698199941F8270005
S21401826001220A21404604F009FF012201212800CB
S21401827004F0CFFE01208DF803005FF00108D4F86A
S21401828048011890189850F8280030F040009DF8E2
S2140182900310890111F040010843B590B59818996B
S2140182A041F8280001208DF802005FF00109D4F89A
S2140182B048011790179850F8290030F020009DF8D3
S2140182C00210490111F020010843B490B49817999F
S2140182D041F8290001220121280004F0CFFE0122E5
S2140182E00021280004F095FE01208DF801005FF0C2
S2140182F0000AD4F848011690169850F82A0030F073
S21401830040009DF80110890111F040010843B39027
S214018310B398169941F82A0001208DF800005FF005
S214018320000BD4F848011590159850F82B0030F042
S21401833020009DF80010490111F020010843B29079
S214018340B298159941F82B0001220021280004F06B
S21401835095FE01220521280004F05BFE012005217F
S214018360D4F8482152F8213033F040030500EDB22D
S214018370AD0115F040052B43B193B19B42F8213076
S21401838001250523D4F8484154F823C03CF0200CBD
S214018390AE465FFA8EFE5FEA4E1E1EF0200E5EEAC5
S2140183A00C0C44F823C00DF5806D03B0BDE8F08FCA
S2140183B070B504000D002000C0B200280AD00228C3
S2140183C056D02FD3042800F0A58077D3052800F0D7
S2140183D0CD80F6E02800C0B2002803D002280CD0D9
S2140183E016D31EE0DFF8DC620021300004F06DFEDB
S2140183F00121300004F069FE13E0DFF8C8620021B5
S214018400300004F05DFE0121300004F05EFE08E05D
S214018410AC4E0121300004F053FE0021300004F080
S21401842054FECEE02800C0B2002803D0022815D0A2
S2140184300AD31CE0A44E0A21300004F046FE0B21AC
S214018440300004F042FE12E09F4E0A21300004F094
S21401845037FE0B21300004F038FE08E09A4E0B215F
S214018460300004F02DFE0A21300004F02EFEA8E0B4
S2140184702800C0B2002803D0022815D00AD31CE079
S214018480914E0421300004F020FE0521300004F056
S2140184901CFE12E08C4E0421300004F011FE052172
S2140184A0300004F012FE08E0874E0521300004F08B
S2140184B007FE0421300004F008FE82E02800C0B266
S2140184C0002803D0022819D00CD322E07F4E0321C6
S2140184D016F5A47004F0F9FD102116F5A07004F04D
S2140184E0F4FD16E0794E032116F5A47004F0E8FDBC
S2140184F0102116F5A07004F0E8FD0AE0734E102175
S21401850016F5A07004F0DCFD032116F5A47004F046
S214018510DCFD56E02800C0B2002803D0022819D09E
S2140185200CD322E0694E092116F5A47004F0CDFDA6
S2140185300F2116F5A07004F0C8FD16E0634E092160
S21401854016F5A47004F0BCFD0F2116F5A07004F01A
S214018550BCFD0AE05D4E0F2116F5A07004F0B0FDDB
S214018560092116F5A47004F0B0FD2AE02800C0B277
S214018570002803D0022819D00CD322E0534E08213C
S21401858016F5A47004F0A1FD052116F5987004F007
S2140185909CFD16E04D4E082116F5A47004F090FDE2
S2140185A0052116F5987004F090FD0AE0474E082163
S2140185B016F5A47004F084FD052116F5987004F0F4
S2140185C084FD70BD10B504002000C0B2002804D0A0
S2140185D009213F4804F074FD03E009213C4804F0FA
S2140185E074FD10BD020000201100C9B20A2905DA87
S2140185F038491300DBB251F82310080040F6E44175
S2140186004843000B704738B5040000252000C0B26F
S214018610002805D002280FD008D3032812D017E06F
S2140186200B212D4804F056FD050011E004212548D4
S21401863004F050FD05000BE00521254804F04AFD35
S214018640050005E00721204804F044FD0500FFE78A
S2140186502800C0B232BD38B504002000C0B20028E0
S2140186600BD01A4D102115F59C7004F029FD04213C
S21401867015F5987004F024FD0AE0144D102115F547
S2140186809C7004F022FD042115F5987004F01DFD80
S21401869031BD70B5040000252000C0B2652801DB9D
S2140186A0642004000D4801682000C0B241436420E4
S2140186B0B1FBF0F6330000220021094803F086FCE6
S2140186C070BD00000033002008330020C0310020B8
S2140186D0F8320020402F0020E8320020E830002049
S2140186E01C330020016070472DE9F04F91B0040063
S2140186F00D0020680068C0F3C0108DF807002068E0
S2140187000068C0F340108DF8090020680068400A30
S21401871010F001008DF808009DF80700002840F0D1
S21401872014819DF80900012840F00F819DF808008A
S214018730012840F00A811822002103A804F0DAFC7F
S2140187400399DFF89C0201400391297803AA106877
S21401875030F4E0200B00DBB21B0413F4E0231843D3
S21401876010901098106068788DF8060003AB1868B2
S21401877030F400409DF80660F60316F400463043D8
S2140187800F900F981860E8788DF8050003AE3068F2
S21401879030F480509DF805703F0317F48057384336
S2140187A00E900E98306068798DF8040003AF386833
S2140187B030F040009DF804C05FEA8C1C1CF0400CB1
S2140187C05CEA00000D900D983860A8798DF80300DA
S2140187D00DF10C0EDEF8000030F020009DF803C00D
S2140187E05FEA4C1C1CF0200C5CEA00000C900C9814
S2140187F0CEF80000E8798DF802000DF10C08D8F8E3
S214018800000030F002009DF802C05FEA4C0C1CF03C
S214018810020C5CEA00000B900B98C8F80000287A5E
S2140188208DF801000DF10C09D9F800004008400050
S2140188309DF801C01CF0010C5CEA00000A900A9841
S214018840C9F80000A878ADF80A000DF10C0ADAF8AC
S214018850000030F48040BDF80AC05FEA8C3C1CF48E
S214018860804C5CEA000009900998CAF80000DAF822
S214018870000028798DF800000DF10C0CDCF800B032
S2140188803BF0800B9DF80000C00110F0800050EA1C
S2140188900B0BCCF800B0287D002806D003A8416950
S2140188A031F0080151F008014161687D03AA53695E
S2140188B033F004030100C9B2890011F004010B432F
S2140188C05361AE7D03AFD7F814C05FEA9C0C5FEA34
S2140188D08C0C3100C9B211F0030151EA0C0CC7F837
S2140188E014C04049D4F800E0CEF80410DDF80CE0DE
S2140188F0D4F80080C8F800E0D5F810E0D4F800807D
S214018900C8F808E020680068800A10F00100C0B2CC
S2140189100028F7D020680068400A10F00100C0B2B5
S2140189200028F7D0687800280FD02F4822685060BA
S21401893023685960E9682368D96020680068400A9E
S21401894010F00100C0B20028F7D011B0BDE8F08FDA
S2140189500121017000214170012181700021C17047
S2140189600021017100214171012181710021C17134
S214018970002101724FF6FF7101610021C1600021E3
S21401898081750121017500214175704701680968EB
S214018990C1F340110A00D2B2012A1CD1114A036860
S2140189A05A600268126832F0800203681A604FF655
S2140189B0FF7203689A6002681268D20A12F0010216
S2140189C0D2B2002AF7D102681268520A12F00102E6
S2140189D0D2B2002AF7D07047034902685160704747
S2140189E09C6FF8FF20C528D902A680B470B5040094
S2140189F00D00A6686068711C884206D320688555FC
S214018A00701CA060E068401CE060A0686168884255
S214018A100DD1A2682168206904F083FCA168884210
S214018A2003D05FF0FF30E06001E00020A06070BD81
S214018A302DE9FE4F0700884691461E000C9CC24653
S214018A4001255FF0010BCA4504D3BAFBF9FA1BF105
S214018A50010BF8E7B34500D2B3460D98C0071AD408
S214018A60002C18D00D98800705D5002E03D1302094
S214018A708DF8000002E020208DF80000002C0AD0BE
S214018A80A34508D2641E9DF800103800FFF7AEFF1C
S214018A90F8680028F2D5F868002830D4022E01D3F1
S214018AA0761E05E0B8FBF5F001900198484502D323
S214018AB009FB05F5F2E7B8FBF5F00190019805FB17
S214018AC0108810480199415C3800FFF78FFFF8685D
S214018AD0002803D4B5FBF9F5002DECD10D98C0079D
S214018AE00DD5002C0BD0002C09D0A34507D2641E4F
S214018AF020213800FFF77AFFF8680028F3D5BDE893
S214018B00F78F0000DC8102002DE9FE4F06000F0002
S214018B1090461D000C9CDDF83490002F02D5D7F14D
S214018B20000A00E0BA465FF0010BC24504DB9AFB7F
S214018B30F8FA1BF1010BF8E7AB4500D2AB46002C67
S214018B4005D0002F02D45FEA497000D5641E5FEAA3
S214018B50897001D5002D10D05FEAC9700DD4002CA4
S214018B600BD0002C09D0A34507D2641E202130006B
S214018B70FFF73CFFF0680028F3D5F068002831D4F1
S214018B80002F05D57F422D213000FFF72FFF06E08D
S214018B905FEA497003D52B213000FFF727FFF06805
S214018BA000281FD419F0030002280FD1002D0DD183
S214018BB0002C0BD0002C09D0A34507D2641E30210F
S214018BC03000FFF713FFF0680028F3D5F06800289F
S214018BD008D4CDF8049000942B00424639003000AA
S214018BE0FFF726FFBDE8F78F2DE9F14F98B08946CC
S214018BF0150007A8029040200390002004901898C2
S214018C0006900020059099F80000060019F1010968
S214018C103000C0B2002800F00F813000C0B2252815
S214018C2040F00181002080460120040099F80000F0
S214018C3006003000C0B2232815D02B280ED02D28D0
S214018C4002D0302805D013E058F0010819F10109C7
S214018C5010E058F0020819F101090BE058F0040879
S214018C6019F1010906E058F0080819F1010901E0B7
S214018C7000200400002CD9D10020824699F800007B
S214018C8006003000C0B2302803DB3000C0B23A28FC
S214018C9008DB0020070099F800100800C0B22E2853
S214018CA020D109E019F101090A2000FB0AFA5AFA53
S214018CB086FABAF1300AE1E719F1010999F80000DC
S214018CC001000800C0B2302803DB0800C0B23A2811
S214018CD000DB07E019F101090A20474357FA81F73B
S214018CE0303FEBE799F800603000C0B26C2803D043
S214018CF03000C0B2682805D119F1010999F80000C1
S214018D000600F1E73000C0B2252800F0848058281C
S214018D1041D063280AD0642817D0702868D07328F9
S214018D204CD0752824D0782835D079E0286828607A
S214018D30286800682968091D29600400A346594669
S214018D40C9B202A8FFF752FE6AE0286828602868C0
S214018D5000682968091D29600400CDF80480CDF853
S214018D6000A03B000A22210002A8FFF7CDFE57E033
S214018D7028682860286800682968091D2960040099
S214018D80CDF80480CDF800A03B000A22210002A8FD
S214018D90FFF74EFE44E028682860286800682968C6
S214018DA0091D29600400CDF80480CDF800A03B0021
S214018DB01022210002A8FFF73BFE31E02868286058
S214018DC02868D0F800B02868001D28609BF80000CD
S214018DD006001BF1010B3000C0B2002807D031009D
S214018DE0C9B202A8FFF702FE05980028EED517E0E3
S214018DF028682860286800682968091D2960040019
S214018E00002001900820009008231022210002A8CB
S214018E10FFF70EFE04E0252102A8FFF7E7FDFFE7B6
S214018E2019F1010904E03100C9B202A8FFF7DEFD1D
S214018E30059800287FF5E7AE059801280BDB049816
S214018E40002804D0049A07A9189804F06AFA05992C
S214018E50049841180591059819B0BDE8F08F0CB437
S214018E6038B504000D0004A800906A4629002000C9
S214018E70FFF7BAFE32BC5DF80CFBFEE72DE9F047C2
S214018E8098B004005FF000085FF000095FF0000A88
S214018E900025002600274022002108A804F02AF910
S214018EA06846DFF8A016202204F074FA082140F282
S214018EB00112002003008C46DBB25FFA8CFC63458E
S214018EC014D25FF0FF330DF1200C86465FFA8EFE5A
S214018ED04CF83E3000230DF1200C86465FFA8EFEDC
S214018EE00CEBCE0CACF80430401CE3E70023180072
S214018EF08C46C0B25FFA8CFC604553D20220060055
S214018F00300080B2824247D32068EC469E465FFA24
S214018F108EFE5CF82EC0B0FBFCF0B4461FFA8CFC4B
S214018F20B0FBFCF005006068854218D108A89C4695
S214018F305FFA8CFC00EBCC00868008A89C465FFAA2
S214018F408CFC00EBCC00837100200DF1200C9E46BA
S214018F505FFA8EFE4CF83E00012007001CE06068B8
S214018F60854217D208A89C465FFA8CFC00EBCC0021
S214018F70868008A89C465FFA8CFC00EBCC008371C7
S214018F806068401B0DF1200C9E465FFA8EFE4CF881
S214018F903E0001E0761CB3E73800C0B2002801D1DC
S214018FA05B1CA4E75FF0000C08A8E6465FFA8EFE9D
S214018FB050F83EE05FF0010843468946DBB25FFAAF
S214018FC089F94B450ED24346DBB250F83330734530
S214018FD005D24346DBB250F833309E46C44618F1FC
S214018FE00108E9E708ABE1465FFA89F903EBC90333
S214018FF09B88022B15DA20686B4689465FFA89F949
S21401900003EB890353F8043CB0FBF3F0B0FBF2F03A
S21401901005000800C0B2401EA060901EE0602561F9
S21401902018E008ABE1465FFA89F903EBC9039B79BF
S214019030A36008ABE1465FFA89F903EBC9039B8895
S2140190409B1EE3606368E1465FFA89F950F83900D0
S2140190501B1A236118B0BDE8F0872DE9F04F87B0E1
S21401906004000D00002000905FF000085FF000098A
S2140190702000006E00900021684600F0D4FC00211C
S214019080684600F0C3FC697B684600F08FFC697A8D
S214019090684600F06AFCA97A684600F05DFC6868DC
S2140190A003902868029002A8FFF7E8FE049E059F39
S2140190B0BA46A346DBF84010090A09025046C0B278
S2140190C0014301910198CBF840003100C9B26846CE
S2140190D000F056FCE889411E89B2684600F0BBFCE8
S2140190E0A87B800604D5E97E684600F06AFC03E0AA
S2140190F00021684600F065FCE97A684600F04BFC02
S214019100687D002805D0022829D010D303283ED038
S2140191104BE00021684600F093FCE97F684600F0CA
S21401912075FC95F82010684600F07DFC4AE00121A8
S214019130684600F06BFC0021684600F074FC287C51
S214019140002804D10021684600F07AFC06E0287C5D
S214019150012803D10121684600F072FC32E0287C28
S214019160002804D10021684600F06AFC06E0287C4D
S214019170012803D10121684600F062FC01216846FE
S21401918000F044FC0021684600F04DFC1AE0002186
S214019190684600F055FCE97F684600F037FC95F814
S2140191A02010684600F03FFC0CE00021684600F005
S2140191B047FCE97F684600F029FC95F820106846D0
S2140191C000F031FC0098206607B0BDE8F08FF0B4DF
S2140191D00D7A03005C6A2A00D2B2012A03D154F048
S2140191E001025A6202E0620852005A620E7B91F94D
S2140191F00B2096400200576A37F47067B4465FFA50
S2140192008CFC5FEA0C2C1CF4706C5CEA0707576256
S214019210F0BC70472DE9FF4F030092F800C01E0016
S214019220F7696046C0B2012803D157F00100F0612A
S21401923002E078084000F06150781C00E569864637
S2140192405FFA8EFEBEF1010F03D155F00206E6610C
S21401925002E035F00206E66196781F00D7F824C0D2
S214019260B6465FFA8EFEBEF1010F03D15CF0080030
S214019270786202E03CF008007862D0781C00256A2B
S21401928086465FFA8EFEBEF1010F03D155F4807655
S214019290266202E035F4807626621F000026D7F8A3
S2140192A024C05FEACC7C01D501200600F6B2002E70
S2140192B00DD155791800446A2E00F6B2012E03D15D
S2140192C054F00406466202E034F004064662D7799A
S2140192D01D002E693800C0B2012803D156F00400E3
S2140192E0286102E036F00400286190798DF80100CB
S2140192F0180004699DF801C0BCF1010F03D154F0B8
S2140193000805056102E034F0080505614D788DF821
S21401931000500193019D2D6C35F47F459DF800604A
S21401932055EA06250395039D019E35648D781E003A
S214019330376C37F47F07AC465FFA8CFC57EA0C476C
S2140193400297029F3764CF789C46DCF840E02EF007
S2140193507F4EB8465FFA88F85EEA086ECCF840E0C1
S21401936091F804809946D9F824A03AF0700AC346C9
S2140193705FFA8BFB5FEA0B1B1BF0700B5BEA0A0ABA
S214019380C9F824A091F805B0BBF1000F07D0BBF1D6
S214019390020F3ED028D3BBF1030F4FD073E088797C
S2140193A0002801D0012000E000201C00656A0600AC
S2140193B0F6B2002E03D055F08066666202E035F004
S2140193C08066666200261F00D7F824C03CF0407C09
S2140193D0B6465FFA8EFE5FEA0E6E1EF0407E5EEACD
S2140193E00C0CC7F824C072E001201C00656A35F039
S2140193F040750600F6B2360616F0407635436562CD
S21401940001261F00D7F824C05CF0806EC7F824E060
S2140194105DE002201C00656A35F040750600F6B274
S214019420360616F040763543656201261F00D7F8EA
S21401943024C05CF0806EC7F824E048E088790028F4
S21401944001D0012000E000201C00656A0600F6B28B
S214019450002E03D055F08066666202E035F0806625
S214019460666203261F00D7F824C03CF0407CB6464F
S2140194705FFA8EFE5FEA0E6E1EF0407E5EEA0C0C10
S214019480C7F824C023E08879002801D0012000E035
S21401949000201C00656A0600F6B2002E03D055F0C7
S2140194A08066666202E035F08066666200261F000E
S2140194B0D7F824C03CF0407CB6465FFA8EFE5FEAE1
S2140194C00E6E1EF0407E5EEA0C0CC7F824C0BDE8A6
S2140194D0FF8FDFF884130160DFF8801341600121FC
S2140194E0017200214172002181720021C1720021A6
S2140194F00173012141730821C1810021C175002139
S214019500017600214176002181760021C176002175
S2140195100177002141770021C177002180F82010D2
S21401952000218177022101740A2141740A21817484
S2140195300A21C17400210175002141750021817540
S21401954070470000DC8002002DE9F84F84B004006B
S2140195500D000026276838690390039840084000EC
S2140195603861D4F80080D8F810000290029850F4C0
S2140195708070C8F81000D4F80090D9F81000019057
S214019580019850F40070C9F8100000BF00BF00BF7A
S21401959029002068FFF71BFE15F1170215F11001CF
S2140195A02068FFF737FE5FF0010AD4F800B0DBF859
S2140195B010000090009850F00100CBF81000290030
S2140195C02068FFF74AFD05B0BDE8F08F2DE9F041B0
S2140195D001600268136953F4807414610468256994
S2140195E055F40076266101260768D7F810C05CF0AE
S2140195F0020EC7F810E000BF00BF00BF5FF0000E0C
S214019600D0F80080C8F810E0BDE8F08170B403001F
S214019610002000220C00012C14D0022C1AD0B4F524
S214019620807F1FD0B4F5007F25D0B4F5806F2BD096
S214019630B4F5006F31D0B4F5805F37D0B4F1807FD8
S2140196403DD045E01C680025666916F00106F6B2B5
S21401965032003DE01C6800256669C6F34006F6B296
S214019660320035E01C6800256669360A16F00106E8
S214019670F6B232002CE01C6800256669760A16F000
S2140196800106F6B2320023E01C6800256669B60AB8
S21401969016F00106F6B232001AE01C68002566696B
S2140196A0F60A16F00106F6B2320011E01C68002533
S2140196B06669360B16F00106F6B2320008E01C6841
S2140196C000256669360E16F00106F6B23200FFE78F
S2140196D0002A01D001242000C0B270BC70472DE9D9
S2140196E0FE4F04000D0016001F00DDF830805FF00D
S2140196F00109002021680022CB6D13F01F03D3F16E
S21401970010038DF8043033009DF804C09BB21FFA95
S2140197108CFC634580F09980002000905FF0000B80
S2140197200020ADF806002068006E00900021684613
S21401973000F061F90121684600F050F90021684601
S21401974000F071F90021684600F060F92900C9B2FD
S214019750C900491E89B2684600F07DF90098216863
S21401976008665FF0000A5046310080B289B288422E
S2140197705FD220680021426912F00102D2B2002AAB
S21401978007D11BF1010B40F2E9308345F1D30020EC
S21401979081462800C0B2012805D1504680B2385C07
S2140197A02168486610E02800C0B2022806D150465B
S2140197B080B237F810002168486605E0504680B24E
S2140197C057F8200021684866002083462268002159
S2140197D0106FC0F34000002801D001200100C9B27B
S2140197E0002907D01BF1010B40F2E9308345EDD388
S2140197F0002081462800C0B2012806D12068406FAB
S214019800514689B208F8010010E02800C0B20228CB
S21401981006D12068406F514689B228F8110005E04C
S2140198202068406F514689B248F821001AF1010AB2
S21401983099E70021684600F0DEF80021684600F04E
S214019840CDF800982168086601E000208146484668
S214019850C0B2BDE8FE8F0000000E270740420F0091
S21401986070B4020000200B00012B11D0022B1AD07D
S214019870B3F5807F22D0B3F5007F2BD0B3F5806F90
S21401988034D0B3F5006F3DD0B3F5805F46D051E0DC
S214019890012415680023AE692640A64201D101269F
S2140198A03300180046E0022415680023AE692640FE
S2140198B0A64201D10126330018003BE04FF4807424
S2140198C015680023AE692640A64201D10126330061
S2140198D018002FE04FF4007415680023AE69264087
S2140198E0A64201D101263300180023E04FF480641C
S2140198F015680023AE692640A64201D10126330031
S214019900180017E04FF4006415680023AE6926407E
S214019910A64201D10126330018000BE04FF4805413
S21401992015680023AE692640A64201D10126330000
S2140199301800FFE7C0B270BC704730B40A00036875
S2140199409C6D34F4F8141500EDB22D0415F4F815D9
S2140199502C439C6530BC7047026822F000420B0025
S214019960DBB252EAC37202607047026832F080428C
S2140199700B00DBB29B0713F080431A43026070476B
S214019980026832F060520B00DBB2DB0613F0605364
S2140199901A4302607047026832F040720B00DBB275
S2140199A01B0613F040731A4302607047026832F4D4
S2140199B000020B00DBB2DB0513F400031A4302605E
S2140199C0704702680B00DBB2012B03D152F480030F
S2140199D0036002E032F480030360704702680B0004
S2140199E0DBB2012B03D152F40013036002E032F420
S2140199F0001303607047026832F480120B00DBB27A
S214019A001B0513F480131A430260704702680B00AB
S214019A10DBB2012B03D152F40023036002E032F4DF
S214019A2000230360704702680B00DBB2012B03D1F1
S214019A3052F48023036002E032F48023036070470F
S214019A40026832F440320B00DBB21B0413F44033DD
S214019A501A43026070470268120B12030B009BB296
S214019A601B051B0D1A4302607047FEE70068C00F16
S214019A70C0B27047026822F000420B00DBB252EA25
S214019A80C37202607047026832F0FE420B00DBB21E
S214019A901B0613F0FE431A4302607047026832F455
S214019AA0FE020B00DBB21B0413F4FE031A43026032
S214019AB07047026832F4FE420B00DBB21B0213F45D
S214019AC0FE431A43026070470268D209D2010B00B6
S214019AD0DBB213F07F031A43026070474068C00F81
S214019AE0C0B27047426822F000420B00DBB252EA75
S214019AF0C37242607047426832F0FE420B00DBB22E
S214019B001B0613F0FE431A4342607047426832F464
S214019B10FE020B00DBB21B0413F4FE031A43426081
S214019B207047426832F4FE420B00DBB21B0213F4AC
S214019B30FE431A43426070474268D209D2010B00C5
S214019B40DBB213F07F031A43426070478068C00F90
S214019B50C0B27047826822F000420B00DBB252EAC4
S214019B60C37282607047826832F0FE420B00DBB23D
S214019B701B0613F0FE431A4382607047826832F474
S214019B80FE020B00DBB21B0413F4FE031A438260D1
S214019B907047826832F4FE420B00DBB21B0213F4FC
S214019BA0FE431A43826070478268D209D2010B00D5
S214019BB0DBB213F07F031A4382607047C068C00FA0
S214019BC0C0B27047C26822F000420B00DBB252EA14
S214019BD0C372C2607047C26832F0FE420B00DBB24D
S214019BE01B0613F0FE431A43C2607047C26832F484
S214019BF0FE020B00DBB21B0413F4FE031A43C26021
S214019C007047C26832F4FE420B00DBB21B0213F44B
S214019C10FE431A43C2607047C268D209D2010B00E4
S214019C20DBB213F07F031A43C26070470069C00FAE
S214019C30C0B27047026922F000420B00DBB252EA62
S214019C40C37202617047026932F0FE420B00DBB25A
S214019C501B0613F0FE431A4302617047026932F491
S214019C60FE020B00DBB21B0413F4FE031A4302616F
S214019C707047026932F4FE420B00DBB21B0213F49A
S214019C80FE431A43026170470269D209D2010B00F2
S214019C90DBB213F07F031A43026170474069C00FBD
S214019CA0C0B27047426922F000420B00DBB252EAB2
S214019CB0C372426170474269D209D2010B00DBB21E
S214019CC013F07F031A43426170478069C00FC0B228
S214019CD07047826922F000420B00DBB252EAC3727F
S214019CE082617047826932F0FE420B00DBB21B06CE
S214019CF013F0FE431A4382617047826932F4FE0212
S214019D000B00DBB21B0413F4FE031A438261704797
S214019D10826932F4FE420B00DBB21B0213F4FE43EF
S214019D201A43826170478269D209D2010B00DBB205
S214019D3013F07F031A4382617047C069C00FC0B237
S214019D407047C26922F000420B00DBB252EAC372CE
S214019D50C2617047C26932F0FE420B00DBB21B06DD
S214019D6013F0FE431A43C2617047C26932F4FE0221
S214019D700B00DBB21B0413F4FE031A43C2617047E7
S214019D80C26932F4FE420B00DBB21B0213F4FE433F
S214019D901A43C2617047C269D209D2010B00DBB215
S214019DA013F07F031A43C2617047006AC00FC0B246
S214019DB07047026A22F000420B00DBB252EAC3721D
S214019DC002627047026A32F0FE420B00DBB21B06EB
S214019DD013F0FE431A4302627047026A32F4FE022F
S214019DE00B00DBB21B0413F4FE031A430262704736
S214019DF0026A32F4FE420B00DBB21B0213F4FE438E
S214019E001A4302627047026AD209D2010B00DBB222
S214019E1013F07F031A4302627047406AC00FC0B254
S214019E207047426A22F000420B00DBB252EAC3726C
S214019E3042627047426A32F0FE420B00DBB21B06FA
S214019E4013F0FE431A4342627047426A32F4FE023E
S214019E500B00DBB21B0413F4FE031A434262704785
S214019E60426A32F4FE420B00DBB21B0213F4FE43DD
S214019E701A4342627047426AD209D2010B00DBB232
S214019E8013F07F031A4342627047806AC00FC0B264
S214019E907047826A22F000420B00DBB252EAC372BC
S214019EA082627047826A32F0FE420B00DBB21B060A
S214019EB013F0FE431A4382627047826A32F4FE024E
S214019EC00B00DBB21B0413F4FE031A4382627047D5
S214019ED0826A32F4FE420B00DBB21B0213F4FE432D
S214019EE01A4382627047826AD209D2010B00DBB242
S214019EF013F07F031A4382627047C06AC00FC0B274
S214019F007047C26A22F000420B00DBB252EAC3720B
S214019F10C2627047C26A32F0FE420B00DBB21B0619
S214019F2013F0FE431A43C2627047C26A32F4FE025D
S214019F300B00DBB21B0413F4FE031A43C262704724
S214019F40C26A32F4FE420B00DBB21B0213F4FE437C
S214019F501A43C2627047C26AD209D2010B00DBB251
S214019F6013F07F031A43C2627047006BC00FC0B282
S214019F707047026B22F000420B00DBB252EAC3725A
S214019F8002637047026BD209D2010B00DBB213F0F9
S214019F907F031A4302637047406BC00FC0B270471D
S214019FA0426B22F000420B00DBB252EAC3724263FC
S214019FB07047426BD209D2010B00DBB213F07F036C
S214019FC01A4342637047806BC00FC0B27047826B02
S214019FD022F000420B00DBB252EAC3728263704782
S214019FE0826B32F0FE420B00DBB21B0613F0FE431F
S214019FF01A4382637047826B32F4FE020B00DBB2B7
S21401A0001B0413F4FE031A4382637047826B32F417
S21401A010FE420B00DBB21B0213F4FE431A438263BB
S21401A0207047826BD209D2010B00DBB213F07F03BB
S21401A0301A4382637047C06BC00FC0B27047C26BD1
S21401A04022F000420B00DBB252EAC372C2637047D1
S21401A050C26BD209D2010B00DBB213F07F031A43A5
S21401A060C2637047016042607047F8B504000D0096
S21401A070002C04D0002D02D02888002800D135E01D
S21401A08000263000298880B2884212D269683200E0
S21401A09092B20320424301EB020042786968330022
S21401A0A09BB203204343C95C200000F020F8761CD5
S21401A0B0E7E700273800298880B2884216D2696807
S21401A0C03A0092B20320424301EB02008078002856
S21401A0D00AD069683A0092B20320424301EB0200BB
S21401A0E04178200000F035F87F1CE3E7F1BD2DE94B
S21401A0F0F04104000D0016003100C9B2200000F046
S21401A1003DF8012801D1002020E0B0465FFA88F82A
S21401A1105FEA980816F00307264A4046C0B20001D7
S21401A12010443900C9B250F8210000280DD029008A
S21401A130C9B220684346DBB21B011A443B00DBB2BE
S21401A14052F823209047012000E00020C0B2BDE86D
S21401A150F08170B504000D002E00F6B2B608164A5E
S21401A1603000C0B252F82000002806D00121206835
S21401A1703300DBB252F82320904770BDF8B50400D7
S21401A1800D0001262F00FFB2BF080C493800C0B2EF
S21401A19051F8200000280AD020683A00D2B251F8BF
S21401A1A022108847012801D1012600E00026300050
S21401A1B0C0B2F2BDC0780200247E0200E47D020037
S21401A1C038B4002243689C6C640864001500EDB244
S21401A1D015F001052C439C6400250095009A8A42DF
S21401A1E003D2009A521C0092F8E7012243689C6C45
S21401A1F0640864001500EDB215F001052C439C645B
S21401A20031BC7047F0B44168096831F0400131F45F
S21401A210003131F4803131F0020131F0800131F04A
S21401A22004014268116000221300DBB2102B5BD2DE
S21401A2301400436800252600F6B276011E4441F25A
S21401A2400807F55100252600F6B276011E4416F5DC
S21401A2508056356000252600F6B276011E4441F28E
S21401A2600407F55300252600F6B276011E4441F296
S21401A2700607F55300252600F6B276011E4441F284
S21401A2800C07F55100252600F6B276011E4441F270
S21401A2901007F55100252600F6B276011E4441F25C
S21401A2A01407F55301252600F6B276011E4441F245
S21401A2B01607F55300252600F6B276011E4441F234
S21401A2C01807F55100252600F6B276011E4441F224
S21401A2D01C07F55301252600F6B276011E4441F20D
S21401A2E01E07F553521C9FE7F0BC70474160826021
S21401A2F07047002101740021417400210170012181
S21401A3004170022181700321C17004210171052170
S21401A3104171062181710721C1710821017209214C
S21401A32041720A2181720B21C1720C2101730D2128
S21401A33041730E2181730F21C1737047FF21417054
S21401A340002101700021817000214160002181609F
S21401A3500021017370472DE9F04704000D00160037
S21401A36000275FF000082560D4F808905FF0000A27
S21401A3705046C0B2102807D200205146C9B209F88B
S21401A38001001AF1010AF3E74021206800F03CFEC3
S21401A3902000FFF737FF307C61680200D2B2002A46
S21401A3A004D00A6852F004020A6003E00A6832F038
S21401A3B004020A6062681268C2F38002D2B2002AFE
S21401A3C01CD100200700102F18D2F05D39006268FA
S21401A3D00B00DBB2134493F800311B091B018446C2
S21401A3E05FFA8CFC1CF00F0C5CEA03038C465FFAE8
S21401A3F08CFC94448CF800317F1CE4E7727C616825
S21401A4001000C0B2002804D0086850F010000860A0
S21401A41003E0086830F0100008604046C0B2BDE8AE
S21401A420F087F8B506000D0014000027002D09D0AE
S21401A430002C07D02200207855F82010300000F0BC
S21401A44004F800E00120C0B2F2BD2DE9F04104009D
S21401A4500D00160037785FF000081021280000F084
S21401A460D3FDB078002806D0337BB278317820004F
S21401A47000F0E0F880463800616800220300DBB295
S21401A4805B010B4441F2080C43F80C200022030048
S21401A490DBB25B010B4413F580531A600022030004
S21401A4A0DBB25B010B4441F2040C23F80C200022C2
S21401A4B00300DBB25B010B4441F2060C23F80C20CF
S21401A4C000220300DBB25B010B4441F20C0C43F8A3
S21401A4D00C2000220300DBB25B010B4441F2100C9E
S21401A4E043F80C2000220300DBB25B010B4441F26F
S21401A4F0140C23F80C2001220300DBB25B010B4491
S21401A50041F2160C23F80C2000220300DBB25B019B
S21401A5100B4441F2180C43F80C2000220300DBB276
S21401A5205B010B4441F21C0C23F80C2001220300B2
S21401A530DBB25B010B4441F21E0C23F80C204246B1
S21401A540D2B2002A40D120683900C9B240F8215061
S21401A55020683900C9B250F8210007702068390018
S21401A560C9B250F821000021017360680068C0F389
S21401A5708000C0B2002819D17078FF2816D07078F4
S21401A580390062680B00DBB2134493F800311B09F3
S21401A5901B0184465FFA8CFC1CF00F0C5CEA03037B
S21401A5A08C465FFA8CFC94448CF8003120683900A4
S21401A5B0C9B250F821007168416020683900C9B2FB
S21401A5C050F82100B16881604046C0B2BDE8F08114
S21401A5D02DE9F04104000D0016000127D4F804808F
S21401A5E0D8F8000050F08000C8F8000032002900BA
S21401A5F0C9B2200000F06EF820682900C9B250F8F0
S21401A6002100002101730020BDE8F081F0B40200B2
S21401A61001230C00556826002F005FF0000C300067
S21401A620C0B210F00F0050EA0C0C87F81BC00020D7
S21401A630F0BC70472DE9F84F04008DF80220002782
S21401A6408DF80110D4F808C05FF0010EBCF81000B8
S21401A6509DF901501EFA05F5A843ACF810009DF8C7
S21401A66002808946D4F808A04846C0B21AF800B05D
S21401A6701BF0800B18F07F0050EA0B0B4846C0B267
S21401A6800AF800B08DF800300E00A5689DF80000AD
S21401A690002808D03000C0B2285C50F08000370097
S21401A6A0FFB2E85507E03000C0B2285C10F07F002A
S21401A6B03700FFB2E85501278C46D4F80880B8F871
S21401A6C010001EFA0CFE5EEA000EA8F810E000204C
S21401A6D0BDE8F28F2DE9F04F90B003008DF8001021
S21401A6E0D3F804E041F208079DF8000040017044E9
S21401A6F00024C4514FF4805A9DF800004001704474
S21401A700002440F80A4041F204009DF8004064012C
S21401A71074440025255241F206089DF80040640164
S21401A7207444002524F8085000249DF800506D015B
S21401A730754441F20C06AC5100249DF800506D01A1
S21401A740754441F21006AC5141F214099DF80040DF
S21401A75064017444002524F8095041F216049DF85A
S21401A76000506D01754401262E5300259DF80060AA
S21401A7707601764441F2180C46F80C5041F21C055D
S21401A7809DF80060760176445FF0000C26F805C05F
S21401A79041F21E069DF800C05FEA4C1CF4445FF0CF
S21401A7A0010B2CF806B0D2F800B0CDF83CB08DF80D
S21401A7B00F10D3F804B0CDF838B0DDF838C09DF8E6
S21401A7C00FB05FEA4B1BDC44DDF83CB04CF80AB036
S21401A7D0D2F804A0CDF834A08DF80E10D3F804A05A
S21401A7E0CDF830A0DDF834C0DDF830A09DF80EB00D
S21401A7F05FEA4B1BDA4441F2100B4AF80BC092F8A1
S21401A80008A08DF80DA092F819A08DF80CA092F86A
S21401A81018A08DF80BA08DF80110D3F804A0CDF880
S21401A8201CA09DF80CA08DF80AA09DF801A08DF83B
S21401A83004A0DDF81CA0CDF828A0DDF828C09DF8FE
S21401A84004A05FEA4A1AD4443CF808A04FF6077CF5
S21401A8501CEA0A0A9DF80AC05FEACC0C1CF0F80C48
S21401A8605CEA0A0AADF818A0DDF828C09DF804A035
S21401A8705FEA4A1AD444BDF818A02CF808A09DF83F
S21401A8800BA08DF809A09DF801A08DF803A0DDF8B6
S21401A8901CA0CDF824A0DDF824C09DF803A05FEA33
S21401A8A04A1AD4443CF808A05FEA4A5A5FEA5A5A60
S21401A8B09DF809C05AEACC2AADF816A0DDF824C0E6
S21401A8C09DF803A05FEA4A1AD444BDF816A02CF8F6
S21401A8D008A09DF80DA08DF808A09DF801A08DF8A0
S21401A8E002A0DDF81CA0CDF820A0DDF820C09DF860
S21401A8F002A05FEA4A1AD4443CF808A04FF6F87C56
S21401A9001CEA0A0A9DF808C01CF0070C5CEA0A0A51
S21401A910ADF814A0DDF820C09DF802A05FEA4A1A3F
S21401A920D444BDF814A02CF808A0B2F90A80ADF8FA
S21401A93012808DF80710D3F80480CDF82C80DDF84E
S21401A9402CC09DF807805FEA4818C444BDF8128001
S21401A9502CF80080B2F90C00ADF810008DF8061046
S21401A960D3F804809DF8060040014044BDF810C0AD
S21401A97020F809C0D2F810908DF80510D3F804C05D
S21401A9809DF805004001604441F20C0A40F80A9027
S21401A99092F82000002825D001208E46D3F80480A6
S21401A9A0F4465FFA8CFC5FEA4C1CC444F1465FFA3D
S21401A9B089F95FEA4919C14439F8059059F0100937
S21401A9C02CF80590D2F824908DF80010D3F804C026
S21401A9D09DF800A05FEA4A1AE24441F2180B4AF8D1
S21401A9E00B9023E05FF0000E8846D3F804904046B3
S21401A9F0C0B2400109EB000C4046C0B240014844D9
S21401AA0030F805A04FF6EF7010EA0A0A2CF805A0F8
S21401AA1050698DF80010D3F804C09DF800A05FEAD5
S21401AA204A1AE24441F2180B4AF80B0092F82890B1
S21401AA308A46D3F804B04846C0B2002810D0504623
S21401AA40C0B240015844D4465FFA8CFC5FEA4C1C05
S21401AA50DC443CF805C05CF0020C20F805C010E0B0
S21401AA605046C0B240010BEB000C5046C0B240014C
S21401AA70584430F805E04FF6FD7010EA0E0E2CF83B
S21401AA8005E092F829C08E46D3F804806046C0B22D
S21401AA90002810D07046C0B240014044F1465FFA2B
S21401AAA089F95FEA4919C14439F8059059F4805982
S21401AAB020F8059010E07046C0B2400108EB00098E
S21401AAC07046C0B24001404430F805A04EF6FF7013
S21401AAD010EA0A0A29F805A0D06A002800F03A828E
S21401AAE0D06A90F804C08E46D3F80480D8F80000E7
S21401AAF0C0F3C010002824D06046C0B2002810D091
S21401AB007046C0B240014044F1465FFA89F95FEAF7
S21401AB104919C14459F8079059F0004940F807907F
S21401AB200FE07046C0B240014044F1465FFA89F931
S21401AB305FEA4919C14459F8079029F0004940F8DD
S21401AB400790D06A90F805908A46D3F804B0DBF8EF
S21401AB500000C0F3C010002824D04846C0B2002828
S21401AB6010D05046C0B240015844D4465FFA8CFC1F
S21401AB705FEA4C1CDC445CF807C05CF0804C40F893
S21401AB8007C00FE05046C0B240015844D4465FFAB1
S21401AB908CFC5FEA4C1CDC445CF807C03CF0804C43
S21401ABA040F807C0D06AD0F808C08E46D3F80480B3
S21401ABB0D8F80000C0F3C01000282FD05FF00009BD
S21401ABC07046C0B240014044C059C00F002801D0B1
S21401ABD0012081467046C0B240014044C059C0F3CE
S21401ABE08070002801D0012081464846C0B2002866
S21401ABF014D07046C0B240014044C0596FF39D2046
S21401AC00DFF800A41AEA8C2A5AEA0000F2465FFA34
S21401AC108AFA5FEA4A1AC2444AF80700D2F81C9038
S21401AC20CDF804908A46D3F804B0DBF80000C0F3F0
S21401AC30C01000283AD05FF0000C5046C0B2400168
S21401AC405844C059C00F002814D15046C0B2400124
S21401AC505844C059C0F3807000280BD15046C0B28A
S21401AC6040015844DDF804E02EF0404E40F807E07D
S21401AC70012084466046C0B200281FD15046C0B2AB
S21401AC8040015844C059800A8002DDF804E05FEABA
S21401AC908E5E5FEA9E5E5EEA0000D6465FFA8EFE34
S21401ACA05FEA4E1EDE444EF8070007E05046C0B28B
S21401ACB040015844DDF804C040F807C0D06A077B5D
S21401ACC0D06A407B02908C46D3F804E08DF8017080
S21401ACD0E046F1469DF80100002810D04046C0B27B
S21401ACE040014844C2465FFA8AFA5FEA4A1ACA44F1
S21401ACF03AF806A05AF4004A20F806A011E04046A9
S21401AD00C0B240014844C2465FFA8AFA5FEA4A1A6C
S21401AD10CA443AF806A05FEA4A4A5FEA5A4A20F865
S21401AD2006A08DF80070E246F3469DF80000002864
S21401AD3010D05046C0B240015844D0465FFA88F859
S21401AD405FEA4818D84438F8048058F4004820F8D8
S21401AD50048011E05046C0B240015844D0465FFA24
S21401AD6088F85FEA4818D84438F804805FEA48480B
S21401AD705FEA584820F804803800C0B2002840D066
S21401AD80DDF808808DF801C0CDF804E001989DF843
S21401AD9001905FEA4919484430F806904EF2FF10D8
S21401ADA010EA09094046C0B2400210F4F05050EAD9
S21401ADB00909ADF8029001989DF801905FEA4919DA
S21401ADC04844BDF8029020F80690DDF808908DF80A
S21401ADD000C0F2469DF800004001504430F804B02F
S21401ADE04EF2FF1010EA0B0B4846C0B2400210F4B8
S21401ADF0F05050EA0B0B9DF800004001504420F83B
S21401AE0004B0D06A90F80E808DF80380D06A90F86E
S21401AE100F80CDF80C808DF80110D3F804809DF8D2
S21401AE2003908DF802909DF80190C2469DF80200AD
S21401AE3000280CD04846C0B2400150444F46FFB2ED
S21401AE407F0157447F5B57F02007475310E0484681
S21401AE50C0B240010AEB00074846C0B24001504468
S21401AE6030F805C04FF6DF7010EA0C0C27F805C065
S21401AE70039F9DF801008DF80000CDF80880029828
S21401AE809DF800C05FEA4C1C604430F805E04FF2C4
S21401AE90FF0010EA0E0E3800C0B2000210F4706017
S21401AEA050EA0E0EADF804E002989DF800C05FEA85
S21401AEB04C1C6044BDF804C020F805C0D06A056883
S21401AEC08C46D3F804E05FF0000B6046C0B2400148
S21401AED07044805B00041ED56046C0B240017044D9
S21401AEE0875B17F47E47E805C00D07436046C0B28E
S21401AEF04001704487536046C0B240017044065B0F
S21401AF0016F47E46E805C00D06436046C0B2400111
S21401AF10704406531DE06046C0B240017044875B32
S21401AF2017F400476804400C07436046C0B240016E
S21401AF30704487536046C0B240017044005B10F411
S21401AF4000406E04760C06436046C0B24001704471
S21401AF50065342E0D4690E005D682868C0F3C0104D
S21401AF60002835D05FF0000C3000C0B24001284404
S21401AF70C059C00F002812D13000C0B24001284489
S21401AF80C059C0F38070002809D13000C0B240011A
S21401AF90284424F0404E40F807E0012084466046ED
S21401AFA0C0B2002819D13000C0B24001284450F880
S21401AFB007E05FEA9E2E5FEA8E2EA005800D50EA1E
S21401AFC00E0E3000C0B24001284440F807E004E00D
S21401AFD03000C0B240012844C45108005C68002516
S21401AFE0E66AC64016F00106F6B2002E06D00C0040
S21401AFF05D68002614F00F000643AE7710B0BDE87A
S21401B000F08F000000FCFF3F002904D000220270F0
S21401B010401C491EF8E7704710B4016042601C7876
S21401B020047210BC7047F0B4002300242200D2B290
S21401B030042A09DA2200D2B28A5C002A02D001224E
S21401B040A2401343641CF1E71A004568AE6936F066
S21401B05070661700FFB23F0617F070673E43AE6199
S21401B060F0BC70472DE9F24F83B0039909790029A6
S21401B0700DD002296FD019D3042900F01781C0F032
S21401B080BF80062900F0BE81C0F0668110E2002173
S21401B0900268136923F07F4333F020030C00E4B207
S21401B0A0640114F020042343136101E201220368C2
S21401B0B0196921F07F4131F020011400E4B26401E6
S21401B0C014F02004214302910299196100240568B5
S21401B0D0296921F07F4131F010012600F6B23601D0
S21401B0E016F010063143019101992961002607687F
S21401B0F0396921F07F4131F00801B4465FFA8CFCD2
S21401B1005FEACC0C1CF0080C5CEA01010091009986
S21401B11039610399B1F800C0D0F800E0DEF8088084
S21401B1205FEA18485FEA0848614689B251EA0808AA
S21401B130CEF808805FF00009D0F800A0DAF80CB06D
S21401B1405FEA1B4B5FEA0B4B494689B251EA0B0B90
S21401B150CAF80CB0ACE101220368196921F07F41FD
S21401B16031F020011400E4B2640114F020042143FC
S21401B17002910299196101240568296921F07F412C
S21401B18031F010012600F6B2360116F010063143F2
S21401B19001910199296100260768396921F07F41EB
S21401B1A031F00801B4465FFA8CFC5FEACC0C1CF067
S21401B1B0080C5CEA01010091009939610399B1F824
S21401B1C000C0D0F800E0DEF808805FEA18485FEAC1
S21401B1D00848614689B251EA0808CEF808805FF04F
S21401B1E00009D0F800A0DAF80CB05FEA1B4B5FEA62
S21401B1F00B4B494689B251EA0B0BCAF80CB057E122
S21401B20001220368196921F07F4131F02001140001
S21401B210E4B2640114F020042143029102991961F9
S21401B22000240568296921F07F4131F010012600CC
S21401B230F6B2360116F010063143019101992961E3
S21401B24001260768396921F07F4131F00801B446CB
S21401B2505FFA8CFC5FEACC0C1CF0080C5CEA01017E
S21401B2600091009939610399B1F800C0D0F800E067
S21401B270DEF808805FEA18485FEA0848614689B246
S21401B28051EA0808CEF808800399B1F80290D0F880
S21401B29000A0DAF80CB05FEA1B4B5FEA0B4B49469D
S21401B2A089B251EA0B0BCAF80CB001E1012203681E
S21401B2B0196921F07F4131F020011400E4B26401E4
S21401B2C014F02004214302910299196100240568B3
S21401B2D0296921F07F4131F010012600F6B23601CE
S21401B2E016F010063143019101992961012607687C
S21401B2F0396921F07F4131F00801B4465FFA8CFCD0
S21401B3005FEACC0C1CF0080C5CEA01010091009984
S21401B31039610399B1F802C0D0F800E0DEF8088080
S21401B3205FEA18485FEA0848614689B251EA0808A8
S21401B330CEF808800399B1F80090D0F800A0DAF8AA
S21401B3400CB05FEA1B4B5FEA0B4B494689B251EAE8
S21401B3500B0BCAF80CB0ABE001220368196921F0A7
S21401B3607F4131F020011400E4B2640114F020049E
S21401B370214302910299196101240568296921F086
S21401B3807F4131F010012600F6B2360116F01006A4
S21401B390314301910199296101260768396921F034
S21401B3A07F4131F00801B4465FFA8CFC5FEACC0CB1
S21401B3B01CF0080C5CEA01010091009939610399BF
S21401B3C0B1F800C0D0F800E0DEF808805FEA18485F
S21401B3D05FEA0848614689B251EA0808CEF8088053
S21401B3E00399B1F80290D0F800A0DAF80CB05FEA41
S21401B3F01B4B5FEA0B4B494689B251EA0B0BCAF865
S21401B4000CB055E001220368196921F07F4131F043
S21401B41020011400E4B2640114F0200421430291D7
S21401B4200299196101240568296921F07F4131F0EB
S21401B43010012600F6B2360116F0100631430191CE
S21401B4400199296101260768396921F07F4131F0A8
S21401B4500801B4465FFA8CFC5FEACC0C1CF0080CC1
S21401B4605CEA01010091009939610399B1F802C0C3
S21401B470D0F800E0DEF808805FEA18485FEA08487E
S21401B480614689B251EA0808CEF808800399B1F8F6
S21401B4900090D0F800A0DAF80CB05FEA1B4B5FEA28
S21401B4A00B4B494689B251EA0B0BCAF80CB0FFE7C1
S21401B4B0BDE8FF8F2DE9F04F89B004000D00012192
S21401B4C02268506930F480300B00DBB21B0413F4A1
S21401B4D0803318430890089850612B7826683068A6
S21401B4E030F48070800880001F00FFB217F0030759
S21401B4F0384307900798306068788DF8050027680C
S21401B500D7F804E05FEA1E2E5FEA0E2E9DF80500CE
S21401B51050EA0E0ECDF818E006987860A8788DF8F7
S21401B5200400D4F800E0DEF8040030F47F409DF813
S21401B53004C050EA0C2005900598CEF80400E8787F
S21401B5408DF80300D4F80080D8F8040030F47C109D
S21401B5509DF803C05FEA0C4C1CF47C1C5CEA0000FE
S21401B56004900498C8F8040028798DF80200D4F8ED
S21401B5700090D9F8100020F07F40400840009DF868
S21401B58002C01CF0010C5CEA000003908F48C9F869
S21401B59020000398C9F810000020C9F82000687937
S21401B5A08DF80100D4F800A0DAF8100020F07F40F2
S21401B5B030F004009DF801C05FEA8C0C1CF0040C0E
S21401B5C05CEA000002900298CAF8100095F8430061
S21401B5D08DF80000D4F800C0DCF810B02BF07F4BDB
S21401B5E03BF0400B9DF80000800110F0400050EA4F
S21401B5F00B0BCCF810B0207A002830D195F8440017
S21401B60061688A6932F020020300DBB25B0113F045
S21401B61020031A438A6195F845306668B76937F0A2
S21401B6201C079C465FFA8CFC5FEA8C0C1CF01C0C19
S21401B6305CEA0707B76195F846C0D4F804E0DEF87F
S21401B64018805FEA98085FEA8808E1465FFA89F998
S21401B65019F0030959EA0808CEF8188032E0207A72
S21401B66001282FD195F8440061688A6932F40052A6
S21401B6700300DBB25B0313F400531A438A6195F8A7
S21401B68045306668B76937F4E0579C465FFA8CFC2C
S21401B6905FEA8C2C1CF4E05C5CEA0707B76195F85E
S21401B6A046C0D4F804E0DEF8188038F44078E14665
S21401B6B05FFA89F95FEA092919F4407959EA080815
S21401B6C0CEF818802E7B2768D7F8148038F0080843
S21401B6D03000C0B2C00010F0080050EA0808C7F8F1
S21401B6E01480A91D2000FFF7BDFCA97B22685369C1
S21401B6F033F004030800C0B2800010F004000343D6
S21401B7005361A87B00280AD0687B21684A699208A1
S21401B71092000300DBB213F003031A434A610026CA
S21401B7203000C0B218283CDA3000C0B205EB400049
S21401B730C07B320021681300DBB201EB8303D3F830
S21401B74000315B095B010700FFB217F01F073B439F
S21401B7501700FFB201EB8707C7F800313700FFB2C9
S21401B76005EB47073F7CB646D4F800C0F0465FFAC3
S21401B77088F80CEB8808D8F8008138F04008B946FC
S21401B7805FFA89F95FEA891919F0400959EA080848
S21401B790F1465FFA89F90CEB8909C9F80081761C34
S21401B7A0BEE715F13F012000FFF73DFC00202168B0
S21401B7B04A6932F480320300DBB21B0413F480338F
S21401B7C01A434A6109B0BDE8F08F0000C3C3D2A591
S21401B7D000210122027004224270302282700B2264
S21401B7E0C27000220271002242710022C280002231
S21401B7F00281002282720022027300224273012219
S21401B800827300221100C9B2042907DA002113004D
S21401B810DBB2034483F83F10521CF3E7002180F8A3
S21401B8204310002180F84410042180F845100021BF
S21401B83080F8461000210A00D2B2182A0CDA0A0053
S21401B840D2B200EB4202D17300220B00DBB200EB56
S21401B85043031A74491CEEE7704710B400210268CE
S21401B860536933F480330C00E4B2240414F48034B6
S21401B8702343536110BC704701604260704710B4A7
S21401B88001210268136833F080030C00E4B2E4017E
S21401B89014F080042343136010BC704710B40021D9
S21401B8A00268136833F080030C00E4B2E40114F07C
S21401B8B080042343136010BC704701680A6852086D
S21401B8C0520052F001020A6070472DE9FF4F002432
S21401B8D02700FFB2032F80F2958000273D00002746
S21401B8E03E0000273B0000273A001700FFB2082F52
S21401B8F02BDA2700FFB201EBC70794465FFA8CFCF0
S21401B90017F80C70002F05D0022F08D003D3032F91
S21401B9100FD018E017E0012797403E4313E05FF091
S21401B920010C1CFA02F73E431CFA02FC5CEA050510
S21401B93009E05FF0010C1CFA02F73E431CFA02FC18
S21401B9405CEA0303FFE7521CCFE78DF801408DF850
S21401B950043007685FF0280E9DF801C00EFB0CFC52
S21401B960BC44DCF8108038F47F089DF804C058EA1F
S21401B9700C48CDF80C809DF801C00EFB0CFCBC44B5
S21401B980DDF80C80CCF810808DF800408DF803505F
S21401B990D0F800809DF800C00EFB0CFCC444DCF817
S21401B9A0109039F47F499DF803C059EA0C29CDF867
S21401B9B008909DF800C00EFB0CFCC444DDF808900E
S21401B9C0CCF81090A1468DF80260D0F800A0CC46C5
S21401B9D05FFA8CFC0EFB0CFCD444DCF810B05FEA7A
S21401B9E01B2B5FEA0B2B9DF802C05CEA0B0BCC46C7
S21401B9F05FFA8CFC0EFB0CFE0AEB0E0CCCF810B0BA
S21401BA00641C65E7BDE8FF8F30B400220270002297
S21401BA104270002282700022C2700F220271002240
S21401BA204271002282710122C2714EF660220281A9
S21401BA300022428100221300DBB2032B1DDA002311
S21401BA4019000B00DBB2082B15DA1300DBB200EB92
S21401BA50C3030C00E4B22344002483F83C401300E3
S21401BA60DBB21B0103440C00E4B203EB44030024E5
S21401BA709C81491CE5E7521CDDE7012380F83C3038
S21401BA8000231C00E4B2002C15D100241D00EDB2E9
S21401BA90054485F8544000241D00EDB200EB450531
S21401BAA0A5F8564000241D00EDB200EB4505A5F8AB
S21401BAB058405B1CE5E7002480F85A4030BC7047CC
S21401BAC02DE9F84F88B004000D002000FFF7E6FED0
S21401BAD02989226853681B0C1B04080080B20343A3
S21401BAE05360B5F80AC0D4F800E0DEF80C805FEACF
S21401BAF018485FEA0848604680B250EA0808CEF85F
S21401BB000C8000273800C0B2032839DA002006006E
S21401BB103000C0B2082831DA31003A003800C0B22D
S21401BB20000128443300DBB200EB43008389D4F8DC
S21401BB3000C05FF0280E1000C0B20EFB00F060449B
S21401BB4088465FFA88F800EB8800D0F818805FEA2C
S21401BB5018485FEA0848180080B250EA0808100042
S21401BB60C0B20EFB00FE0CEB0E008E465FFA8EFE98
S21401BB7000EB8E00C0F81880761CC9E77F1CC1E771
S21401BB8015F13C012000FFF7A0FE68788DF806004D
S21401BB902068016831F400319DF80620520412F441
S21401BBA000321143079107990160A9788DF80510B5
S21401BBB021680A6832F400429DF80530DB0313F46D
S21401BBC000431A430692069A0A60EA788DF8042022
S21401BBD02268136833F4E0439DF804C05FEA0C3C26
S21401BBE01CF4E04C5CEA03030593059B13602B7978
S21401BBF08DF803302368D3F800E03EF4706E9DF8AC
S21401BC0003C05FEA0C2C1CF4706C5CEA0E0ECDF8D7
S21401BC1010E0DDF810C0C3F800C095F805E08DF817
S21401BC2002E0D4F800E0DEF8008038F020089DF845
S21401BC3002C05FEA4C1C1CF0200C5CEA0808CDF838
S21401BC400C80DDF80CC0CEF800C095F806808DF8A3
S21401BC500180D4F800A0DAF8008038F00C089DF8CE
S21401BC6001C05FEA8C0C1CF00C0C5CEA0808CDF8ED
S21401BC700880DDF808C0CAF800C095F807808DF87E
S21401BC800080D4F800C0DCF800B03BF0020B9DF851
S21401BC9000805FEA480818F0020858EA0B0BCCF857
S21401BCA000B05FF000085FF000094846C0B2002807
S21401BCB026D14846C0B205EB4000B0F856004946CA
S21401BCC0C9B205EB4101B1F8581051EA00414A46A4
S21401BCD00B00D4F800C01000C0B20CEB8000C0F816
S21401BCE094314846C0B2284490F85400002804D045
S21401BCF0012010FA09F050EA080819F10109D4E701
S21401BD008DF80280D4F800A0DAF89011090A090229
S21401BD109DF80200014304910498CAF8900195F831
S21401BD205A008DF80100606801900198C069C0084A
S21401BD30C0009DF8011011F0070108430390039815
S21401BD400199C8612000FFF79AFD00208DF80000D8
S21401BD50D4F800B0DBF8000030F440209DF8001065
S21401BD60890411F44021084302900298CBF80000A0
S21401BD702000FFF7A2FD2000FFF790FD287821683C
S21401BD800A6832F440220300DBB29B0413F440231A
S21401BD901A430A6009B0BDE8F08FFEE7026932F087
S21401BDA07C520B00DBB21B0613F07C531A43026174
S21401BDB07047026932F47C120B00DBB21B0413F4E9
S21401BDC07C131A4302617047026932F47C520B00FD
S21401BDD0DBB21B0213F47C531A43026170470269FB
S21401BDE0920992010B00DBB213F03F031A43026182
S21401BDF07047426932F07C520B00DBB21B0613F02F
S21401BE007C531A4342617047426932F47C120B003C
S21401BE10DBB21B0413F47C131A4342617047426978
S21401BE2032F47C520B00DBB21B0213F47C531A4330
S21401BE30426170474269920992010B00DBB213F02E
S21401BE403F031A4342617047F8B504000D0016001F
S21401BE502560666000273800C0B2082807DA3A0075
S21401BE60D2B22821200000F0D1F87F1CF3E7F1BD03
S21401BE70F8B504000D00200000F09AF82868216843
S21401BE804A68002303434B602E792768D7F800C021
S21401BE903CF0020CB6465FFA8EFE5FEA4E0E1EF0CE
S21401BEA0020E5EEA0C0CC7F800C0F1BD002101606D
S21401BEB00021017170472DE9FE4F04000D001600A8
S21401BEC0200000F075F872783178200000F09EF8B6
S21401BED0706802908DF80150206802999DF8012043
S21401BEE0120102445161B1688DF8005022689DF834
S21401BEF000301B0113449961337B2F00D4F800E016
S21401BF00BC465FFA8CFC5FEA0C1CF444DCF810803B
S21401BF105FEA98085FEA88089C465FFA8CFC1CF08A
S21401BF20030C5CEA0808CDF80480DDF804C0B846C6
S21401BF305FFA88F85FEA0818F044C8F810C096F867
S21401BF400DC0A846D4F80090C2465FFA8AFA5FEAA6
S21401BF500A1ACA44DAF810A03AF00C0AE3465FFA65
S21401BF608BFB5FEA8B0B1BF00C0B5BEA0A0AC346E2
S21401BF705FFA8BFB5FEA0B1BCB44CBF810A0BDE846
S21401BF80F78F0321017303214173002141600021D2
S21401BF908160704710B40121026813685B085B007A
S21401BFA00C00E4B214F001042343136010BC704784
S21401BFB010B40021026813685B085B000C00E4B251
S21401BFC014F001042343136010BC70472DE9FE4FA3
S21401BFD004000D0016001F0001968DF80050D4F8DD
S21401BFE0008001989DF80010090141444861B94656
S21401BFF0AB46D4F800A05846C0B200015044C0F881
S21401C0001890200000F016F8BDE8F78F70B5040010
S21401C0100D0016003000C0B2082808DA2900C9B29F
S21401C0206068034A3300DBB252F82320904770BDA4
S21401C030BC80020010B401210268D36833F0020309
S21401C0400C00E4B2640014F002042343D36010BC75
S21401C0507047FEE718B589B000F041F86846FDF76D
S21401C06038FA01208DF808008548019001208DF8E6
S21401C0700900844C6A46432114F11800F7F730FF93
S21401C0800028F6D014F5F07469462000FDF75CFA36
S21401C09000212000FDF751FC00200AB010BD7CB540
S21401C0A004000D00784B1C705D70784E00960222DD
S21401C0B001217748FDF713FB3078000271780843B9
S21401C0C080B276BD10B5724C02212000FDF79EFAB3
S21401C0D0012803D102212000FDF7C2FB10BD2DE986
S21401C0E0F04F8FB0674C14F59C7503220E21280083
S21401C0F000F08FFF01208DF805000E26D4F83801D8
S21401C1000790079850F8260030F040009DF805107B
S21401C110890111F0400108430E900E98079941F8E5
S21401C120260001208DF804000E27D4F83801069069
S21401C130069850F8270030F020009DF804104901B9
S21401C14011F0200108430D900D98069941F827003B
S21401C15003220F21280000F05CFF01208DF8030068
S21401C1605FF00F08D4F838010590059850F82800BC
S21401C17030F040009DF80310890111F0400108439A
S21401C1800C900C98059941F8280001208DF80200C2
S21401C1905FF00F09D4F838010490049850F829008C
S21401C1A030F020009DF80210490111F020010843EB
S21401C1B00B900B98049941F82900032200212800CE
S21401C1C000F027FF01208DF801005FF0000AD4F887
S21401C1D038010390039850F82A0030F040009DF88B
S21401C1E00110890111F0400108430A900A98039949
S21401C1F041F82A0001208DF800005FF0000BD4F80A
S21401C20038010290029850F82B0030F020009DF87B
S21401C2100010490111F0200108430990099802997C
S21401C22041F82B0003220121280000F0F2FE012034
S21401C2300121D4F8382152F8213033F040030500AB
S21401C240EDB2AD0115F040052B430893089B42F86B
S21401C250213001250123D4F8384154F823C03CF09D
S21401C260200CAE465FFA8EFE5FEA4E1E1EF0200ED2
S21401C2705EEA0C0C44F823C00FB0BDE8F08F000056
S21401C28040420F00C03100209C3A0020A83A00200E
S21401C290A0330020704710B50400627814F108013D
S21401C2A0606800F0ABF810BD10B5DFF8244400203C
S21401C2B0FCF798F90A21B0FBF1F0E0700520FCF7D5
S21401C2C091F90A21B0FBF1F020710120FCF78AF9FF
S21401C2D00A21B0FBF1F060710220FCF783F90A2114
S21401C2E0B0FBF1F0A0710820FCF77CF90A21B0FB45
S21401C2F0F1F0E07110BD2DE9F84793B00400DFF8C6
S21401C300D4030188491C01800188322936DB0021CB
S21401C3100180FFF7C9FFDFF8B853DFF8BC633100CF
S21401C320280001F04FF9DFF8B473390015F1080061
S21401C33001F08DF9DFF8A883414615F1100001F0F0
S21401C340CAF9DFF8A093494615F1180001F007FA7B
S21401C350DFF894A3514615F1200001F044FA3000AD
S21401C360FFF799FF3800FFF796FF4046FFF793FF68
S21401C3704846FFF790FF5046FFF78DFF684600F0EE
S21401C38009F9012819D1009840F23271884204D087
S21401C390009840F2DF71884208D19DF8443001AA26
S21401C3A0009914F1180001F0FFFC06E09DF84430F6
S21401C3B0009A01A9CD4801F018FFFFF76BFF200096
S21401C3C001F0CFFF14B0BDE8F08710B50400002CD3
S21401C3D00DD000200100C9B2082908DA0100C9B24F
S21401C3E0615CC34A0300DBB2D154401CF2E7082269
S21401C3F0BF4940F2222000F001F810BD2DE9F84FA8
S21401C40094B004000D001600002700205FF000081D
S21401C410B849404691F84920C0B290420ED2CA6C43
S21401C4204346DBB21420434302EB030040688442D8
S21401C43001D1474602E018F10108E9E71420CA6C69
S21401C4403B00DBB24343D25A8DF800208DF848609A
S21401C450C96C3A00D2B200FB02F008444068019071
S21401C460B1465FFA89F9AA460DF1080B4A465146CC
S21401C470584600F07FFFDFF880B26946DBF800001F
S21401C480F9F7F3FD6946DBF80000F9F7E1FD002056
S21401C49015B0BDE8F08F2DE9FE4F0020029041F265
S21401C4A004340025954E2A002100300001F0C6FF15
S21401C4B080260027DFF83C82C1463A003100484614
S21401C4C001F0BCFF8E490020FCF7C9FC4046F7F797
S21401C4D0F2FF0B2088F849008A48C8F84C00DFF8BC
S21401C4E01892DFF824A21AF19800C9F800001AF58C
S21401C4F0987B05220021584600F08BFD052201217C
S21401C500584600F086FD012088F80000002088F8D3
S21401C5100100002088F80200012088F804000020AD
S21401C52088F83000012088F8440002AA0E211AF18A
S21401C5301800F7F7D5FC98F8010001280CD1012066
S21401C54001904FF4FA60009041F64C536F4A0299FD
S21401C55018F11C00F9F7C6FE0020019040F6C41041
S21401C560009041F64C536A4A029918F10800F9F70F
S21401C570B9FE4146D9F80000F8F7E2FF01225FF064
S21401C5808051D9F80000F9F7C9FF6F2000F0EAF8EA
S21401C590BDE8F78F2DE9F0470400002541F201368A
S21401C5A0564F17F598500078B95D884216D05FF05F
S21401C5B04C08B95D4C20414307EB0109A2464246AF
S21401C5C04946504600F0D6FEB85D401CB855B85DE9
S21401C5D0202801D30020B855012005002800C0B24C
S21401C5E0BDE8F0872DE9F04794B0434C5FF08051E9
S21401C5F02068FAF734F8012842D12068FAF77EF865
S21401C6002068FAF76CF800283AD1424D2068FAF70C
S21401C61084F828702878002832D069462068FAF70E
S21401C62085F89DF8485002AE4C274FF49858DFF82D
S21401C630CC9019F808007843484410F1040A2A00FF
S21401C6403100504600F096FE19F80800784301992B
S21401C65049F8001019F8080007FB00F709EB070076
S21401C6609DF8481080F8441019F80800401C09F895
S21401C670080019F80800202802D3002009F808004D
S21401C6805FF000512068F9F7EAFF012804D15FF056
S21401C69000512068F9F7C6FF5FF080412068F9F77E
S21401C6A0DEFF012804D15FF080412068F9F7BAFF68
S21401C6B05FF000412068F9F7D2FF012804D15FF04E
S21401C6C000412068F9F7AEFF14B0BDE8F08700001E
S21401C6D08C3500200E3B00205C2E00206C2E0020A6
S21401C6E07C2E00208C2E00209C2E002088350020D9
S21401C6F07404FF1FD41A0020582E0020541B00205B
S21401C700FC800200C0790200C031002080841E0037
S21401C71020A107001F3B0020010009B2002909D40F
S21401C720012210F01F018A400C4903001BB25B096D
S21401C73041F823207047000009480168012906DBFB
S21401C7400168491E01600068012800DA62B6704778
S21401C75072B603480168491C0160704700E100E0B9
S21401C760F030002010B50400200000B2FFF7D4FF1F
S21401C77010BDFEE71CB5032000F00AF804000022F5
S21401C7802100C9B2032000F00BF80090009816BDF6
S21401C79010B50400002114F07F00FFF780FC10BDE7
S21401C7A0F8B505000E0014003100C9B255F080003E
S21401C7B0C0B2FFF774FC0700002C00D027808DF86C
S21401C7C000502800C0B2FFF7E3FF70408DF801006B
S21401C7D08DF802600098F2BD2DE9FC4705000E00B9
S21401C7E0170098460A9C2800C0B2FFF7D1FF814681
S21401C7F0002C01D0A4F80090CA463AEA060A404640
S21401C800C0B2B84050EA0A0A5146C9B255F0800093
S21401C810C0B2FFF744FC8DF800504046C0B2B840A5
S21401C8208DF802002800C0B2FFF7B2FF01003140C8
S21401C8309DF8020048408DF801000098BDE8F68793
S21401C8402DE9F04F97B01521152400250800C0B238
S21401C85091EA10110800C0B291EA90010800C0B236
S21401C86091EA50018DF804109DF8040010F00100C3
S21401C870012801DB952004005FF0000A5FF0000B41
S21401C880504680B2C0088DF809005FEA4A108DF85C
S21401C890080000208DF8070000265846C0088DF8CD
S21401C8A006005FEA4B108DF8050000275FF00008D0
S21401C8B003A83349502200F06DFD0DF10C0989F8EB
S21401C8C001409DF809008DF835009DF808008DF8A7
S21401C8D037009DF807008DF839008DF83B609DF80C
S21401C8E006008DF83D009DF805008DF83F008DF897
S21401C8F041708DF843808DF85750FFF7ABFB002849
S21401C9000AD000208DF80000FF208DF801000020DD
S21401C9108DF80200009830E05FF0000A5046C0B281
S21401C92019F81000002807D103A85146C9B200EB38
S21401C93041004078002816D0002203A85146C9B20B
S21401C94000EB410041785046C0B219F81000FFF7DD
S21401C95027FF00909DF80100002801D000980CE008
S21401C9601AF1010ADAE700208DF8000000208DF8A0
S21401C970010000208DF80200009817B0BDE8F08F86
S21401C980947D0200DFF834264FF47A714843B2FBF7
S21401C990F0F0401C70470A00D2B2521C0E2303FB73
S21401C9A002F3DFF81C2653434FF47A725043B3FB6D
S21401C9B0F0F0401C704710B402001000C0B292EABA
S21401C9C050041000C0B294EA90041000C0B294EA79
S21401C9D01014A40114F04004130193EA821393EA9D
S21401C9E0C20393EA820313F0800393F08003234388
S21401C9F00800C0B201280CD11000C0B210F0C0006F
S21401CA001C00E4B2A04201D0FF2004E012F03F0077
S21401CA1001E053EA0200C0B210BC70472DE9F843AA
S21401CA200400894615001E0000275FF0000820005C
S21401CA30C0B201280DD14846C0B23C2809D04846AC
S21401CA40C0B23D2805D000214846C0B2FFF7B3FF6B
S21401CA500700002108003200C0B2D2B290420ED2C6
S21401CA600800C0B2285C3F18380080B2B0F5807F5D
S21401CA7003DB7F1C07F0FF07FFE7491CEAE7BFB2AD
S21401CA80FF433800C0B2BDE8F28370B504000D0064
S21401CA90002000263000A178C0B2884216D2207A43
S21401CAA00121B140084208D0DFF81C053100C9B2A7
S21401CAB0405C3100C9B2685406E060683100C9B212
S21401CAC0405C3100C9B26854761CE3E7A3782A00BB
S21401CAD021780120FFF7A2FF287270BD38B5DFF874
S21401CAE0EC442078002815D1DFF8E454012208210F
S21401CAF0280002F0C3F8DFF8DC040168DFF8D80488
S21401CB0000684118DFF8D404016001202070280075
S21401CB1002F01AFB31BD10B5DFF8B4445FF4802192
S21401CB20200002F039F8002810D05FF480212000A0
S21401CB3002F07EF80020DFF8A81408700220DFF863
S21401CB408C1408705521200002F00AF810BD2DE95A
S21401CB50FE4F002500208DF8000000208DF806000D
S21401CB6000208DF8050000208DF8040000208DF8C7
S21401CB70030000208DF8020000208DF80100DFF888
S21401CB8050442021200002F007F8002800F05B81C5
S21401CB902021200002F046F9012840F05481DFF8F8
S21401CBA02C64307802280BD0C0F04A81042800F0AB
S21401CBB0A38027D3062800F00C81C0F0DE803FE179
S21401CBC0200001F0DBFF8DF800009DF800005528DD
S21401CBD015D10021DFF8EC23DFF8080403780C20D8
S21401CBE04343D05CFFF7E7FE8DF804009DF8041080
S21401CBF089B2200001F0B4FF0320307001E000206C
S21401CC00307020E1200001F0B9FF8DF8000001210D
S21401CC109DF80000FFF7CFFE8DF803000C27DFF824
S21401CC20C483DFF8A0939DF8030098F800107943B9
S21401CC3019F80110884202D00020307003E198F8FC
S21401CC40000078434844C078002843D1DFF898A311
S21401CC50514698F8000078434844FFF716FF042031
S21401CC603070DFF87CB300208BF80000200002F063
S21401CC701DFAD0F104008DF80200002005002800FE
S21401CC809DF80210C0B2884235D29BF800001AF80F
S21401CC90001089B2200001F063FF9BF80000401CE1
S21401CCA08BF800009BF8000098F80010794349447F
S21401CCB0897888420CD39BF80000042808DA9AF891
S21401CCC0081089B2200001F04BFF0620307012E0F8
S21401CCD06D1CD4E798F8000007FB00F709EB070086
S21401CCE0C078012805D10020C049087005203070A1
S21401CCF001E000203070A6E0200002F0CEF98DF8A9
S21401CD000100002738009DF80110C0B2884204D205
S21401CD10200001F033FF7F1CF4E7200002F0C6F983
S21401CD20D0F104008DF80200002528009DF80210BD
S21401CD30C0B2884220D2AA4F3978A24AA9480378BD
S21401CD400C20434302EB03008078814208D3A648B7
S21401CD50017A89B2200001F003FF062030700BE053
S21401CD60A1483978415C89B2200001F0F9FE387893
S21401CD70401C38706D1CD8E765E0200002F08DF984
S21401CD808DF801000020050028009DF80110C0B2B2
S21401CD9088421DD2200001F0F1FE8DF80000934874
S21401CDA09DF80010924A0378D1540178491C01700D
S21401CDB00178844A8B4803780C20434302EB030036
S21401CDC08078814202D30620307001E06D1CDBE7DB
S21401CDD039E0200001F0D2FE8DF806000C27DFF8BE
S21401CDE00482DFF8E09198F8000078434844C07860
S21401CDF0012822D1DFF8F8A1DFF8F0B19BF8003066
S21401CE00524698F80000784319F800100120FFF701
S21401CE1005FE8DF805009DF805009DF80610884270
S21401CE200BD19BF80020514698F8000007FB00F74D
S21401CE3009EB0700406802F0BFF90020307002E0FD
S21401CE40200002F03DF961480078002803D1012155
S21401CE50200002F07FF9BDE8F78F10B55B4908782E
S21401CE60401E052810D85D4C2068401E20602068B2
S21401CE70002808D1002008700121554802F06AF9FF
S21401CE80554800682060FFE710BD38B58CB0594C96
S21401CE9014F59C7504220221280000F0BAF8042239
S21401CEA00321280000F0B5F801220D21280000F02A
S21401CEB0B0F801220D21280000F0E0F801220D2132
S21401CEC0280000F0EEF8684602F04EF84FF496405F
S21401CED0019001208DF82C006A46452114F11800B6
S21401CEE0F6F7FEFF14F5F6746946200002F086F8A0
S21401CEF00021200002F0F1F80021200002F0EDF8F8
S21401CF0001220821200001F0B9FE01222021200083
S21401CF1001F0B4FE1F20FFF725FC2E4C4FF496407F
S21401CF20FFF730FD20602C4D08214FF49640FFF7A7
S21401CF3032FD2860216828684118284801600020D1
S21401CF40224908700DB030BDF0B40C241D4D03000D
S21401CF50DBB263432B445B680E00F6B29B5D1A4E50
S21401CF600F00FFB2F35501260300DBB2634305EB66
S21401CF7003070300DBB263432B4493F808C016FA99
S21401CF8001F353EA0C0C87F808C00300DBB26343D5
S21401CF902B445B680F00FFB2DA550300DBB2634334
S21401CFA02B440700FFB204FB07F42C44247A8E407E
S21401CFB034EA06061E72F0BC704700008051D602A5
S21401CFC040420F00EC04FF1FAC310020263B00203E
S21401CFD0AC330020B8310020BC310020B431002031
S21401CFE0233B0020253B00206C310020243B002001
S21401CFF078310020C031002080B5FFF76FFD01BDFC
S21401D00080B5FFF788FDFFF7A2FD01BD0160426014
S21401D0107047F0B413000C00056855F8246036F428
S21401D020E0661F00FFB23F0217F4E0673E4345F893
S21401D03024601700FFB2002F0FD101230C000568F2
S21401D04055F8246036F004061F00FFB2BF0017F043
S21401D05004073E4345F824600EE000230C000568F3
S21401D06055F8246036F004061F00FFB2BF0017F023
S21401D07004073E4345F82460F0BC704730B443686B
S21401D0805B6901248C40A3431400E4B28C40234323
S21401D0901C0045686C6130BC70470A0043689A61A1
S21401D0A0704730B443681B6801248C40A3431400C6
S21401D0B0E4B28C4023431C0045682C6030BC7047AA
S21401D0C001228A4043685A60704701228A404368B9
S21401D0D09A60704710B40300002458680069012262
S21401D0E08A400240002A01D1002000E00120C0B29F
S21401D0F010BC704710B5044610460A460146204645
S21401D10001F09CF9204610BD10B5DFF8544203200B
S21401D110206103206061DFF84C02A061DFF848124D
S21401D120E1614FF4806121620021A1620021616208
S21401D1300021E1622066DFF8340260661020A066F6
S21401D140002020670020E0660020606753A1E01DF4
S21401D15002F038F8BFF35F8FDFF81412200002F0F8
S21401D16031F8BFF35F8F2020A071BFF35F8F10BD32
S21401D1702DE9FE4F05000E0014005FF00008D5F8FB
S21401D1800C9028690700B94503D2B7EB0900401E89
S21401D19004E0A868B0EB09003818401EA968B1EB96
S21401D1A00901884201D2824603E0D5F808A0BAEB0D
S21401D1B0090AA24500D3A246686848440090CDF803
S21401D1C008A00196DDF800B0029A0199584600F0D1
S21401D1D0D1F81AEB08085644B4EB0A041AEB09090D
S21401D1E0A868814501D100208146BFF35F8FC5F84D
S21401D1F00C90002CC5D14046BDE8FE8F2DE9F84FB6
S21401D20084B004000D001600E768D4F80880B8EB77
S21401D210070846450FD2606800EB07090196AA4643
S21401D220CB46019A5146584600F0A4F8BFF35F8FEB
S21401D230F019E06021E0CDF8008060683844019084
S21401D240009803900295DDF80490039A02994846E7
S21401D25000F090F8B6EB08000090D4F8049000981F
S21401D260019005EB080ACB46019A5146584600F054
S21401D27081F8BFF35F8F0098E06005B0BDE8F08FDE
S21401D28001000A69CB68934204D38868401EC01A1D
S21401D290101801E0D01A401E704700005254540086
S21401D2A02DE9F04704000D001600A846DFF8B0008F
S21401D2B0182101FB04F1084410F1180ADAF81400E9
S21401D2C0002803D0022820D010D325E05046FFF7CF
S21401D2D0D7FF0700B74202D25FF0000905E0B1466A
S21401D2E0320041465046FFF789FF17E05046FFF7E8
S21401D2F0C7FF0700B74201D2B94600E0B1464A4629
S21401D30041465046FFF77AFF08E032004146504654
S21401D310FFF72EFF814601E05FF000094846BDE8B1
S21401D320F0872DE9F04104000D001600DFF830709B
S21401D3303878002801D1FFF7E7FEEFF311882020A7
S21401D34080F31188320029002000FFF7A9FF88F337
S21401D3501188BDE8F08180B5FFF7D6FE01BD00005B
S21401D360E4350020EC8102008C3600208C3A002047
S21401D3700082020062B38B0708D0521E11F8013BEF
S21401D38000F8013B00F024808B07F6D1830740F0BC
S21401D390208000BF103A07D330B4B1E83810103AF5
S21401D3A0A0E83810F9D230BC530724BFB1E8081002
S21401D3B0A0E8081044BF51F8043B40F8043BD207EC
S21401D3C024BF31F8022B20F8022B44BF0B780370E0
S21401D3D07047121F17D35B0009D151F8043B20F8A0
S21401D3E0023B1B0C121F20F8023BF6D20BE051F851
S21401D3F0043B00F8013B1B0A20F8023B1B0C121FE2
S21401D40000F8013BF3D238BF121D521E24BF11F89B
S21401D410013B00F8013BF8D8704710B403000878C8
S21401D42010F001001C7814F0FE04204318700878F0
S21401D430C0B240081C7860F341041C700878C0B282
S21401D44080081C7860F382041C700878C0B2C0089B
S21401D4501C7860F3C3041C700878C0B200091C78FD
S21401D46060F304141C700878C0B240091C7860F39D
S21401D47045141C700878C0B280091C7860F38614C5
S21401D4801C700878C0B2C0091C7814F07F0454EAF6
S21401D490C0141C70487810F001005C7814F0FE048B
S21401D4A0204358704878C0B240085C7860F3410465
S21401D4B05C704878C0B280085C7860F382045C7067
S21401D4C04878C0B2C0085C7860F3C3045C708878A2
S21401D4D05C7860F304145C708878C0B240085C78AD
S21401D4E060F345145C708878C0B200095C7860F31C
S21401D4F086145C70C87810F001005C7814F07F0424
S21401D50054EAC0145C70C878C0F340009C7814F0EC
S21401D510FE0420439870C878C0B280089C7860F3F7
S21401D52041049C70C878C0B2C0089C7860F382043D
S21401D5309C7008799C7860F3C3049C700879C0B22B
S21401D54040089C7860F304149C7048799C7860F3DA
S21401D55045149C704879C0B240089C7860F38614E4
S21401D5609C704879C0F380009C7814F07F0454EADC
S21401D570C0149C704879C0F3C000DC7814F0FE0437
S21401D5802043D8704879C0B20009DC7860F34104C2
S21401D590DC704879C0B24009DC7860F38204DC7044
S21401D5A04879C0B28009DC7860F3C304DC7048793E
S21401D5B0C0B2C009DC7860F30414DC7040F20120CC
S21401D5C010BC704710B4020000231800C0B208282F
S21401D5D006D200201C00E4B20C4420725B1CF4E767
S21401D5E00C7A107804430C72487A547814F00F04BD
S21401D5F0204348728C7A5078C0F301100443507867
S21401D600C0B2800954EA80049078000110F030001E
S21401D61004438C72CC7AD0780443CC720C7B10799C
S21401D62004430C734C7B507904434C738C7B907988
S21401D63004438C73CC7BD0790443CC7340F2013025
S21401D640486008244C7000240C7010BC704710B45D
S21401D650020000231800C0B2082806D200201C00D1
S21401D660E4B20C4420725B1CF4E70C7A1078044395
S21401D6700C72487A547814F0030420435478C4F3A7
S21401D680800450EA840048728C7A508804438C7275
S21401D690C87A5488A4B2240A2043C8720C7B9088A6
S21401D6A004430C73487B9488A4B2240A204348732D
S21401D6B08C7BD08804438C73C87BD488A4B2240A9C
S21401D6C02043C87340F20140486008244C7000248F
S21401D6D00C7010BC704710B4020000231800C0B2D2
S21401D6E0082806D200201C00E4B20C4420725B1C01
S21401D6F0F4E70C7A107804430C72487A547814F0E4
S21401D700030420435478C4F3800450EA840048722A
S21401D7108C7A508804438C72C87A5488A4B2240A3E
S21401D7202043C8720C7B908804430C73487B948812
S21401D730A4B2240A204348738C7BD08804438C739C
S21401D740C87BD488A4B2240A2043C87340F202409E
S21401D750486008244C7000240C7010BC704710B44C
S21401D760020000231800C0B2082806D200201C00C0
S21401D770E4B20C4420725B1CF4E70C7A1078044384
S21401D7800C72487A547814F0030420435478C4F396
S21401D790800450EA840048728C7A508804438C7264
S21401D7A0C87A5488A4B2240A2043C8720C7B908895
S21401D7B004430C73487B9488A4B2240A204348731C
S21401D7C08C7BD08804438C73C87BD488A4B2240A8B
S21401D7D02043C87340F20340486008244C7000247C
S21401D7E00C7010BC704710B4020000231800C0B2C1
S21401D7F0082806D200201C00E4B20C4420725B1CF0
S21401D800F4E70C7A107804430C72487A547814F0D2
S21401D810030420435478C4F3800450EA8400487219
S21401D8208C7A508804438C72C87A5488A4B2240A2D
S21401D8302043C8720C7B908804430C73487B948801
S21401D840A4B2240A204348738C7BD08804438C738B
S21401D850C87BD488A4B2240A2043C87340F204408B
S21401D860486008244C7000240C7010BC7047FEE71A
S21401D870010008000200D2B2802A01DB7F221000DC
S21401D880C0B2704701000800C0B2F12805DB0800ED
S21401D890C0B2FA2801DA012006E00800C0B28028EA
S21401D8A001DA080000E00020C0B270472DE9FC4113
S21401D8B004000D0016001F005FF000083F208DF8E1
S21401D8C000009DF8001055F0F00001408DF80010A2
S21401D8D08DF801603800C0B2FFF7CAFF8DF802006C
S21401D8E02078002813D0032080464046C0B208287E
S21401D8F007DA002069464246D2B2885418F1010878
S21401D900F3E708226946E068A36D984704E003221E
S21401D9106946E068A36D984740B2BDE8F6817CB5DC
S21401D9200400002500200F218DF800109DF800103E
S21401D930E28A52F0F00211408DF800100026300005
S21401D940C0B2E18A80B288420AD220693100C9B2E7
S21401D950405C69463200D2B211444870761CEEE74C
S21401D9602078002817D0002005002800C0B2E18AE0
S21401D970D1F10701884208DA6846E18A51FA85F151
S21401D9800844002141706D1CEFE708226946E068F3
S21401D990A36D984706E0E28A521CD2B26946E06857
S21401D9A0A36D984740B276BD3EB504001F208DF8A2
S21401D9B000009DF80000E18A89B2090A51F0F001E1
S21401D9C008408DF80000E08A8DF80100002000254F
S21401D9D02800C0B206280ADA20692900C9B2405CCC
S21401D9E069462A00D2B2114488706D1CF0E70822FD
S21401D9F06946E068A36D9847010049B2002904D141
S21401DA00218B891D21830121A17640B23EBDFEB541
S21401DA10040000212F208DF800009DF80000A27E52
S21401DA2052F0F00210408DF80000E58A208B2D1A86
S21401DA30280080B2082801DB0720050000263000F8
S21401DA40C0B2290080B289B288420BD22069218BEC
S21401DA5051FA86F1405C69463200D2B211444870F0
S21401DA60761CECE72078002819D000200027380023
S21401DA70C0B2290089B2D1F10701884209DA6846A5
S21401DA80290089B251FA87F10844002141707F1CB0
S21401DA90EDE708226946E068A36D984705E06A1C31
S21401DAA0D2B26946E068A36D9847010049B20029E1
S21401DAB00AD1218B69182183A17E491CA176A17EFA
S21401DAC0102901DB0021A17640B2FEBDF8B50400A5
S21401DAD00D0016000027287810F00F0F07D0300031
S21401DAE0C0B2401E297811F00F01884208DA606D35
S21401DAF0002802D0A448616D88477FF0060017E031
S21401DB00287810F00F00A4F8420000210800C0B2E7
S21401DB10B4F8422080B2904209D20800C0B228442C
S21401DB204078E26B0B00DBB2D054491CEEE70020D4
S21401DB30F2BD2DE9F04104000D001600002730006B
S21401DB40C0B2082808D0606D002802D08F48616DE9
S21401DB5088477FF006003AE02878000210F47060EB
S21401DB60697810EB0108404680B2082808DA606D33
S21401DB70002802D08648616D88477FF0060026E0BF
S21401DB80B4F84000414689B2884208D2606D002848
S21401DB9002D08048616D88477FF0020017E0A4F844
S21401DBA0428000210800C0B2062809DA0800C0B287
S21401DBB028448078E26B0B00DBB2D054491CF1E7B5
S21401DBC00620A4F84400012084F846000020BDE8A1
S21401DBD0F0812DE9F04104000D001600002794F8AD
S21401DBE04600297811F00F01884202D07FF0030029
S21401DBF042E0B4F84280B4F84400B8EB000840466E
S21401DC0080B2082801DB072080463000C0B2401EE3
S21401DC10414689B2884208DA606D002802D05E4823
S21401DC20616D88477FF0060026E000210800C0B23B
S21401DC30424680B292B290420BD2E06BB4F84420D6
S21401DC4052FA81F20B00DBB22B445B788354491CF9
S21401DC50ECE7B4F8440018EB0000A4F8440094F88C
S21401DC604600401C84F8460094F84600102802DB63
S21401DC70002084F846000020BDE8F08170B504005D
S21401DC800D0016003000C0B2032808DA606D0028C7
S21401DC9002D04248616D88477FF0060000E0002010
S21401DCA070BD70B504000D00160033009BB22A004B
S21401DCB0E168200000F001F870BD2DE9F84304008A
S21401DCC0894615001E005FF00008002C02D15FF0A7
S21401DCD0FF3056E0A08A310089B2884208D2606DD2
S21401DCE0002802D02E48616D88477FF0020048E088
S21401DCF094F83400012808D1606D002802D0294824
S21401DD00616D88477FF001003BE0E68200202083BA
S21401DD1000273800C0B2310080B289B2884208D2EA
S21401DD203800C0B2285C21693A00D2B288547F1C00
S21401DD30EFE7E08A082804DA2000FFF7F0FD8046C6
S21401DD401DE02000FFF730FE8046404640B2002826
S21401DD5015D10020A0830020A0770020E077E06D99
S21401DD608047C4E90801E06D8047643051F1000145
S21401DD70C4E90A0100202063012084F834004046EB
S21401DD8040B2BDE8F2830000D07F0200FC7F0200B3
S21401DD90647E02009C7E02007C8002009C80020061
S21401DDA00C7F0200407F02002DE9FE4304000D00B7
S21401DDB091461E003000C0B2022803DB3000C0B21C
S21401DDC0092800DB27E10020002108003200C0B24C
S21401DDD0D2B2904209D20800C0B219F800006A46D1
S21401DDE00B00DBB2D054491CEFE75FF00008404659
S21401DDF0C0B23100C9B2D1F10801884209DA002067
S21401DE0069463200D2B252FA88F2885418F10108F3
S21401DE10EDE79DF80000C0B20009002806D00228F0
S21401DE2061D01FD3032800F0A880F4E094F85100D5
S21401DE30012804D17FF0050084F8500002E000209C
S21401DE4084F850003200D2B269462000FFF73EFE49
S21401DE500700380040B2002803D1A563022084F8E9
S21401DE605100D8E094F85100012804D17FF0050054
S21401DE7084F8500002E0002084F850003200D2B24C
S21401DE8069462000FFF755FE070038007FF00201C3
S21401DE9040B288420DD17FF0070084F85000002080
S21401DEA084F851000023002202212000FFF7FEFC27
S21401DEB0B1E0380040B2002814D1A563012084F8EF
S21401DEC05100607884F84700002394F84720002129
S21401DED02000FFF7EBFCE06D8047643051F1000154
S21401DEE0C4E9120197E094F85100012804D07FF0AC
S21401DEF0050084F850008EE0A06B854240F08B80D0
S21401DF003200D2B269462000FFF763FE07007FF0B9
S21401DF1003003900020049B2914205D184F850004D
S21401DF20002084F8510076E0380040B2002823D162
S21401DF30E06D8047643051F10001C4E91201B4F884
S21401DF404400B4F84210884203D3022084F85100FA
S21401DF5012E094F84700401E84F8470094F8470002
S21401DF60002809D1607884F84700002394F84720F8
S21401DF7000212000FFF79AFC4DE094F834000128B8
S21401DF8049D13200D2B269462000FFF777FE07007A
S21401DF90380040B200283DD1E06D8047643051F131
S21401DFA00001C4E90A019DF8000010F00F000228E4
S21401DFB006D17FF007002063022084F8340029E0B0
S21401DFC09DF8000010F00F0001280CD1E07F401CE6
S21401DFD0E077E07F02281DDB7FF006002063022049
S21401DFE084F8340016E09DF8000010F00F0F11D1F0
S21401DFF09DF80100002803D14FF6FF70A08302E0D0
S21401E0009DF80100A0839DF80200FFF73BFCA07776
S21401E0100020E077FFE7BDE8F783F0B40400049D35
S21401E020002694F85100022802D07FF0040028E070
S21401E030A06BA768B84201D1012000E0002008705B
S21401E040B4F842701800BC4680B21FFA8CFC6045DA
S21401E05000D21F005FF0000C60463E0080B2B6B2F0
S21401E060B04209D2E06B6646B6B2805D6646B6B28D
S21401E07090551CF1010CEFE72F80002084F8510029
S21401E0800020F0BC70470A7802704A7842704A68ED
S21401E09042608A688260CA68C2600A6902618A8AC6
S21401E0A082820022C282002202830022827600221D
S21401E0B08283002282770022C27700220023C0E9F1
S21401E0C0082300220023C0E90A230022026300225B
S21401E0D080F834208A69C2638A8BA0F84020002227
S21401E0E0A0F842200022A0F84420002280F8462012
S21401E0F0002280F8472000220023C0E912230022D4
S21401E10080F85020002280F851200A6A42654A6A47
S21401E11082658A6AC265704770B5040094F8340057
S21401E12001284DD14FF6FF76A08BB04202D0A08BCE
S21401E130002836D0A07F00280BD0A07F002830D042
S21401E140E06D8047D4E90823101A73EB010100291A
S21401E15027D52000FFF75BFC0500280040B2002809
S21401E1601CD1A08BB04202D0A08B401EA083E06DD4
S21401E1708047643051F10001C4E90A01E06D80472F
S21401E180A27F002380185941C4E90801208BE18A47
S21401E190884206D3002084F8340002E0022084F886
S21401E1A03400E06D8047D4E90A23101A73EB0101AD
S21401E1B0002905D57FF001002063022084F8340091
S21401E1C094F8510001280FD1E06D8047D4E912235D
S21401E1D0101A73EB0101002906D57FF0020084F8BE
S21401E1E05000002084F8510070BD2DE9F041040074
S21401E1F00D0016001F005FF0000840F20120864265
S21401E20006D13A00D2B229002000FFF706F980466F
S21401E2104046BDE8F08100210160002141600021F7
S21401E22001720021417270470022026041600122A2
S21401E2300272002242727047407A7047FEB50400AF
S21401E2400D001600082100226F46380000F0F6F88F
S21401E2503000C0B2782807D041F28C00215A41F232
S21401E260A8002044FFF7E0FF94F87900002814D0B6
S21401E2703000C0B211280FD03000C0B212280BD027
S21401E2803000C0B2312807D03000C0B27E2803D09B
S21401E2903000C0B27F2800D10CE07F208DF800004E
S21401E2A08DF801508DF802600322694614F11800BA
S21401E2B0FFF7F7FCF7BD10B402000020002318009A
S21401E2C080B25468A0420CD290681C00A4B210F828
S21401E2D034000C00E4B2A04201D1012002E05B1C34
S21401E2E0EDE7002010BC704738B504000D0029008A
S21401E2F014F11800FFF7C7FE012060700020A0701F
S21401E300002084F878000020002114F58452C2E928
S21401E3100001A88D41F288016052E88D41F28A0120
S21401E3206052288E41F28C01605241F290002044E6
S21401E330FFF771FF41F29C002044FFF76CFF41F2AA
S21401E340A8002044FFF767FF00200021B1F5805F99
S21401E35006D2002004EB010282F87B00491CF5E797
S21401E36031BD2DE9FC4104000020ADF804005FF04A
S21401E37000080025002614F11800FFF7CDFE01A8BD
S21401E38000904FF4805314F17B0214F1790114F1DB
S21401E3901800FFF742FE0700380040B200283AD1C5
S21401E3A094F87B0005002900C9B22000FFF783FF1F
S21401E3B000282AD000200600606886422BD2A0687A
S21401E3C010F836002900C9B288421CD1A06800EBBB
S21401E3D0C6008078002806D094F87C00C0B2C00938
S21401E3E084F8780002E0002084F8780084F87A60E7
S21401E3F0BDF8042014F17B012000A36803EBC603DB
S21401E4005B68984707E0761CD6E711222900C9B257
S21401E4102000FFF713FF41F2A80804EB0800FFF7FE
S21401E4200BFF012807D1012060700020A07004EBCB
S21401E4300800FFF7F0FEBDE8F381000062F30F224B
S21401E44062F31F42401810F0030308D0C91A1FD305
S21401E450DB0748BF00F8012D28BF20F8022D130066
S21401E46030B414461546103928BF20E93C00FAD8C6
S21401E470490728BF20E90C0048BF40F8042D890051
S21401E48028BF20F8022D48BF00F8012D30BC704788
S21401E490C91818BF00F8012DCB0728BF00F8012DB9
S21401E4A0704700002DE9F0430200C87A022813DA0B
S21401E4B0C87A13681C6834F400740500EDB26D0266
S21401E4C015F400752C431C6001251668376857F44F
S21401E4D0806CC6F800C005E0002013681C6834F4A0
S21401E4E080651D600B7A1468256835F48055180020
S21401E4F0C0B2000310F48050054325604E7A1768B9
S21401E500D7F804C03CF4005C3000C0B2400310F4FD
S21401E510005050EA0C0CC7F804C091F80AE0D2F893
S21401E5200080D8F8049039F400297046C0B2C004BF
S21401E53010F4002050EA0909C8F80490487B002826
S21401E54001D0012000E0002013681C680500EDB230
S21401E550002D03D054F400451D6002E034F400455C
S21401E5601D600D7B1668B76837F40067AC465FFA26
S21401E5708CFC5FEACC2C1CF4006C5CEA0707B760E5
S21401E580D1F804C01CF1010F23D000204B7B012BD6
S21401E5900AD10B684C686408B3FBF4F31C09240128
S21401E5A0C3F34203234303E00B684C68B3FBF4F365
S21401E5B01C001568EE6816F07F46200080B2064300
S21401E5C0EE6000201768D7F804C03CF4801EC7F838
S21401E5D004E0887B00282ED002281ED00FD3032803
S21401E5E037D1012013681C6854F004051D6001250D
S21401E5F01668376857F0080CC6F800C036E00020E9
S21401E60013681C6834F004051D6001251668376818
S21401E61057F0080CC6F800C028E0012013681C68F3
S21401E62054F004051D6000251668376837F0080C9D
S21401E630C6F800C01AE0002013681C6834F0040510
S21401E6401D6000251668376837F0080CC6F800C04C
S21401E6500CE0002013681C6834F004051D600025DA
S21401E6601668376837F0080CC6F800C0BDE8F083B6
S21401E6702DE9F04F8AB0557903689C682E00F6B2F2
S21401E680012E03D154F004069E6002E034F0040625
S21401E6909E60167A012E07D0C0F00E81032E00F080
S21401E6A0BD80C0F0978007E100238DF80530036830
S21401E6B09C680994099C34F400749C6000248DF8CD
S21401E6C004400468A5680895089D35F48075A56022
S21401E6D000250668B7680797079F37F48047B76035
S21401E6E00F798DF803700768D7F804E05FEA9E0E8D
S21401E6F05FEA8E0E9DF803C01CF0030C5CEA0E0E5A
S21401E700CDF818E0DDF818C0C7F804C091F805E0A8
S21401E7108DF802E0D0F800C0DCF8048038F0040878
S21401E7209DF802E05FEA8E0E1EF0040E5EEA08080F
S21401E730CDF81480DDF814E0CCF804E091F80680FA
S21401E7408DF80180D0F800E0DEF8049039F0600919
S21401E7509DF801805FEA481818F0600858EA090930
S21401E760CDF81090DDF81080CEF804805FF0010837
S21401E770D0F80090D9F804B0CDF80CB0DDF80CA0B4
S21401E7805AF4804AC9F804A092F807B08DF800B090
S21401E790D0F800A0DAF804B0CDF808B09DF800B0C3
S21401E7A0BBF1010F05D1029B53F40043CAF80430B4
S21401E7B004E0029B33F40043CAF80430D379012BFA
S21401E7C007D10B7C0468656925F07F4555EA03652A
S21401E7D0656194E00023046865680195019D35F440
S21401E7E08045656000250668B7680097009F37F486
S21401E7F08047B7600127D0F800C0DCF808E05EF477
S21401E8000078CCF808805FF00108D0F80090D9F8BD
S21401E81008A05AF4807BC9F808B070E000230468A9
S21401E820656835F4804666604E7B0768D7F800E079
S21401E8303EF4F81EB4465FFA8CFC5FEA0C4C1CF4FE
S21401E840F81C5CEA0E0ECDF804E0DDF804C0C7F84B
S21401E85000C091F80EE0D0F80080D8F8009039F0AA
S21401E860F879F4465FFA8CFC5FEA4C5C1CF0F87CA5
S21401E8705CEA0909CDF80090DDF800C0C8F800C0D0
S21401E88091F80FC0D0F80090D9F808A0E3465FFAD7
S21401E8908BFBBBF1010F04D15AF40043C9F80830D1
S21401E8A003E03AF40043C9F8083001230468A56878
S21401E8B055F48046A66022E000230468A568019509
S21401E8C0019D35F40075A56000250668B7680097B8
S21401E8D0009F37F48077B7600027D0F800C0DCF8D7
S21401E8E008E03EF48048CCF808805FF00008D0F8D5
S21401E8F00090D9F804A03AF4804BC9F804B092F815
S21401E90002C0066877686346DBB2012B03D157F471
S21401E9108033736002E037F480337360D378046821
S21401E92065689E465FFA8EFEBEF1010F03D155F46F
S21401E9300036666002E035F40036666092F804C080
S21401E94006687768E6465FFA8EFEBEF1010F03D1D0
S21401E95057F48023736002E037F4802373605378A2
S21401E960012B17D101230468656855F4801666608B
S21401E9700E780768D7F804C03CF4C00CB6465FFAB8
S21401E9808EFE5FEA4E5E1EF4C00E5EEA0C0CC7F801
S21401E99004C005E000230468656835F480166660E7
S21401E9A08B68002B11D08C6805686E6916F07F465F
S21401E9B024F07F431E436E6101230768D7F804C025
S21401E9C05CF4000EC7F804E005E0002304686568FF
S21401E9D035F4000666609379012B42D1CB78012B82
S21401E9E01BD10B7B0468656825F07F451E00F6B2D7
S21401E9F055EA066565608E780768D7F804C03CF46A
S21401EA00C00CB6465FFA8EFE5FEA4E5E1EF4C00E7E
S21401EA105EEA0C0CC7F804C00BE0CB7904686568A5
S21401EA2035F4E0651E00F6B2360216F4E0663543AC
S21401EA30656001230468256855F400562660CE7883
S21401EA400768D7F800C03CF4006CB6465FFA8EFE45
S21401EA505FEACE2E1EF4006E5EEA0C0CC7F800C00C
S21401EA6016E000230468256835F400562660CE7942
S21401EA700768D7F804C03CF4E06CB6465FFA8EFE31
S21401EA805FEA0E2E1EF4E06E5EEA0C0CC7F804C0B8
S21401EA901378012B53D14B78002B05D0022B21D0B4
S21401EAA011D3032B2DD03BE000230468A56835F075
S21401EAB04006A66000260768D7F808C03CF0800E1E
S21401EAC0C7F808E049E000230468A56835F0400669
S21401EAD0A66001260768D7F808C05CF0800EC7F864
S21401EAE008E03AE001230468A56855F04006A660F0
S21401EAF000260768D7F808C03CF0800EC7F808E083
S21401EB002BE001230468A56855F04006A66001269F
S21401EB100768D7F808C05CF0800EC7F808E01CE06C
S21401EB2000230468A56835F04006A660002607683D
S21401EB30D7F808C03CF0800EC7F808E00DE00023C7
S21401EB400468A56835F04006A66000260768D7F871
S21401EB5008C03CF0800EC7F808E00AB0BDE8F08FA8
S21401EB6030B40A0003689C6A640A64021500ADB2F8
S21401EB70ED05ED0D2C439C6230BC704701004FF64D
S21401EB80FF700A68526A12F4604F03D11300DB0566
S21401EB90DB0D180080B2704770B40200002000231D
S21401EBA0214CA1422AD2B1F5805F02D0B1F5005FB7
S21401EBB01CD1B1F5805F0CD114680025E66A360CCD
S21401EBC016F00106F6B2002E01D0012028E0002042
S21401EBD026E014680025E66A760C16F00106F6B201
S21401EBE0002E01D001201BE0002019E01468E46922
S21401EBF023000B4214D00124200011E00B4CA1424B
S21401EC000ED21468E46A2300B1F5001F04D15C0239
S21401EC1006D50124200003E01C0201D501242000B2
S21401EC20C0B270BC7047000001000800010020005F
S21401EC3010B411F4405F0DD08A0405D50268D36A7A
S21401EC4053F40033D36217E00268D36A53F4803377
S21401EC50D36211E04A0405D50268936953F00104B2
S21401EC60946109E08A0305D50268136A53F4807338
S21401EC70136201E00268116210BC704770B4CB07E2
S21401EC800DD515000368DC6A2E00F6B2012E03D1FD
S21401EC9054F40076DE6202E034F40076DE628B071E
S21401ECA00DD5150003681C682E00F6B2012E03D19F
S21401ECB054F080061E6002E034F080061E604B07AA
S21401ECC00DD5150003681C682E00F6B2012E03D17F
S21401ECD054F040061E6002E034F040061E600B074A
S21401ECE00DD5150003681C682E00F6B2012E03D15F
S21401ECF054F480461E6002E034F480461E60CB0663
S21401ED000DD515000368DC6A2E00F6B2012E03D17C
S21401ED1054F48076DE6202E034F48076DE628B069E
S21401ED200DD5150003681C682E00F6B2012E03D11E
S21401ED3054F020061E6002E034F020061E604B06EA
S21401ED400DD5150003681C682E00F6B2012E03D1FE
S21401ED5054F080661E6002E034F080661E600B068A
S21401ED600DD5150003685C682E00F6B2012E03D19E
S21401ED7054F080065E6002E034F080065E60CB05EB
S21401ED800DD5150003681C682E00F6B2012E03D1BE
S21401ED9054F010061E6002E034F010061E608B056B
S21401EDA00DD5150003689C682E00F6B2012E03D11E
S21401EDB054F480669E6002E034F480669E604B05E3
S21401EDC00DD5150003681C682E00F6B2012E03D17E
S21401EDD054F480761E6002E034F480761E6011F4EE
S21401EDE0605F0DD0150003689C682E00F6B2012EF8
S21401EDF003D154F001069E6002E0660876009E602C
S21401EE004B040DD5150003681C682E00F6B2012EC2
S21401EE1003D154F000661E6002E034F000661E6006
S21401EE2070BC704770B4020000200B00012B23D089
S21401EE30022B2AD0042B31D0082B38D0102B3FD0F0
S21401EE40202B46D0402B4DD0802B54D0B3F5807F5D
S21401EE505AD0B3F5007F60D0B3F5806F66D0B3F5B6
S21401EE60006F6CD0B3F5805F69D0B3F5005F66D0F4
S21401EE70B3F5804F6CD074E014680023E56AAD05E5
S21401EE8001D501252B0018006BE0146800232568C6
S21401EE902D0601D501252B00180062E01468002319
S21401EEA025686D0601D501252B00180059E0146868
S21401EEB0002325686D0401D501252B00180050E0BC
S21401EEC014680023E56AED0501D501252B0018001D
S21401EED047E0146800232568AD0601D501252B00FF
S21401EEE018003EE01468002325686D0101D5012550
S21401EEF02B00180035E01468002365682D0601D53F
S21401EF0001252B0018002CE0146800232568ED0667
S21401EF1001D501252B00180023E014680023A568FD
S21401EF206D0501D501252B0018001AE01468002391
S21401EF302568ED0501D501252B00180011E01468A0
S21401EF400023A568ED0701D501252B00180008E070
S21401EF501468002325682E0101D501263300180008
S21401EF60FFE7C0B270BC70474FF496414160002184
S21401EF70017200214172002181720221C1720021B9
S21401EF80017300214173032181730121817455218D
S21401EF9001770221C1750021C174FF218161002121
S21401EFA001750021417500218175642180F82010CA
S21401EFB000210174002141740421817702214177E7
S21401EFC00121C177002180F82A10002180F8241041
S21401EFD0002180F82510002180F82610002180F8F5
S21401EFE02710002180F82810002180F82910002120
S21401EFF080F82B10002180F82C1070472DE9FE4F69
S21401F00004000D0000208DF8010026683768780896
S21401F01040003060D4F80080D8F82C0002900298A6
S21401F02050F40040C8F82C0000BF00BF00BF00BF6E
S21401F030029830F40040C8F82C00D4F80090D9F8B3
S21401F0402C000190019850F48040C9F82C0000BFB4
S21401F05000BF00BF00BF019830F48040C9F82C0003
S21401F06029002000FFF71EFA15F1240215F1100100
S21401F0702000FFF7FDFA01208DF80000D4F800A06B
S21401F080DAF800B05BF00100CAF800007FF44051E6
S21401F0902000FFF7CDFDBDE8F78F01000A680023C9
S21401F0A0106B000E10F00700C0B2704701000A682E
S21401F0B00023106B000A10F00700C0B27047000072
S21401F0C00168CA6A52F48043CB6200BF00BF00BF2A
S21401F0D000BF32F48043CB6270472DE9F0430268EB
S21401F0E0126812F00102D2B2012A1FD1002203686F
S21401F0F01C6865086D001D600D000668376B37F4E7
S21401F1004037AC465FFA8CFC5FEA0C4C1CF4403C82
S21401F1105CEA070737635FF0010CD0F800E0DEF821
S21401F120008058F00109CEF800900BE00A00036851
S21401F1301C6B34F440341500EDB22D0415F4403543
S21401F1402C431C63BDE8F08301688A6952F0020310
S21401F1508B61704730B40C00026853682500EDB22D
S21401F160012D03D153F48045556002E033F4804508
S21401F170556030BC70470000F0B401600268D36A85
S21401F18053F40044D46200BF00BF00BF00BF33F495
S21401F1900044D4620468E56A55F48046E66200BF1E
S21401F1A000BF00BF00BF35F48046E6620026076850
S21401F1B03E60F0BC7047000010B50446FEF7DAF872
S21401F1C0204610BD5FEA000C11F8012B00F8012B58
S21401F1D012B111F8012BF9E76046704770B50400CB
S21401F1E0A06840688568022028700020688000209A
S21401F1F0A8800020A8710020A8600020E860A06810
S21401F2004068466802203070002070800020B08080
S21401F2100020B0710020B0600020F0600020A168DE
S21401F220496808700020A1680870200001F036F9CE
S21401F23070BDF8B50400A068007800280AD002283E
S21401F2402AD019D3042800F08E8074D3052800F044
S21401F250A280C9E0200001F025F900280BD020008B
S21401F26000F00CFA002803D00120A168087002E023
S21401F2700620A1680870B7E0200000F043FA0028D5
S21401F28009D0200000F027FAA0684068012101702B
S21401F2900221A2681170A7E0A068C568A068466848
S21401F2A00027310000208A681278012A01D1012244
S21401F2B01000C0B2002806D02800B1681022FEF760
S21401F2C069F801200700FFB2002F08D0A068C068C7
S21401F2D0807903282ED1200000F083FB2AE0A06865
S21401F2E0C568A06846680027310000204A68127881
S21401F2F0012A01D101221000C0B2002806D0280040
S21401F30071681022FEF746F801200700FFB2002FB1
S21401F31010D0A068C0688079012803D10320A168B5
S21401F320087007E0A068C0688079022802D104202E
S21401F330A168087058E0200000F073FA002811D088
S21401F340A0684068406802210170002141800021C8
S21401F350818000218171002181600021C16002212C
S21401F360A268117040E0200000F099FA002811D040
S21401F370A068406840680221017000214180002198
S21401F380818000218171002181600021C1600221FC
S21401F390A268117028E0200000F02FFB002822D080
S21401F3A0A068406880680221017000214180002128
S21401F3B0818000218171002181600021C160A168E6
S21401F3C009690978072906D1200001F067F80020AD
S21401F3D0A168087007E0A06800690078062802D1D5
S21401F3E00220A1680870FFE7F1BD2DE9F34F85B053
S21401F3F0040015001E00109F5FF00108BDF81810EC
S21401F400206800F0DCFF814648464FF6FF7180B267
S21401F410884244D0ADF80690ADF80850039604979C
S21401F42001208DF80A0001208DF80400A0684168CB
S21401F43000204A681278012A01D101221000C0B2C8
S21401F44000282FD10DF1040AA068406800905FF0F3
S21401F450000B00980078002816D0009900204A6812
S21401F4601278012A01D101221000C0B200280BD166
S21401F4700098406851461022FDF78CFF0120009944
S21401F48049680870012083465FFA8BFBBBF1000FC9
S21401F49008D00220A16808750020804602E00420FA
S21401F4A0A16808754046C0B207B0BDE8F08F2DE9E7
S21401F4B0F04F85B004000D0016001F005FF0010834
S21401F4C0290089B2206800F07AFF814648464FF647
S21401F4D0FF7180B2884200F09A802068C068494671
S21401F4E089B200EBC101A06882680023D068D0F819
S21401F4F008C0D0684068BCEB000C604680B2D1F80A
S21401F50000E0BEF802E01EF1070E3EF0070EB0EB7B
S21401F5100E001838012802DB5FF0010E7346DBB2DD
S21401F520002B42D0ADF806900396049702208DF882
S21401F5300A0001208DF80400A068416800204A688E
S21401F5401278012A01D101221000C0B2002861D12F
S21401F5500DF1040AA068406800905FF0000B009867
S21401F5600078002816D0009900204A681278012AEF
S21401F57001D101221000C0B200280BD100984068CA
S21401F58051461022FDF706FF0120009949680870D0
S21401F590012083465FFA8BFBBBF1000F3AD00220B5
S21401F5A0A16808750020804634E003208DF80A0023
S21401F5B0A068416800208A681278012A01D10122D8
S21401F5C01000C0B2002825D10DF1040AA0684068D9
S21401F5D000905FF0000B00980078002816D0009984
S21401F5E000208A681278012A01D101221000C0B2D7
S21401F5F000280BD10098806851461022FDF7CAFEFC
S21401F60001200099896808700120834602E00420E1
S21401F610A16808754046C0B205B0BDE8F08F01008C
S21401F620052288680078052801D1042024E088682E
S21401F6300078032801D102201EE08868007804289B
S21401F64001D1032018E088680078022801D1012042
S21401F65012E088680078062801D106200CE0886848
S21401F6600078002801D1002006E08868007801288B
S21401F67001D1002000E00520C0B2704710B401009F
S21401F6800020002924D08A689268002A20D000220F
S21401F69013000A681289934208DA00220C68E468AB
S21401F6A004EBC304646822605B1CF2E78A68926814
S21401F6B05268503A8C68A468E46822608A68926846
S21401F6C0126840328C68A468E46862600122100007
S21401F6D0C0B210BC704710B504000821A06880684D
S21401F6E0C06840686268D2689047012809D1A0685E
S21401F6F08068C06840680830A1688968C968486041
S21401F700EBE710BD2DE9FE4F050000260024A86892
S21401F710806800684030A9688968C96809688842B5
S21401F7207BD21021A8688068C06800686A68D268C1
S21401F7309047012867D11022E968A8688068C068E8
S21401F74000686B685B689847002852D1EF68686864
S21401F7500290D5F800805FF0000917F10C0B0C2120
S21401F7603800029A126990479BF800100200D2B244
S21401F770914229D10197391D009101990968B1F18A
S21401F780AA3F21D100218A46B8F808108A451BDA1B
S21401F79000990988D8F80C2052F83A200023B2F8CC
S21401F7A000C08E461FFA8EFEF44502D15FF0010CB2
S21401F7B06346DBB2002B02D11AF1010AE4E7D8F85E
S21401F7C00C1001EBCA0189464C46002C11D0E868A2
S21401F7D010F1080109686268116063681B68276890
S21401F7E07F88FF1D37F007073B44AF68BF68FF6897
S21401F7F07B60A8688068C06800681038A968896856
S21401F800C968086009E0A8688068C0680068A968D7
S21401F8108968C9688860012006003000C0B2BDE86A
S21401F820FE8FF8B50500012601270120A968087595
S21401F8302868C068A968C968498800EBC104002C1B
S21401F8401FD060680068002818D020684288D21D42
S21401F85032F00702A868C0688168606800686B6853
S21401F8605B689847002805D10020A9680875002024
S21401F870070006E00320A968087502E00420A968CD
S21401F8800875A868C068C068002805D03800C0B2EE
S21401F890A968C968C96888473000C0B2F2BD2DE9B9
S21401F8A0F04F89B00500012601270120A9680875D7
S21401F8B02868C068A968C968498800EBC104002C9B
S21401F8C07AD020684188C91D4FF6F8700140ADF81E
S21401F8D00010BDF80020A868C0688168A868806824
S21401F8E0C06840686B681B689847002858D16068F4
S21401F8F000680290A8688068C068406808906068E0
S21401F9000790089807990860D5F80C806868006920
S21401F910069001945FF010095FF0000AC346524654
S21401F92049465846FEF78AFDCDF8148018F10400C2
S21401F930049018F10800039018F10C0B5FF0AA3040
S21401F9400599086001980068008804990880019864
S21401F95040680068039908600C214046069A904763
S21401F9608BF800001022E968A8688068C068806883
S21401F9706B681B689847002805D10020A9680875A0
S21401F9800020070002E0029861680860A8688068A5
S21401F990C06880681038A9688968C9688860FFE708
S21401F9A0A8688068C0684068BDF800100844A96867
S21401F9B08968C968486004E00420A96808750020C1
S21401F9C00700A868C068C068002805D03800C0B223
S21401F9D0A968C968C96888473000C0B209B0BDE8DF
S21401F9E0F08F0021826812691176002182681269FF
S21401F9F0117005218268117070472DE9F84F84B0A7
S21401FA0004000025A0680069007800280ED00128AF
S21401FA106AD0022800F0C380042800F0408105283F
S21401FA2000F07981062800F0CD81A2E2200000F0E6
S21401FA30ACFCA16809694860A068006940680028B4
S21401FA4049D0A0680069406801684031C2685160C9
S21401FA5041685039C268916041685039C268116086
S21401FA600021C2685182FF21C26811746668A168CC
S21401FA7009694F685FF001085FF00009B8688145C1
S21401FA800ED24FF4806138685FEA89221044F2682A
S21401FA909047012802D019F10109EFE700208046BE
S21401FAA05FFA88F8B8F1000F0AD10120A168096948
S21401FAB00870A068006940680021C268D16012E041
S21401FAC0A06800694068C068082101740220A16826
S21401FAD00969087007E00420A1680969087607200B
S21401FAE0A1680969087046E26668A0680069476807
S21401FAF0F868007C09282DD0F868007C0A2829D0EF
S21401FB00F868C068B968884221D23868F968C96857
S21401FB108902084480465FEA9820800208F2FF3195
S21401FB20890A8902884203D20820F968488211E0CE
S21401FB304046B1688847002803D00420F968488207
S21401FB4008E0F868C068401CF968C86002E00A204E
S21401FB50F9680874A06800694068C068B0F91200C6
S21401FB6000280BD1A06800694068C068007C0A289C
S21401FB7004D10220A168096908700FE0A068006935
S21401FB804068C068B0F91200002807D00520A168B7
S21401FB90096908760720A16809690870EBE1E6683B
S21401FBA06768A0680069D0F80480D8F80C00007C6B
S21401FBB0082804D0D8F80C00007C0A2852D1D8F8BE
S21401FBC00C00B0F9120000284CD10020D8F80C1017
S21401FBD008745A203070012070700020B070032124
S21401FBE030003A699047F07000208146B9F1040F61
S21401FBF007DA16F8090006EB0901087119F101097F
S21401FC00F4E70196D8F800B000975FF0000A0822E2
S21401FC1001995846009B1B689847002801D101208E
S21401FC2082465FFA8AFABAF1000F16D00196D8F822
S21401FC300400B0F1400B00975FF0000A082201991A
S21401FC405846009B1B689847002801D10120824630
S21401FC500120D8F80C10087408E02020D8F80C1001
S21401FC60488203E02020D8F80C104882A06800697A
S21401FC704068C068B0F91200002808D00620A168C4
S21401FC80096908760720A1680969087006E020005E
S21401FC9000F076F90420A168096908706BE120007C
S21401FCA000F077F900280DD0A06880680021C268AE
S21401FCB0D1600821A2689268D26811740521A268F1
S21401FCC012691170A06800694078062808D10720DB
S21401FCD0A168096908760720A1680969087019E012
S21401FCE0A06800694068C068B0F91200002808D012
S21401FCF00720A168096908760720A16809690870C4
S21401FD0008E0A0680069007E002803D00720A168EB
S21401FD10096908702FE16668A0688768F868007C42
S21401FD2009282DD0F868007C0A2829D0F868C06810
S21401FD30B968884221D23868F968C96889020844D6
S21401FD4080465FEA9820800208F2FF31890A89021C
S21401FD50884203D20820F968488211E04046B1681B
S21401FD608847002803D00420F968488208E0F8682C
S21401FD70C068401CF968C86002E00A20F968087487
S21401FD80A0688068C068B0F9120000280AD1A0688F
S21401FD908068C068007C0A2804D10620A168096929
S21401FDA008700EE0A0688068C068B0F912000028EC
S21401FDB007D00820A168096908760720A1680969A3
S21401FDC00870D8E0D4F80C9060680290A0680069CA
S21401FDD0D0F804A0DAF80C00007C052853D10620E0
S21401FDE0DAF80C1008745A2089F80000042089F803
S21401FDF00100002089F8020003214846029A126990
S21401FE00904789F8030000208346BBF1040F07DA08
S21401FE1019F80B0009EB0B0108711BF1010BF4E754
S21401FE20CDF80090DAF8000010F11806029F5FF096
S21401FE3000080822009930003B689847002801D145
S21401FE40012080465FFA88F8B8F1000F16D0CDF889
S21401FE500090DAF80400B0F12806029F5FF000086F
S21401FE600822009930003B689847002801D10120FC
S21401FE7080460720DAF80C10087408E01020DAF83B
S21401FE800C10488203E01020DAF80C104882E06873
S21401FE90019060680390A068006946683068203069
S21401FEA00090306810F14008F068007C072838D1CF
S21401FEB05FF0080A5FF0000BDDF804905A465146E1
S21401FEC04846FEF7BBFADDF80090C14510D208227D
S21401FED001994846039B1B689847002802D119F1EF
S21401FEE00809F2E7F068408A50F40070F168488229
S21401FEF070682038009070688046009F474516D28B
S21401FF00082201993800039B1B689847002801D1F5
S21401FF100837F3E7F068408A50F40070F1684882C9
S21401FF2005E0F068408A50F40070F1684882A068E5
S21401FF3000694068C068B0F91200002808D009209E
S21401FF40A168096908760720A168096908700FE0A9
S21401FF50A06800694068A16888600020A1680969F6
S21401FF6048600920A1688968C968087401200500ED
S21401FF7001E0012005002800C0B205B0BDE8F08F01
S21401FF8001218268126951700021826812699160AC
S21401FF9070472DE9FE4F04000025A06800694078EF
S21401FFA0012808D002287CD0042800F0A880052863
S21401FFB000F0AF801BE1E6686768A0680069D0F8CA
S21401FFC00480D8F80C00007C012854D1D8F80C0025
S21401FFD0B0F9120000284ED10220D8F80C1008748F
S21401FFE05A203070022070700020B070032130005B
S21401FFF03A699047F07000208146B9F1040F07DA9C
S21402000016F8090006EB0901087119F10109F4E76F
S2140200100196D8F8000010F1080A00975FF0000B6E
S214020020082201995046009B1B689847002801D178
S214020030012083465FFA8BFBBBF1000F16D00196B8
S214020040D8F80400B0F1380A00975FF0000B0822D7
S21402005001995046009B1B689847002801D1012051
S21402006083460320D8F80C10087408E04020D8F81D
S2140200700C10488203E04020D8F80C104882A06892
S21402008000694068C068B0F91200002804D0062053
S214020090A1680969487003E00220A16809694870EE
S2140200A0A5E0A0680069806821680989884221D293
S2140200B02068C068A1680969896800EBC101200050
S2140200C000F099F8002804D00420A1680969487055
S2140200D008E0A0680069007E032803D10620A16814
S2140200E009694870A06800698068401CA1680969AF
S2140200F0886003E00520A1680969487077E020005F
S21402010000F0AAF8002803D00220A1680969487006
S2140201106DE0E6686768A0680069D0F80480D8F8E1
S2140201200C00007C03284ED10420D8F80C1008746A
S2140201305A203070032070700020B0700321300007
S2140201403A699047F07000208146B9F1040F07DA49
S21402015016F8090006EB0901087119F10109F4E71E
S2140201600196D8F8000010F1100A00975FF0000B15
S214020170082201995046009B1B689847002801D127
S214020180012083465FFA8BFBBBF1000F16D0019667
S214020190D8F80400B0F1300A00975FF0000B08228E
S2140201A001995046009B1B689847002801D1012000
S2140201B083460520D8F80C10087408E08020D8F88A
S2140201C00C10488203E08020D8F80C104882A06801
S2140201D000694068C068B0F91200002804D0062002
S2140201E0A1680969487001E001200500FFE72800C0
S2140201F0C0B2BDE8FE8FF8B506000C000027002C42
S21402020027D0B0680069C460B0680069C06800683A
S2140202104188C91D4FF6F87001400D00B0680069AC
S214020220C06840680068002813D02A0092B2F168BD
S214020230B0680069C0684068006873685B68984781
S214020240002804D00320B1680969087601E001207D
S21402025007003800C0B2F2BD2DE9F04F87B00400A7
S2140202600025A0680069C06800684088C01D4FF677
S214020270F8760640320092B2E168A06800694068EB
S214020280C068406863681B689847002874D1A068F5
S2140202900069C068406800680190A068006940680C
S2140202A0C0684768A0680069C068406806900698FB
S2140202B00760D4F80C80606800690590A068006941
S2140202C0C06800905FF010095FF0000AC34652460D
S2140202D049465846FEF7B2F8CDF8108018F10400E9
S2140202E0039018F10800029018F10C0B5FF0AA3088
S2140202F004990860009800680088039908800098AE
S21402030040680068029908600C214046059A9047AA
S2140203108BF800001022E168A06800694068C06897
S214020320806863681B68984700280DD1A06800693A
S2140203304068C068A16809694968C968896810394F
S21402034081600120050009E00198A1680969C96871
S214020350496808600222A3681B691A76A0680069C9
S2140203604068C068A16809694968C9684968320076
S21402037092B21144416003E00220A168096908763E
S2140203802800C0B207B0BDE8F08F10B4010000200C
S21402039000220B681B889A420FDA0B685B6814010E
S2140203A02344DB681B7C092B05D00B685B681401B1
S2140203B02344180001E0521CEBE710BC70472DE9FD
S2140203C0F04303004FF6FF7000241A89521E0225DE
S2140203D092FBF5F51A89561E00273A00D2B2002A79
S2140203E059D10A00D3F80CC0AE461FFA8EFE5CF84E
S2140203F03EE05FF0000CBEF8008091461FFA89F9D5
S214020400C84502D15FF00108C4465FFA8CFCBCF115
S214020410000F03D0280001221700DEE7B4461FFAB9
S2140204208CFC220092B2BCEB020CBCF1020F1CDA6E
S214020430012217000A00D3F80CC0B6461FFA8EFE39
S2140204405CF83EE05FF0000CBEF8008091461FFAB2
S21402045089F9C84502D15FF00108C4465FFA8CFCF0
S214020460BCF1000FB9D03000B7E7DA68AC461FFA25
S2140204708CFC52F83C2012888C461FFA8CFC624593
S21402048002D26A1C140001E06A1E1600A21992B279
S21402049052081500A1E780B2BDE8F0830021826809
S2140204A05170704738B504000025A06840780028CF
S2140204B00BD0022811D00CD3042812D01DD3062844
S2140204C017D012D307281CD021E0200000F00AFB28
S2140204D01DE0200000F01EF819E0200000F026FBC8
S2140204E015E0200000F0E1FD11E0200000F0B7FB6F
S2140204F00DE0200000F099FB09E0200000F088FBE8
S21402050005E0200000F01CFE01200500FFE72800A1
S214020510C0B232BD2DE9F14F88B0002408980068B9
S2140205200088844280F2D782089846680898006855
S2140205304068210100EB0107B046B9465FF0010AA8
S21402054000200500D9F8080085420ED24FF48061DB
S214020550D9F80000AA021044D8F80C2090470128C7
S21402056001D06D1CEEE7002082465FFA8AFABAF1E5
S214020570000F02D00A20F9680874089800684068DC
S21402058021010844C068007CC0B20A2800F0A1829B
S2140205900898C0680790089840680690089800680F
S2140205A04068210108440490402207990498006894
S2140205B0069B5B68984706003000C0B2002840F0F1
S2140205C03081079F0698D0F8108004980590B946A7
S2140205D0C2465FF0000B03214846D0478DF80F0055
S2140205E099F803009DF80F1088420DD199F8000083
S2140205F05A2809D199F80100012805D199F8020074
S214020600002801D1012083465FFA8BFBBBF1000F65
S21402061023D117F10409C2465FF0000B03214846B6
S214020620D0478DF80E0099F803009DF80E10884208
S2140206300DD199F800005A2809D199F8010001282D
S21402064005D199F80200002801D1012083465FFAFD
S2140206508BFBBBF1000F00F0E38001200599C9680F
S214020660087417F10809C2465FF0000B03214846DA
S214020670D0478DF80D0099F803009DF80D108842BA
S2140206800DD199F800005A2809D199F801000228DC
S21402069005D199F80200002801D1012083465FFAAD
S2140206A08BFBBBF1000F23D117F10C09C2465FF09A
S2140206B0000B03214846D0478DF80C0099F803003A
S2140206C09DF80C1088420DD199F800005A2809D1DD
S2140206D099F80100022805D199F80200002801D1F4
S2140206E0012083465FFA8BFBBBF1000F00F0988077
S2140206F003200599C968087417F11009C2465FF00D
S214020700000B03214846D0478DF80B0099F80300EA
S2140207109DF80B1088420DD199F800005A2809D18D
S21402072099F80100032805D199F80200002801D1A2
S214020730012083465FFA8BFBBBF1000F22D117F133
S2140207401409C2465FF0000B03214846D0478DF8D5
S2140207500A0099F803009DF80A1088420DD199F80C
S21402076000005A2809D199F80100032805D199F802
S2140207700200002801D1012083465FFA8BFBBBF101
S214020780000F4DD005200599C968087417F118099D
S214020790C2465FF0000B03214846D0478DF8090099
S2140207A099F803009DF8091088420DD199F80000C7
S2140207B05A2809D199F80100042805D199F80200AF
S2140207C0002801D1012083465FFA8BFBBBF1000FA4
S2140207D022D117F11C09C2465FF0000B03214846DE
S2140207E0D0478DF8080099F803009DF80810884253
S2140207F00DD199F800005A2809D199F80100042869
S21402080005D199F80200002801D1012083465FFA3B
S2140208108BFBBBF1000F03D007200599C96808744B
S21402082057E13000C0B2022811D03000C0B204280E
S2140208300DD03000C0B2072804D1FF200499C96841
S214020840087446E101200499C968488241E14022C1
S2140208500799049840684038069B5B6898470600EC
S2140208603000C0B2002840F03081079F0698D0F8CA
S214020870108004980590B946C2465FF0000B03212B
S2140208804846D0478DF8070099F803009DF80710F0
S21402089088420DD199F800005A2809D199F801002A
S2140208A0012805D199F80200002801D101208346CB
S2140208B05FFA8BFBBBF1000F23D117F10409C24686
S2140208C05FF0000B03214846D0478DF8060099F8E2
S2140208D003009DF8061088420DD199F800005A28A8
S2140208E009D199F80100012805D199F802000028DB
S2140208F001D1012083465FFA8BFBBBF1000F00F0AB
S214020900E38001200599C968087417F10809C246F0
S2140209105FF0000B03214846D0478DF8050099F892
S21402092003009DF8051088420DD199F800005A2858
S21402093009D199F80100022805D199F80200002889
S21402094001D1012083465FFA8BFBBBF1000F23D156
S21402095017F10C09C2465FF0000B03214846D04748
S2140209608DF8040099F803009DF8041088420DD112
S21402097099F800005A2809D199F80100022805D1F1
S21402098099F80200002801D1012083465FFA8BFB0A
S214020990BBF1000F00F0988003200599C96808741F
S2140209A017F11009C2465FF0000B03214846D047F4
S2140209B08DF8030099F803009DF8031088420DD1C4
S2140209C099F800005A2809D199F80100032805D1A0
S2140209D099F80200002801D1012083465FFA8BFBBA
S2140209E0BBF1000F22D117F11409C2465FF0000BCB
S2140209F003214846D0478DF8020099F803009DF877
S214020A00021088420DD199F800005A2809D199F8A7
S214020A100100032805D199F80200002801D101201F
S214020A2083465FFA8BFBBBF1000F4DD0052005997C
S214020A30C968087417F11809C2465FF0000B032153
S214020A404846D0478DF8010099F803009DF801103A
S214020A5088420DD199F800005A2809D199F8010068
S214020A60042805D199F80200002801D10120834606
S214020A705FFA8BFBBBF1000F22D117F11C09C246AD
S214020A805FF0000B03214846D0478DF8000099F826
S214020A9003009DF8001088420DD199F800005A28EC
S214020AA009D199F80100042805D199F80200002816
S214020AB001D1012083465FFA8BFBBBF1000F03D006
S214020AC007200599C968087403E001200499C968DB
S214020AD04882641C22E5022008998968487009B099
S214020AE0BDE8F08FF0B4C1684268036800241D8830
S214020AF0AC4216DA5D68260135442E684036EF6849
S214020B007E606E68503EEF68BE606E68503EEF686C
S214020B103E600026EF687E82FF26EF683E74641C05
S214020B20E5E7012586687570F0BC7047F0B40100F1
S214020B3006208A68507000208A6890600B6800223F
S214020B40002400251888854215DA58682E0130449C
S214020B50C068007C07280CD158682E013044C06853
S214020B60B0F91200002804D1641C58682E013044E3
S214020B7002006D1CE6E7012C01D000200200002ACC
S214020B8004D08868826007208B68587000208B68C3
S214020B901B6958600C6800230025002620888642C0
S214020BA016DA606837013844C068007C07280DDA18
S214020BB0606837013844C068B0F91200002805D1D1
S214020BC0012005006068370138440300761CE5E71B
S214020BD02800C0B2002801D100200300002B15D047
S214020BE0D868007C052806D188680069436003201F
S214020BF08C6860700AE0D868007C052806DA886887
S214020C008068002802D106208C686070F0BC7047AD
S214020C1081688968002904D18168096949688268FF
S214020C209160072182685170704710B403680022F1
S214020C305968002901D059680A00002A0AD081683A
S214020C408A60816889680023CC68E360052384682B
S214020C50637002E008218368597010BC70472DE962
S214020C60F84F86B004006568A0688668F068007C65
S214020C7009282CD0F068007C0A2828D0F068C068C2
S214020C80B168884220D23068F168C968890208448F
S214020C900700B80A800207F2FF31890A89028842F1
S214020CA003D20820F168488211E03800A968884714
S214020CB0002803D00420F168488208E0F068C06883
S214020CC0401CF168C86002E00A20F1680874A06857
S214020CD08068C068B0F91200002803D00820A16816
S214020CE04870DFE1A0688068C068007C0A2840F08F
S214020CF0D9810820A1688968C9680874E0680290EA
S214020D0060680190A068806800900098C068007CC7
S214020D10082840F0C481029D019E009FF868007C6E
S214020D20082803D0F868007C0A284DD1F868B0F984
S214020D301200002848D10020F96808745A2028704A
S214020D40012068700020A8700321280032699047AD
S214020D50E87000208046B8F1040F07DA15F808009C
S214020D6005EB0801087118F10108F4E70395D7F8B6
S214020D700090B2465FF0000B082203994846DAF864
S214020D8000309847002801D1012083465FFA8BFB8A
S214020D90BBF1000F14D003957868B0F14009B24653
S214020DA05FF0000B082203994846DAF800309847AD
S214020DB0002801D1012083460120F968087406E064
S214020DC02020F968488202E02020F9684882DDF88F
S214020DD0089001980390DDF800A0DAF80C00007C79
S214020DE0012857D1DAF80C00B0F91200002851D1C8
S214020DF00220DAF80C1008745A2089F80000022043
S214020E0089F80100002089F8020003214846039A67
S214020E101269904789F8030000208346BBF1040F4D
S214020E2007DA19F80B0009EB0B0108711BF1010B2D
S214020E30F4E74D46DAF8000010F10806039F5FF06B
S214020E4000080822290030003B689847002801D194
S214020E50012080465FFA88F8B8F1000F15D04D469B
S214020E60DAF80400B0F13806039F5FF000080822A3
S214020E70290030003B689847002801D101208046AF
S214020E800320DAF80C10087408E04020DAF80C1098
S214020E90488203E04020DAF80C104882029D019E48
S214020EA0009FF868007C032849D10420F96808747A
S214020EB05A202870032068700020A870032128009A
S214020EC032699047E87000208046B8F1040F07DACE
S214020ED015F8080005EB0801087118F10108F4E797
S214020EE00395386810F11009B2465FF0000B08222D
S214020EF003994846DAF800309847002801D10120C5
S214020F0083465FFA8BFBBBF1000F14D0039578681B
S214020F10B0F13009B2465FF0000B0822039948464A
S214020F20DAF800309847002801D1012083460520D0
S214020F30F968087406E08020F968488202E080209A
S214020F40F9684882DDF8089001980490DDF800A060
S214020F50DAF80C00007C052851D10620DAF80C10CD
S214020F6008745A2089F80000042089F8010000203D
S214020F7089F8020003214846049A1269904789F8C4
S214020F80030000208346BBF1040F07DA19F80B00B2
S214020F9009EB0B0108711BF1010BF4E74D46DAF879
S214020FA0000010F11806049F5FF0000808222900CE
S214020FB030003B689847002801D1012080465FFA3E
S214020FC088F8B8F1000F15D04D46DAF80400B0F1F3
S214020FD02806049F5FF000080822290030003B68BC
S214020FE09847002801D1012080460720DAF80C1025
S214020FF0087408E01020DAF80C10488203E010208B
S214021000DAF80C104882029D01980590009E30681E
S21402101020300390306810F14008F068007C072802
S21402102037D15FF0080A5FF0000BA9465A465146D0
S2140210304846FDF703FADDF80C90C14510D20822A7
S21402104029004846059B1B689847002802D119F1DB
S2140210500809F2E7F068408A50F40070F1684882A6
S21402106070682038039070688046039F474516D202
S214021070082229003800059B1B689847002801D1E2
S2140210800837F3E7F068408A50F40070F168488247
S21402109005E0F068408A50F40070F1684882072044
S2140210A0A168487007B0BDE8F08FF8B5040065681F
S2140210B0A0688668F068007C09282CD0F068007C5E
S2140210C00A2828D0F068C068B168884220D2306802
S2140210D0F168C968890208440700B80A800207F264
S2140210E0FF31890A8902884203D20820F1684882C1
S2140210F011E03800A9688847002803D00420F16868
S214021100488208E0F068C068401CF168C86002E0E7
S2140211100A20F1680874A0688068C068B0F91200F6
S214021120002803D00820A168487008E0A0688068FC
S214021130C068007C0A2802D10720A1684870F1BD69
S21402114081688968002904D0092182689268D26879
S21402115011747047030000200A00511ED2B2002A02
S21402116002D01A881018F7E780F47F4090F0FF004C
S21402117080B2704710B500242000C0B206280FDAED
S2140211804FF40040DFF8DC1B2200D2B221F8120036
S2140211900020DFF8D41B2200D2B28854641CEBE78E
S2140211A04E22DFF8C81B102000F0DEFF0020DFF81A
S2140211B0881C087010BD70B5DFF8B04B4821A01C23
S2140211C0FFF7C8FF218845F2AA52914254D1B4F8DB
S2140211D04C104AF6552291424ED10100B4F84A20EC
S2140211E089B2914248D100210A00D2B2062A73DAA5
S2140211F006220B00DBB253432344DB88DFF8645B32
S2140212000E00F6B225F816300B00DBB25343234429
S2140212105B88DFF8285C0E00F6B225F816300B0065
S214021220DBB202FB03F222449288DFF8143C0D0084
S214021230EDB223F81520DFF80C2C0B00DBB204EB22
S2140212404303DB8C0D00EDB222F815300B00DBB247
S21402125004EB43035B8E0D00EDB202EB4505AB815A
S2140212600B00DBB204EB4303DB8F0D00EDB202EBA7
S21402127045021383491CB7E700210A00D2B2062AA8
S2140212802ADA4FF40042DFF8DC3A0C00E4B223F824
S21402129014200022DFF8A43B0C00E4B223F814204A
S2140212A00022DFF89C3B0C00E4B223F81420DFF89F
S2140212B0942B00230C00E4B222F8143000230C0016
S2140212C0E4B202EB4404A38100230C00E4B202EB76
S2140212D044021383491CD0E770BD38B5DFF88C4A48
S2140212E045F2AA5020804AF65520A4F84C00002564
S2140212F02800C0B2062843DA06202900C9B24143B4
S2140213002144DFF8602A2B00DBB232F81320CA80B1
S2140213102900C9B241432144DFF8202B2B00DBB25F
S21402132032F813204A802900C9B200FB01F020449B
S214021330DFF80C1B2A00D2B231F812108180DFF8D7
S214021340040B2900C9B230F811102A00D2B204EBFD
S2140213504202D1842900C9B200EB410189892A00E0
S214021360D2B204EB420251862900C9B200EB410018
S214021370008B2900C9B204EB4101C8876D1CB7E790
S2140213804821A01CFFF7E6FEA4F84A0031BD38B596
S214021390DFF8A45A2878002813D100F0F4FE0400DF
S2140213A02000C0B2032804D1FFF705FF01202870F1
S2140213B007E02000C0B2042803D10120287000F004
S2140213C0DFFBDFF8E41B0878002814D0DFF8242CB3
S2140213D01088002803D01088401E10800BE00020E2
S2140213E0108000200870FFF778FF4E22DFF87C1985
S2140213F0102000F0A0FE31BDF8B5DFF84C6B307857
S214021400002805D002284ED00FD3032873D073E0ED
S2140214100020DFF8981B08700020DFF8941B087085
S2140214200020DFF8901B087044E20120DFF87C1BE6
S21402143008700120DFF8781B08700120DFF8741BA3
S21402144008700121002000F02EFC0121022000F08D
S2140214502AFCDFF8A40B0021018000214180002134
S2140214608180307840003070002005002800C0B22D
S214021470042817DA0020DFF8C4192A00D2B221F8AD
S21402148012000020DFF8B8192A00D2B221F81200A2
S2140214904FF40040DFF8CC182A00D2B221F812002E
S2140214A06D1CE3E728E0DFF8040B0178DFF8000B99
S2140214B000780143C9B200291CD10020050028008B
S2140214C0C0B2062816DADFF874092900C9B230F865
S2140214D01100DFF86C192A00D2B231F81210401847
S2140214E004002100490889B22800C0B200F0E9FBD6
S2140214F06D1CE4E700E0FFE7DFF8B06A3078012809
S2140215000ED0C0F0E880032848D033D3052800F078
S21402151083806DD3072800F0B980C0F0A380DAE09C
S214021520DFF8D47A3888401C3880DFF81009008843
S21402153000280AD03078400030700020DFF8BC1A4D
S21402154008700021002000F0AEFB388840F6B93162
S214021550884204DADFF810080078002809D0042050
S21402156030700020DFF8941A08700021002000F086
S2140215709AFBB0E0DFF8840A0178491C0170007813
S21402158033280ADB3078401C30700221002000F03D
S2140215908AFB0020DFF8601A08809CE0DFF8587AA1
S2140215A03888401C3880DFF89808008800280AD05F
